:100000000C94237C0C94597C0C94597C0C94528253
:100010000C94597C0C94597C0C94597C0C94597C0C
:100020000C94597C0C94597C0C94597C0C94597CFC
:100030000C94597C0C94597C0C946BC80C94597C8E
:100040000C94597C0C94597C0C94597C0C94597CDC
:100050000C947CA80C94597C0C94597C0C94597C7D
:100060000C94597C0C94DAB50C94597C0C94597C02
:100070000C9411B60C94597C0C94597C0C94597CBA
:100080000C94597C0C94597C0C94597C0C941D82D2
:100090000C94597C0C94597C0C94597C0C94597C8C
:1000A0000C94597C0C94597C0C94597C0C94597C7C
:1000B0000C94BC820C94597C0C94597C0C941D8F2C
:1000C0000C94597C0C94597C0C94597C0C94597C5C
:1000D0000C94597C0C94597C0C94597C0C94597C4C
:1000E0000C94597C0C94597C0C9448B60C94597C13
:1000F0000C94597C0C94597C0C94597C0C94597C2C
:100100000C94597C0C9487820C94597C0C94E88153
:100110000C94597C0C94597C0C94597C0C94597C0B
:100120000C94597C0C94597C0C94597C0C94597CFB
:100130000C94597C0C94667C0C94597C0C94597CDE
:100140000C94597C0C94597C0C94597C0C94A27C92
:100150000C94597C0C94597C0C94597C0C94597CCB
:100160000C946CB50C94597C0C94597C0C94A3B5EC
:100170000C94597C0C94597C0C94597C0C94597CAB
:100180000C94597C0C94597C0C94597C0C94597C9B
:100190000C94597C0C94597C0C94597C0C94597C8B
:1001A0000C94597C0C94597C0C94597C0C94597C7B
:1001B0000C94597C0C94597C0C94597C0C94597C6B
:1001C0000C94597C0C94597C0C94597C0C94597C5B
:1001D0000C94597C0C94597C0C94597C0C94597C4B
:1001E0000C94597C0C94597C0C94597C0C94597C3B
:1001F0000C94597C0C9470D50C94597C16A01BA0BF
:1002000020A0BCA029A02EA033A038A089A043A084
:10021000D6A06CA04CA0AEA052A056A06CA06CA022
:100220006CA06CA05CA05CA061A067A06CA071A099
:1002300077A080A08FA089A0D6A089A08FA095A02C
:100240009AA09FA0A5A0AEA0B3A0BCA0C7A0C1A02B
:10025000C7A0CDA0D6A0DCA0E5A0E1C933CA22CAC0
:1002600018CA08CAB2CA9FCA97CA85CA76CA63CAD8
:1002700056CA3FCAADCB9DCB97CB86CB74CB61CB57
:1002800054CB41CB30CB1BCB10CBFBCAE8CAD4CA72
:10029000C5CAC1CAD1C9BACDB6CDA7CD97CD82CD79
:1002A00073CD5FCD4CCD33CD28CD13CD0FCDF3CC59
:1002B000EFCCDECCC7CCC1CCB7CCA3CC8DCC73CC2F
:1002C00064CC4ECC3DCC27CC1CCC04CCF3CBE0CBC7
:1002D000D3CBC0CBF9C9EBC9C9CDA1D196D186D1B9
:1002E0007DD16DD15FD14ED147D135D127D120D12C
:1002F00014D1FFD0EED0DFD0DAD0CAD0B8D0A6D09B
:100300009AD095D085D071D067D053D042D02FD01D
:1003100022D00FD000D0F3CFF0CFE2CFD2CFBFCFDB
:10032000B1CF9ECF8DCF75CF6BCF56CF46CF2CCFD1
:100330001ECF0DCFF7CEE4CEDACEC6CEB1CE99CE5B
:100340008BCE74CE63CE4DCE43CE2CCE1CCE0ACEF9
:10035000FCCDEACDDBCDAAD1B6D107634236B79B3F
:10036000D8A71A39685618AEBAAB558C1D3CB7CC15
:100370005763BD6DEDFD753EF6177231BF0000008D
:10038000803F08000000BE922449123EABAAAA2A70
:10039000BECDCCCC4C3E00000080BEABAAAAAA3E8B
:1003A00000000000BF000000803F000000000008C7
:1003B0004178D3BB4387D1133D190E3CC3BD428264
:1003C000AD2B3E68EC8276BED98FE1A93E4C80EF22
:1003D000FFBE01C4FF7F3F00000000000C94FCCD75
:1003E0000C949FCA0C9471A00C94A6D00C94DAD0F3
:1003F0000C946BCF0C9482CD0C94C1CC0C949AA02D
:100400000C9453B40C94F3CF0C9473CC0C943B9E8B
:100410000C94E1D10C9495D00C94E1C90C9496D134
:100420000C94EBC90C9447D10C9464CC0C945FCD24
:100430000C948FA00C949ECF0C9461A00C9410CBC4
:100440000C94E2CF0C9438A10C94C7CC0C94C49FAC
:100450000C94CDA00C9443CE0C94B2CA0C94D1C988
:100460000C94C7A00C947DD10C9480A00C944CA04B
:100470000C941ECF0C94A7CD0C9418CA0C94AEA06B
:100480000C94D3CB0C9441CB0C94E8CA0C949BB441
:100490000C94B6CD0C945FD10C9499CE0C94C6CE2E
:1004A0000C9438A00C94BED10C94D6A00C9433CDEF
:1004B0000C9442D00C9461CB0C9420A00C94A3CC4F
:1004C0000C94DACE0C9474CE0C94A1D10C9497CAEF
:1004D0000C94C0CB0C94409A0C9489A00C9473CDCE
:1004E0000C94EACD0C9422D00C9467D00C9427CCB9
:1004F0000C948BCE0C949FA00C948DCC0C9420D19A
:100500000C94AAD10C9428CD0C9433CA0C940FD01F
:100510000C9429A00C94DFD00C9486CB0C942CCE98
:100520000C94E5A00C94B6D10C94DCA00C94F0CF04
:100530000C94C9CD0C9463CE0C940DCF0C94E0CBED
:100540000C9414D10C94DECC0C94C1CA0C9408CA3F
:100550000C9474CB0C946CA00C943DCC0C9486D170
:100560000C94C1A00C9471D00C94B8D00C94B1CF61
:100570000C9485CA0C94A9B40C9497CB0C941CCE03
:100580000C94F7CE0C94FBCA0C9443A00C94B1CEFF
:100590000C94CAD00C94EFCC0C9463B40C942EA0A1
:1005A0000C94DD9E0C94F3CB0C941BA00C94599AE4
:1005B0000C941CCC0C9475CF0C9435D10C94D2CFE8
:1005C0000C9495A00C9404CC0C9427D10C94D5D207
:1005D0000C9454CB0C9433A00C9456CA0C945CA08D
:1005E0000C94389E0C94C5CA0C940ACE0C9497CDEA
:1005F0000C9422CA0C94D1D20C94DBCD0C945B7C6D
:100600000C942FD00C9467A00C9430CB0C9456CF44
:100610000C943FCA0C94DB9E0C94BCA00C944DCE61
:100620000C9400D00C94A5A00C94C09E0C94F9C915
:100630000C94F3CC0C941BCB0C9413CD0C94BACD2E
:100640000C9485D00C942CCF0C9453D00C9446CFA2
:100650000C940FCD0C94ADB60C949AD00C9476CA31
:100660000C946DD10C94FFD00C94ADCB0C944CCD6C
:100670000C94509A0C94BFCF0C948DCF0C944ECC0C
:100680000C94EED00C944ED10C949DCB0C9463CA78
:100690000C94E4CE0C9477A00C947BB40C9416A02C
:1006A0000C9456A00C94B7CC0C94B3A00C94D4CA60
:1006B0000C9452A0000038083A083C083E0878081C
:1006C0007A0838093A093C093E0978097A09380A52
:1006D0003A0A3C0A3E0A000102030405060708091B
:1006E0000A0B0000010203000100010203000100E7
:1006F000010203000000000000000000004008406C
:10070000080000000000000000400940090000004F
:1007100000000000000000000800080008000800B9
:1007200000000000090009000900090000000000A5
:100730000A000A000A000A00000000000000000091
:1007400000000001020304050600000708090A0B67
:100750000C00000D0E0F10000001020408102040D4
:1007600080010204080102040810204080010204F4
:10077000081020408001020408010201010101016A
:100780000101010202020203030303030303030442
:10079000040404040404040505050506060000001D
:1007A000062006400660068006E007090013001ECA
:1007B00000290033003E00490053005E00690073C9
:1007C000007E00890093009E00A800B300BE00C810
:1007D00000D300DD00E700F200FC00070111011B5F
:1007E00001260130013A0144014E01580163016DB7
:1007F00001770180018A0194019E01A801B201BB29
:1008000001C501CE01D801E101EB01F401FE0107B0
:10081000021002190222022B0234023D0246024F4C
:100820000258026002690271027A0282028A02930D
:10083000029B02A302AB02B302BB02C302CA02D2F2
:1008400002D902E102E802F002F702FE0205030CFF
:100850000313031A03210327032E0334033B03412D
:100860000347034D03530359035F0365036A037092
:100870000375037A03800385038A038F0394039827
:10088000039D03A203A603AA03AF03B303B703BBED
:1008900003BF03C203C603C903CD03D003D303D6EA
:1008A00003D903DC03DF03E203E403E703E903EB1B
:1008B00003ED03EF03F103F303F403F603F703F986
:1008C00003FA03FB03FC03FD03FE03FE03FF03FF28
:1008D00003FF03FF03FF03FF03FF03FF03FF03FF08
:1008E00003FE03FE03FD03FC03FB03FA03F803F717
:1008F00003F603F403F203F103EF03ED03EA03E865
:1009000003E603E303E103DE03DB03D903D603D2EB
:1009100003CF03CC03C803C503C103BE03BA03B6A8
:1009200003B203AE03A903A503A0039C039703929C
:10093000038E03890384037E03790374036E0369C2
:100940000363035D03570352034C0345033F03391D
:100950000333032C0325031F03180311030A0303A6
:1009600003FC02F502EE02E602DF02D802D002C862
:1009700002C102B902B102A902A102990291028840
:1009800002800278026F0267025E0255024D024445
:10099000023B0232022902200217020E020402FB6D
:1009A00001F201E801DF01D601CC01C201B901AFBA
:1009B00001A5019C01920188017E0174016A016018
:1009C0000156014C01420137012D01230119010E8D
:1009D000010401FA00EF00E500DA00D000C500BB19
:1009E00000B000A6009B00910086007B00710066AD
:1009F000005B00510046003B00310026001B001048
:100A0000000600FBFFF0FFE6FFDBFFD0FFC6FFBBE9
:100A1000FFB0FFA6FF9BFF90FF86FF7BFF70FF6686
:100A2000FF5BFF51FF46FF3CFF31FF27FF1CFF121A
:100A3000FF07FFFDFEF3FEE8FEDEFED4FEC9FEBFAB
:100A4000FEB5FEABFEA1FE97FE8DFE83FE79FE6F26
:100A5000FE65FE5BFE52FE48FE3EFE35FE2BFE228C
:100A6000FE18FE0FFE06FEFCFDF3FDEAFDE1FDD8DB
:100A7000FDCFFDC6FDBDFDB4FDABFDA3FD9AFD920E
:100A8000FD89FD81FD78FD70FD68FD60FD58FD501C
:100A9000FD48FD40FD38FD31FD29FD22FD1AFD1305
:100AA000FD0CFD04FDFDFCF6FCEFFCE9FCE2FCDBCB
:100AB000FCD5FCCEFCC8FCC1FCBBFCB5FCAFFCA962
:100AC000FCA3FC9DFC98FC92FC8DFC87FC82FC7DC9
:100AD000FC78FC73FC6EFC69FC65FC60FC5BFC57FD
:100AE000FC53FC4FFC4BFC47FC43FC3FFC3BFC38FD
:100AF000FC34FC31FC2EFC2BFC28FC25FC22FC1FCA
:100B0000FC1DFC1AFC18FC16FC14FC12FC10FC0E5C
:100B1000FC0CFC0BFC09FC08FC06FC05FC04FC03BB
:100B2000FC03FC02FC01FC01FC00FC00FC00FC00DE
:100B3000FC00FC00FC01FC01FC02FC02FC03FC04C8
:100B4000FC05FC06FC07FC08FC0AFC0BFC0DFC0F7A
:100B5000FC11FC13FC15FC17FC19FC1CFC1EFC21F1
:100B6000FC24FC27FC29FC2DFC30FC33FC36FC3A31
:100B7000FC3DFC41FC45FC49FC4DFC51FC55FC5A3C
:100B8000FC5EFC63FC67FC6CFC71FC76FC7BFC800F
:100B9000FC85FC8AFC90FC95FC9BFCA1FCA7FCACB2
:100BA000FCB2FCB9FCBFFCC5FCCBFCD2FCD8FCDF22
:100BB000FCE6FCEDFCF3FCFAFC01FD09FD10FD1761
:100BC000FD1FFD26FD2EFD35FD3DFD45FD4DFD5472
:100BD000FD5CFD65FD6DFD75FD7DFD86FD8EFD9762
:100BE000FD9FFDA8FDB1FDB9FDC2FDCBFDD4FDDD2E
:100BF000FDE6FDEFFDF8FD02FE0BFE14FE1EFE27D6
:100C0000FE31FE3AFE44FE4EFE57FE61FE6BFE755F
:100C1000FE7FFE89FE93FE9DFEA7FEB1FEBBFEC5D4
:100C2000FECFFEDAFEE4FEEEFEF9FE03FF0DFF1836
:100C3000FF22FF2DFF37FF42FF4CFF57FF61FF6C84
:100C4000FF77FF81FF8CFF96FFA1FFACFFB6FFC1CE
:100C5000FFCCFFD7FFE1FFECFFF7FF000009001119
:100C6000001A0022002B0033003C0044004C0054CA
:100C7000005C0065006D0075007D0085008C0094AF
:100C8000009C00A400AB00B300BB00C200CA00D1AE
:100C900000D900E000E800EF00F600FD0005010CBF
:100CA0000113011A01210128012F0136013D0144E0
:100CB000014A01510158015F0165016C017201791E
:100CC000017F0186018C01930199019F01A601AC6E
:100CD00001B201B801BE01C401CA01D001D601DCD4
:100CE00001E201E801EE01F401F901FF0105020A48
:100CF00002100216021B02210226022C02310236C9
:100D0000023C02410246024C02510256025B026062
:100D10000265026A026F02740279027E028302880F
:100D2000028D02920297029B02A002A502A902AEC6
:100D300002B302B702BC02C002C502C902CE02D28F
:100D400002D602DB02DF02E302E702EC02F002F469
:100D500002F802FC020003040308030D031003144D
:100D60000318031C032003240328032C032F03333D
:100D70000337033A033E034203450349034D03503F
:100D800003540357035B035E036103650368036B4E
:100D9000036F037203750379037C037F038203856A
:100DA0000388038C038F039203950398039B039E90
:100DB00003A103A403A703A903AC03AF03B203B5C4
:100DC00003B803BA03BD03C003C203C503C803CA03
:100DD00003CD03D003D203D503D703DA03DC03DF4B
:100DE00003E103E403E603E803EB03ED03EF03F29F
:100DF00003F403F603F803FB03FD030004FC03EE16
:100E000003E003D203C503B703A9039C038F038147
:100E100003740367035A034D034003330326031986
:100E2000030C030003F302E602DA02CE02C102B5AC
:100E300002A9029D029002840278026C02610255AE
:100E40000249023D02320226021B020F020402F98D
:100E500001ED01E201D701CC01C101B601AB01A056
:100E60000195018B01800175016B01600156014BF9
:100E700001410137012C01220118010E010401FA80
:100E800000F000E600DC00D300C900BF00B600ACF3
:100E900000A3009900900086007D0074006B006143
:100EA0000058004F0046003D0034002C0023001A7B
:100EB00000110009000000F7FFEFFFE6FFDEFFD69C
:100EC000FFCDFFC5FFBDFFB5FFACFFA4FF9CFF94A6
:100ED000FF8CFF84FF7CFF75FF6DFF65FF5DFF5694
:100EE000FF4EFF46FF3FFF37FF30FF29FF21FF1A6C
:100EF000FF13FF0BFF04FFFDFEF6FEEFFEE8FEE131
:100F0000FEDAFED3FECCFEC5FEBEFEB7FEB1FEAAE3
:100F1000FEA3FE9DFE96FE90FE89FE83FE7CFE767D
:100F2000FE70FE69FE63FE5DFE57FE51FE4AFE4402
:100F3000FE3EFE38FE32FE2CFE26FE21FE1BFE1576
:100F4000FE0FFE09FE04FEFEFDF9FDF3FDEDFDE8DA
:100F5000FDE2FDDDFDD7FDD2FDCDFDC7FDC2FDBD2E
:100F6000FDB8FDB2FDADFDA8FDA3FD9EFD99FD946C
:100F7000FD8FFD8AFD85FD80FD7BFD77FD72FD6D9A
:100F8000FD68FD64FD5FFD5AFD56FD51FD4DFD48B8
:100F9000FD44FD3FFD3BFD36FD32FD2EFD29FD25C7
:100FA000FD21FD1DFD18FD14FD10FD0CFD08FD04C7
:100FB000FD00FDFCFCF8FCF4FCF0FCECFCE8FCE4BF
:100FC000FCE0FCDDFCD9FCD5FCD1FCCEFCCAFCC6A7
:100FD000FCC3FCBFFCBCFCB8FCB4FCB1FCAEFCAA7E
:100FE000FCA7FCA3FCA0FC9DFC99FC96FC93FC8F49
:100FF000FC8CFC89FC86FC83FC7FFC7CFC79FC7609
:10100000FC73FC70FC6DFC6AFC67FC64FC61FC5EBC
:10101000FC5CFC59FC56FC53FC50FC4EFC4BFC4861
:10102000FC45FC43FC40FC3DFC3BFC38FC36FC33FF
:10103000FC31FC2EFC2CFC29FC27FC24FC22FC1F90
:10104000FC1DFC1BFC18FC16FC14FC11FC0FFC0D19
:10105000FC0BFC08FC0FFC1EFC2BFC39FC47FC5570
:10106000FC62FC6FFC7DFC8AFC97FCA5FCB2FCBF1B
:10107000FCCCFCD9FCE6FCF2FCFFFC0CFD18FD25C9
:10108000FD31FD3EFD4AFD56FD63FD6FFD7BFD8795
:10109000FD93FD9FFDABFDB7FDC2FDCEFDDAFDE585
:1010A000FDF1FDFCFD07FE13FE1EFE29FE34FE3F92
:1010B000FE4AFE55FE60FE6BFE76FE81FE8BFE96BE
:1010C000FEA1FEABFEB6FEC0FECAFED5FEDFFEE907
:1010D000FEF3FEFDFE07FF11FF1BFF25FF2FFF386C
:1010E000FF42FF4CFF55FF5FFF69FF72FF7BFF85EB
:1010F000FF8EFF97FFA0FFAAFFB3FFBCFFC5FFCE87
:10110000FFD7FFDFFFE8FFF1FFFAFF000000046FE9
:1011100003CC038203B2038A039E038D038F038AE9
:1011200003850384037E037C037603760373036FD6
:10113000036B036803640360035D035903560352A2
:10114000034E034B034703440340033C0339033579
:101150000332032E032A032703230320031C03184F
:1011600003150311030E030A0307030303FF02FC25
:1011700002F802F502F102EE02EA02E702E302E0FF
:1011800002DC02D902D502D202CE02CB02C702C4CF
:1011900002C002BD02B902B602B202AF02AB02A89F
:1011A00002A402A1029D029A02960293028F028C6F
:1011B000028802850282027E027B0277027402703C
:1011C000026D026902660263025F025C0258025508
:1011D0000252024E024B024702440241023D023AD1
:1011E000023602330230022C022902250222021F9B
:1011F000021B021802150211020E020B0207020462
:10120000020102FD01FA01F701F301F001ED01E92C
:1012100001E601E301DF01DC01D901D501D201CFF3
:1012200001CC01C801C501C201BE01BB01B801B5B5
:1012300001B101AE01AB01A701A401A1019E019A78
:10124000019701940191018D018A01870184018038
:10125000017D017A017701740170016D016A0167F6
:1012600001630160015D015A015701530150014DB5
:10127000014A014701440140013D013A013701346F
:101280000131012D012A012701240121011E011A2A
:10129000011701140111010E010B010801040101E4
:1012A00001FE00FB00F800F500F200EF00EC00E8A2
:1012B00000E500E200DF00DC00D900D600D300D05A
:1012C00000CD00C900C600C300C000BD00BA00B711
:1012D00000B400B100AE00AB00A800A500A2009FC2
:1012E000009C009900960092008F008C0089008677
:1012F00000830080007D007A007700740071006E2A
:10130000006B006800650062005F005C00590056D9
:1013100000530050004D004A004700440041003F88
:10132000003C0039003600330030002D002A002731
:1013300000240021001E001B001800150012000FE1
:10134000000C000A00070004000100FEFFFBFFF88C
:10135000FFF5FFF2FFEFFFEDFFEAFFE7FFE4FFE13C
:10136000FFDEFFDBFFD8FFD5FFD3FFD0FFCDFFCAE5
:10137000FFC7FFC4FFC1FFBFFFBCFFB9FFB6FFB38C
:10138000FFB0FFADFFABFFA8FFA5FFA2FF9FFF9C33
:10139000FF9AFF97FF94FF91FF8EFF8CFF89FF86D6
:1013A000FF83FF80FF7DFF7BFF78FF75FF72FF6F7C
:1013B000FF6DFF6AFF67FF64FF62FF5FFF5CFF591D
:1013C000FF56FF54FF51FF4EFF4BFF49FF46FF43BF
:1013D000FF40FF3EFF3BFF38FF35FF33FF30FF2D5F
:1013E000FF2AFF28FF25FF22FF20FF1DFF1AFF17FE
:1013F000FF15FF12FF0FFF0DFF0AFF07FF04FF029B
:10140000FFFFFEFCFEFAFEF7FEF4FEF2FEEFFEEC3E
:10141000FEEAFEE7FEE4FEE2FEDFFEDCFED9FED7DA
:10142000FED4FED2FECFFECCFECAFEC7FEC4FEC274
:10143000FEBFFEBCFEBAFEB7FEB4FEB2FEAFFEAD0E
:10144000FEAAFEA7FEA5FEA2FE9FFE9DFE9AFE98A6
:10145000FE95FE92FE90FE8DFE8BFE88FE85FE833D
:10146000FE80FE7EFE7BFE78FE76FE73FE71FE6ED3
:10147000FE6CFE69FE66FE64FE61FE5FFE5CFE5A67
:10148000FE57FE54FE52FE4FFE4DFE4AFE48FE45FC
:10149000FE43FE40FE3EFE3BFE38FE36FE33FE318E
:1014A000FE2EFE2CFE29FE27FE24FE22FE1FFE1D20
:1014B000FE1AFE18FE15FE13FE10FE0EFE0BFE09B0
:1014C000FE06FE04FE01FEFFFDFCFDFAFDF7FDF544
:1014D000FDF2FDF0FDEEFDEBFDE9FDE6FDE4FDE1D5
:1014E000FDDFFDDCFDDAFDD7FDD5FDD2FDD0FDCE63
:1014F000FDCBFDC9FDC6FDC4FDC1FDBFFDBDFDBAEF
:10150000FDB8FDB5FDB3FDB0FDAEFDACFDA9FDA779
:10151000FDA4FDA2FDA0FD9DFD9BFD98FD96FD9403
:10152000FD91FD8FFD8CFD8AFD88FD85FD83FD818C
:10153000FD7EFD7CFD79FD77FD75FD72FD70FD6E14
:10154000FD6BFD69FD66FD64FD62FD5FFD5DFD5B9C
:10155000FD58FD56FD54FD51FD4FFD4DFD4AFD4822
:10156000FD46FD43FD41FD3FFD3CFD3AFD38FD35A7
:10157000FD33FD31FD2FFD2CFD2AFD28FD25FD232A
:10158000FD21FD1EFD1CFD1AFD18FD15FD13FD11AD
:10159000FD0EFD0CFD0AFD08FD05FD04FD00FDFF2F
:1015A000FCFBFCFBFCF7FCF4FCF8FCE8FCFDFCD6C7
:1015B000FC09FDBEFC1FFD89FC01FE0000FF03FFCE
:1015C00003FF03FF03FF03FF03FF03FF03FF03FF0B
:1015D00003FF03FF03FF03FF03FF03FF03FF03FFFB
:1015E00003FF03FF03FF03FF03FF03FF03FF03FFEB
:1015F00003FF03FF03FF03FF03FF03FF03FF03FFDB
:1018100003FF03000000FC00FC00FC00FC00FC00D7
:10182000FC00FC00FC00FC00FC00FC00FC00FC00D8
:10183000FC00FC00FC00FC00FC00FC00FC00FC00C8
:10184000FC00FC00FC00FC00FC00FC00FC00FC00B8
:10185000FC00FC00FC00FC00FC00FC00FC00FC00A8
:101A6000FC00FC00FC00FC00FC00FC03001B00363A
:101A700000530071008F00AC00C700DF00F100FFD1
:101A80000008010A0109010401FE00F900F500F453
:101A900000F700FD00060111011F012C013A014869
:101AA00001550162016E017801810186018801857D
:101AB00001800176016901590147013501220110B8
:101AC000010201F900F500FA000901220146017541
:101AD00001AB01EA012C027102B502F70234036B7B
:101AE000039A03BF03D903E803EA03E103CE03B17A
:101AF000038C03610332030003CD029A0268023AA9
:101B0000020F02E801C401A301850169014D012F03
:101B1000011001ED00C7009E00740049002100FE85
:101B2000FFE1FFCFFFC8FFCEFFE2FF03002F0064FD
:101B300000A100E10024016501A401DD0111023DC5
:101B40000262027F0293029F02A3029E0291027D23
:101B50000260023E021602E901B901870155012324
:101B600001F400C7009D0075004F0029000300DA52
:101B7000FFB1FF85FF58FF2AFFFBFECBFE9AFE6BED
:101B8000FE3CFE0EFEE4FDBCFD98FD78FD5CFD45CF
:101B9000FD33FD25FD1EFD1BFD1EFD26FD31FD3F18
:101BA000FD4EFD5EFD6DFD7BFD8AFD98FDA7FDB739
:101BB000FDC7FDD7FDE7FDF6FD06FE16FE27FE3B41
:101BC000FE53FE71FE94FEBFFEF0FE26FF62FFA2F2
:101BD000FFE5FF29006C00AD00EA00220153017C03
:101BE000019C01B201C001C401C001B501A501926F
:101BF000017E016A01580148013C0133012D012A8F
:101C0000012A012E0135013F014B0159016801757F
:101C10000183019101A001B101C601DF01FE012292
:101C2000024A0275029F02C702EA0207031C032749
:101C3000032B03260319030503EA02C802A1027558
:101C40000245021202DE01AD017E01540130011194
:101C500001F900E600D600CC00C400C100C400CAEF
:101C600000D600E600F9000F0125013A014D015EA2
:101C7000016C01770180018501880186018101776E
:101C8000016901570142012A011201FA00E200CA6A
:101C900000B4009D00880072005D004900340021FE
:101CA000000F00FFFFF1FFE4FFD7FFCBFFBFFFB442
:101CB000FFAAFFA2FF9DFF9CFF9EFFA4FFAEFFB8FF
:101CC000FFC3FFCCFFD2FFD6FFD7FFD5FFD3FFD096
:101CD000FFCBFFC6FFBDFFB0FF9DFF84FF63FF3951
:101CE000FF0AFFD5FE9DFE65FE2DFEFBFDCDFDA886
:101CF000FD8DFD79FD70FD70FD78FD87FD99FDADD1
:101D0000FDC0FDD2FDE0FDEBFDF5FDFDFD05FE0E88
:101D1000FE18FE23FE2FFE3AFE43FE4AFE4EFE4F05
:101D2000FE4DFE48FE40FE35FE26FE16FE05FEF484
:101D3000FDE7FDDEFDDDFDE5FDF6FD12FE39FE6A87
:101D4000FEA2FEE1FE22FF62FF9FFFD7FF080032E6
:101D500000550073008B009F00AF00BA00C200C5A1
:101D600000C400BF00B300A3008C006F004A002035
:101D700000F0FFBBFF83FF4BFF15FFE5FEBBFE9AA4
:101D8000FE84FE77FE74FE7BFE8AFEA0FEBBFEDBB9
:101D9000FE00FF28FF53FF81FFB3FFE8FF2000593B
:101DA000009500D20010014E018A01C401FB012BF5
:101DB00002520270028202880282027202580238C3
:101DC000021502F101D001B2019A0188017B017470
:101DD0000172017401790181018A0194019E01A7B8
:101DE00001B001BA01C501D201E401FA0113022FC9
:101DF000024C0267027F0292029E02A302A0029698
:101E00000285026F02530233021002EB01C4019CEF
:101E10000173014A012001F400C8009B006D0041DC
:101E2000001500EBFFC4FFA1FF81FF67FF50FF3EDD
:101E3000FF31FF25FF1CFF13FF0AFF01FFF6FEE83D
:101E4000FED6FEC1FEA7FE88FE66FE3FFE16FEEA37
:101E5000FDBEFD93FD6AFD44FD22FD03FDE8FCD1BE
:101E6000FCBBFCA6FC92FC7DFC68FC52FC3DFC2902
:101E7000FC18FC0BFC03FC00FC05FC13FC2BFC4CCD
:101E8000FC78FCAEFCEBFC30FD77FDBEFD05FE46AC
:101E9000FE82FEB6FEE2FE05FF1DFF2BFF2DFF2595
:101EA000FF12FFF7FED4FEA9FE7AFE47FE12FEDC0B
:101EB000FDA7FD75FD48FD21FD03FDECFCDEFCD713
:101EC000FCD6FCD9FCDFFCE7FCF0FCFAFC03FD0BC4
:101ED000FD14FD1BFD23FD2BFD34FD3FFD4CFD5C82
:101EE000FD70FD86FD9FFDBCFDDBFDFCFD21FE4779
:101EF000FE70FE9AFEC5FEF0FE18FF3EFF5FFF7902
:101F0000FF8DFF98FF9EFF9EFF9AFF94FF90FF902A
:101F1000FF94FFA0FFB1FFCBFFEAFF0600240043C0
:101F20000060007D009B00BA00D900F80016013562
:101F300001550176019601B501D401F3011102307A
:101F4000024E026B028702A302BE02D802F102090E
:101F500003200337034C036003730385039603A533
:101F600003B303BF03CB03D603E003E803EE03F49C
:101F700003F803FC03FE0300040004FE03FB03F765
:101F800003F303F103EE03E903E103D803D003C92C
:101F900003C203B903AE03A3039903900387037C31
:101FA000036F03630358034E03430336032A031FDF
:101FB0000314030A03FE02F202E602DC02D102C5A8
:101FC00002B802AC02A20298028D02810276026B74
:101FD00002620258024C02410237022D0224021909
:101FE000020F020602FE01F401EA01E001D801D06D
:101FF00001C801BE01B501AC01A5019D0195018D8E
:102000000185017E0177016F01680161015A015369
:10201000014B0145013E01380131012A0123011E16
:1020200001180112010B010501FF00F900F300EE98
:1020300000E800E200DC00D500D000CB00C500C005
:1020400000B900B300AD00A700A2009C009600906C
:10205000008A0084007F00790073006D00670061D2
:10206000005C0056005000490043003D003800323B
:10207000002B0025001F00190013000E00070001AF
:1020800000FAFFF4FFEEFFE8FFE2FFDCFFD5FFCF31
:10209000FFC8FFC2FFBCFFB6FFB0FFA9FFA2FF9CB5
:1020A000FF97FF91FF8BFF84FF7EFF78FF71FF6B2F
:1020B000FF65FF5FFF59FF53FF4DFF47FF41FF3BA8
:1020C000FF35FF2EFF28FF22FF1CFF16FF10FF0920
:1020D000FF03FFFDFEF8FEF2FEECFEE6FEDFFEDA99
:1020E000FED4FECEFEC7FEC1FEBBFEB5FEAFFEA90E
:1020F000FEA2FE9CFE96FE90FE8AFE84FE7EFE7888
:10210000FE71FE6AFE63FE5EFE58FE52FE4BFE440A
:10211000FE3EFE38FE32FE2CFE25FE1EFE18FE128E
:10212000FE0CFE05FEFFFDF9FDF2FDECFDE6FDDF18
:10213000FDD9FDD3FDCCFDC6FDC0FDBAFDB4FDAD9E
:10214000FDA6FDA0FD9AFD95FD8FFD89FD82FD7C1C
:10215000FD77FD72FD6CFD66FD60FD5BFD56FD5279
:10216000FD4DFD47FD42FD3DFD39FD34FD30FD2CAB
:10217000FD27FD22FD1EFD1BFD18FD14FD10FD0CAD
:10218000FD09FD07FD05FD03FD01FDFEFCFCFCFB5B
:10219000FCF9FCF8FCF7FCF7FCF7FCF6FCF7FCF7A5
:1021A000FCF8FCF9FCFBFCFCFCFFFC01FD05FD0858
:1021B000FD0CFD11FD15FD1BFD21FD28FD2EFD363D
:1021C000FD3EFD47FD52FD5DFD68FD73FD80FD8F09
:1021D000FD9EFDAEFDBEFDCFFDE1FDF4FD08FE1C44
:1021E000FE32FE49FE60FE78FE91FEAAFEC5FEE0CC
:1021F000FEFCFE18FF35FF52FF71FF8FFFADFFCBD6
:10220000FFEBFF0B002A00490067008500A300C117
:1022100000DF00FC00180134014F01690182019ABE
:1022200001B101C701DC01F00103021502260235EC
:1022300002430250025B0266026F0276027D028256
:102240000287028A028D028E028E028D028A028825
:1022500002850280027A0274026D0266025E0255F5
:10226000024B02410237022C02210215020902FD33
:1022700001F101E401D801CB01BE01B001A201943A
:102280000187017A016D015F015001420136012988
:10229000011C010F010201F400E700DB00CE00C2C7
:1022A00000B500A8009D00920087007C00700064CB
:1022B0000059004F0045003B00300026001C001371
:1022C0000009000000F7FFEFFFE6FFDEFFD6FFCEBC
:1022D000FFC5FFBDFFB4FFACFFA5FF9EFF97FF8FBB
:1022E000FF87FF80FF79FF74FF6DFF66FF5EFF5879
:1022F000FF52FF4DFF46FF3FFF38FF32FF2DFF2704
:10230000FF21FF1BFF14FF0FFF0AFF05FFFFFEF970
:10231000FEF3FEEEFEE8FEE2FEDCFED6FED1FECCD3
:10232000FEC7FEC1FEBBFEB6FEB1FEACFEA6FEA021
:10233000FE9BFE97FE92FE8CFE86FE81FE7CFE7763
:10234000FE73FE6EFE69FE63FE5FFE5AFE56FE528F
:10235000FE4EFE49FE45FE41FE3DFE39FE35FE3194
:10236000FE2EFE2BFE28FE25FE23FE20FE1EFE1C5A
:10237000FE1AFE19FE18FE17FE17FE17FE18FE19AC
:10238000FE1AFE1BFE1DFE1FFE22FE25FE29FE2E4E
:10239000FE34FE3AFE40FE46FE4EFE56FE5FFE68EE
:1023A000FE72FE7DFE89FE97FEA4FEB2FEC1FED146
:1023B000FEE2FEF4FE06FF18FF2DFF42FF58FF6EFF
:1023C000FF85FF9DFFB6FFD0FFEBFF03000E001956
:1023D0000023002E00380042004D00580062006DBE
:1023E00000770082008C009600A100AB00B500BF12
:1023F00000C800D200DC00E500EF00F80001010A8F
:102400000113011C0125012E0136013F0147015036
:1024100001580160016801700178017F0187018E18
:102420000196019D01A401AC01B201B901C001C72F
:1024300001CE01D401DB01E101E701ED01F301F976
:1024400001FF0105020B02110216021C02210226E5
:10245000022C02310236023B02400245024A024F80
:1024600002540259025E02620267026C0270027537
:102470000279027E02820287028B028F0294029806
:10248000029C02A102A502A902AD02B202B602BAE2
:1024900002BE02C202C602CA02CE02D202D602DACC
:1024A00002DF02E202E602EA02EE02F202F602FABB
:1024B00002FE020103050309030C031003140317B2
:1024C000031B031E032203250328032B032F0332C0
:1024D00003350338033B033E0341034403460349EA
:1024E000034B034E0351035303560359035C035F2D
:1024F00003630367036B036F03730378037D038335
:102500000388038E0394039A03A003A603AD03B3C9
:1025100003B903C003C603CC03D103D703DC03E133
:1025200003E503EA03EE03F103F403F703FA03FC04
:1025300003FD03FE03FF03000400040004FF03FE89
:1025400003FD03FC03FA03F803F603F303F103EEC0
:1025500003EB03E703E403E003DC03D803D403CF76
:1025600003CA03C603C003BB03B603B003AA03A494
:10257000039E03980391038A0383037C0375036D11
:102580000365035D0355034C0344033B03320328F7
:10259000031F0315030B030103F702EC02E102D74B
:1025A00002CC02C002B502AA029E02930287027BFD
:1025B000026F02630257024A023E023202250219EA
:1025C000020D020002F401E701DB01CE01C201B5F8
:1025D00001A9019D019001840178016C0160015401
:1025E0000148013C013001240119010D010101F6EE
:1025F00000EB00DF00D400C900BE00B300A8009DBE
:1026000000930088007E00730069005F0055004A57
:1026100000400037002D002300190010000600FCC8
:10262000FFF2FFE9FFDFFFD5FFCBFFC1FFB7FFAE32
:10263000FFA4FF9BFF91FF88FF7EFF75FF6CFF6289
:10264000FF59FF50FF47FF3EFF35FF2CFF23FF1AC6
:10265000FF11FF08FFFFFEF7FEEEFEE5FEDDFED4F4
:10266000FECBFEC3FEBAFEB1FEA9FEA0FE98FE8F11
:10267000FE86FE7EFE75FE6DFE64FE5CFE53FE4A27
:10268000FE42FE39FE31FE28FE1FFE17FE0EFE063C
:10269000FEFDFDF4FDECFDE3FDDBFDD2FDCAFDC159
:1026A000FDB8FDB0FDA7FD9FFD96FD8EFD85FD7D6E
:1026B000FD74FD6CFD64FD5BFD53FD4BFD43FD3B77
:1026C000FD33FD2BFD23FD1BFD13FD0BFD04FDFC68
:1026D000FCF5FCEDFCE6FCDFFCD8FCD1FCCAFCC33D
:1026E000FCBDFCB6FCB0FCAAFCA3FC9DFC98FC92D3
:1026F000FC8CFC87FC82FC7CFC78FC73FC6EFC6A26
:10270000FC65FC61FC5DFC5AFC56FC53FC4FFC4C28
:10271000FC49FC47FC44FC42FC40FC3EFC3CFC3BCE
:10272000FC39FC38FC37FC37FC36FC36FC35FC3514
:10273000FC36FC36FC37FC37FC38FC39FC3BFC3CF7
:10274000FC3EFC3FFC41FC44FC46FC48FC4BFC4E80
:10275000FC50FC54FC57FC5AFC5EFC61FC65FC69B7
:10276000FC6DFC71FC75FC79FC7EFC82FC87FC8CAA
:10277000FC90FC95FC9AFC9FFCA4FCAAFCAFFCB46A
:10278000FCBAFCBFFCC4FCCAFCD0FCD5FCDBFCE002
:10279000FCE6FCECFCF2FCF7FCFDFC02FD08FD0D88
:1027A000FD11FD16FD1AFD1EFD21FD24FD26FD284F
:1027B000FD2AFD2BFD2CFD2CFD2DFD2DFD2DFD2CD1
:1027C000FD2CFD2CFD2BFD2BFD2BFD2BFD2BFD2BC7
:1027D000FD2CFD2DFD2EFD30FD32FD34FD37FD3A83
:1027E000FD3DFD41FD45FD4AFD4EFD54FD59FD5F9A
:1027F000FD65FD6BFD72FD78FD7FFD86FD8DFD9510
:10280000FD9CFDA4FDABFDB3FDBBFDC3FDCBFDD326
:10281000FDDBFDE3FDECFDF4FDFCFD05FE0EFE160B
:10282000FE1FFE28FE31FE3AFE43FE4DFE56FE5FC1
:10283000FE69FE73FE7DFE87FE91FE9BFEA6FEB046
:10284000FEBBFEC5FED0FEDBFEE6FEF1FEFDFE0891
:10285000FF13FF1FFF2AFF36FF41FF4DFF58FF64A4
:10286000FF70FF7BFF87FF92FF9EFFA9FFB5FFC0B0
:10287000FFCCFFD7FFE2FFEDFFF8FF0000030010E1
:102880000029003C004900550061006F0082009A59
:1028900000B300C600D500E200EA00EC00E700E467
:1028A00000E300DF00D900D100CC00C500B900ACC6
:1028B000009F009300860079006D00650060006055
:1028C00000670075008A00A700CA00F3001F014CD2
:1028D0000175019701B401D101EF010C0225023805
:1028E0000244024A024D024D024B024A024E025A73
:1028F000026D0285029E02B802D502FA0225035338
:10290000037D03A503C903E703FB030004FA03ECFB
:1029100003DB03C603AF03990389037C036F0360E2
:10292000034C0336031D030203E702CF02BB02ABD5
:10293000029D0291028302730262024E0239022258
:10294000020B02F501DE01C701B2019E018D017A81
:1029500001630148012C010D01ED00C900A4007FB5
:10296000005B0036001000E8FFBFFF97FF6FFF4BD2
:10297000FF2DFF15FFFFFEEEFEE4FEDFFED7FEC6D5
:10298000FEB2FE9BFE81FE5FFE36FE0EFEE6FDBD44
:10299000FD8FFD5EFD2DFDFFFCD6FCB6FC9BFC848F
:1029A000FC73FC6AFC69FC6EFC7AFC8BFC9FFCB13E
:1029B000FCBDFCC4FCC9FCCEFCD5FCDEFCE9FCF68D
:1029C000FC02FD07FD05FDFDFCF2FCE6FCD9FCCF99
:1029D000FCC7FCC0FCBBFCBAFCBFFCCAFCDAFCF3C5
:1029E000FC14FD3AFD5CFD79FD95FDB2FDCFFDEADD
:1029F000FDFEFD06FEFEFDEAFDD6FDC3FDB2FDA017
:102A0000FD8DFD7CFD6EFD68FD68FD6BFD70FD7A42
:102A1000FD8AFDA0FDB5FDC9FDDCFDEDFDFBFD065C
:102A2000FE13FE23FE33FE43FE52FE5FFE6BFE7777
:102A3000FE85FE93FEA3FEB4FEC4FED3FEE6FEFDBD
:102A4000FE13FF26FF34FF45FF5EFF81FFA9FFD382
:102A5000FFFBFF1F003B004E005B00660070007E26
:102A6000008F00A500BB00CC00D800E000E600EE1F
:102A700000F900070111011501160113010B01FEF8
:102A800000EF00E400DC00D500CD00C300B900ACCD
:102A9000009F0094008F008F008C008800800074DD
:102AA0000063004C0030001200F4FFD6FFBBFFA40F
:102AB000FF8FFF7DFF6EFF63FF5AFF54FF51FF54EE
:102AC000FF5EFF6AFF76FF81FF89FF89FF82FF7645
:102AD000FF6EFF6BFF69FF64FF5CFF59FF57FF54F8
:102AE000FF4FFF4DFF52FF59FF62FF73FF8EFFAD97
:102AF000FFC9FFE4FF01002100440067008800A235
:102B000000B000BE00CE00DF00E400D700C900C066
:102B100000C500C200B800AD00B200C700DD00E88B
:102B200000E500E700EF00FF0005010201010106DA
:102B30000115012F014A015B015801540168017818
:102B4000017B016C0164016D0174017D0187018AC3
:102B50000188018B01910196019101A101CB01ED49
:102B600001050215023102480247023B0234023ECF
:102B7000025802750280027A026C0270027F02849F
:102B8000027B026702510242023A022B020E02E964
:102B900001DF01E101DA01BC018D0166014601346A
:102BA0000136013B0132011A01FE00E900C2008931
:102BB0000048000F00E5FFC1FFA1FF80FF61FF4B50
:102BC000FF45FF45FF4BFF58FF75FF9DFFBFFFDF30
:102BD000FFFFFF1D0033003C004000420043004067
:102BE00000360024000B00F4FFE9FFEAFFF1FFF7D5
:102BF000FFFDFF0D002D0057008100A300BD00DE8A
:102C000000090139015D0170017901750166014614
:102C1000011901E200A50067002E00F9FFC4FF8F33
:102C2000FF60FF3AFF17FFF8FEDFFECEFEC3FEBCDB
:102C3000FEB4FEA5FE8BFE6CFE4BFE27FEFEFDD114
:102C4000FDAAFD87FD63FD3FFD1DFD01FDEBFCE0E1
:102C5000FCE1FCEAFCF8FC10FD30FD4FFD64FD7565
:102C6000FD92FDB6FDDDFD01FE20FE3DFE55FE6739
:102C7000FE75FE7EFE86FE8FFE9BFEAAFEBBFECC90
:102C8000FEDCFEE9FEF8FE0CFF24FF3BFF4EFF6773
:102C9000FF88FFABFFC8FFDCFFECFFFAFF06000B6D
:102CA000000600F6FFE2FFD1FFC6FFBCFFB4FFB194
:102CB000FFB2FFB7FFBDFFC5FFD0FFE4FF01002853
:102CC00000510075009600AE00BC00BD00B400A924
:102CD0000095007D00680058004E003F002F001F47
:102CE000000E00FEFFEFFFE6FFE5FFE7FFEBFFF062
:102CF000FFF1FFEEFFEBFFE7FFE0FFD3FFC8FFC0F0
:102D0000FFB8FFABFF9AFF8CFF84FF82FF83FF8732
:102D1000FF8DFF94FF9DFFA7FFB3FFBFFFCBFFD643
:102D2000FFE1FFEBFFF4FFFBFFFDFF07000B000FD0
:102D3000001300150013000E00090008000A000C23
:102D400000100019002C0049006F009F00D7000CF4
:102D5000013F017401AF01EB012A026B02AA02E6F6
:102D600002200354038503B203D503EE03FD0300E1
:102D700004FB03EB03D003AF038A036003330301B7
:102D800003C8028F0256022002EA01BA018E0163D3
:102D9000013C011A01FC00E500D700D100D400DDA0
:102DA00000EE0007012501480171019D01C801F3F2
:102DB000011A02400264028902AC02CF02EC02FF57
:102DC000020A03110315031603160316031603174D
:102DD000031803190319031C0322032B03320336C0
:102DE00003370335032F03250316030203EA02CD3D
:102DF00002AA0285025D0230020402D601A301701C
:102E0000013B010501CC00970064003100FCFFC3C9
:102E1000FF87FF4DFF15FFDAFEA1FE6BFE3BFE13A1
:102E2000FEF3FDD9FDC4FDB5FDA9FDA0FD9AFD95FC
:102E3000FD93FD95FD9AFD9FFDA6FDACFDB1FDB690
:102E4000FDBAFDBDFDC0FDC4FDCBFDD1FDD5FDD658
:102E5000FDD6FDD4FDD1FDCBFDC2FDB7FDADFDA17D
:102E6000FD93FD83FD70FD5CFD48FD33FD1DFD08F8
:102E7000FDF4FCE1FCD1FCC5FCBCFCB6FCB3FCB32E
:102E8000FCB5FCBBFCC3FCD1FCE3FCF8FC11FD2C45
:102E9000FD4CFD72FD9AFDC4FDEEFD19FE42FE6B78
:102EA000FE94FEBBFEE1FE07FF2BFF4DFF6EFF8C85
:102EB000FFA6FFBBFFCCFFD8FFDFFFE2FFE3FFE28F
:102EC000FFDFFFDBFFD6FFCFFFC7FFBFFFB6FFACC3
:102ED000FFA1FF96FF89FF7CFF6EFF5FFF4DFF3A6A
:102EE000FF28FF18FF08FFF9FEEAFEDCFECEFEC158
:102EF000FEB6FEAEFEABFEAFFEBAFECAFEDCFEF4D0
:102F0000FE13FF39FF5FFF84FFABFFD3FFFEFF2BF4
:102F10000056008000AB00D200F7001A013C015AB5
:102F20000174018B019D01AC01B801C101C601CA48
:102F300001CC01CD01CC01CA01C701C301BD01B65D
:102F400001AE01A4019C0194018B017F0172016318
:102F500001520141013201230114010401F400E690
:102F600000DC00D400CD00C500BF00BC00BB00BC2D
:102F700000BD00BE00BF00BF00BE00BC00B800B472
:102F800000B200B000AB00A3009C00960091008D41
:102F9000008800840080007C00790078007700774A
:102FA00000770079007D0083008A0094009F00ABC9
:102FB00000B900C700D500E300F100FF000D0119C2
:102FC0000124012B0131013201300128011D010EC4
:102FD00001FD00E800CF00B40097007A005E0043D6
:102FE000002B001400FEFFE8FFD7FFCBFFC3FFC29A
:102FF000FFC8FFD1FFDDFFEBFFFEFF13002A0040FB
:103000000055006B0081009700AB00BC00CB00D6E0
:1030100000DF00E400E400E200DF00DA00D500CFCA
:1030200000C800C000B900B200AC00A600A300A315
:1030300000A400A500A300A1009F009E009B009794
:103040000092008A00810077006B005F0050003F13
:10305000002D001C000B00FBFFEBFFDCFFCFFFC4CB
:10306000FFBBFFB6FFB5FFB7FFBBFFC1FFC9FFD373
:10307000FFDDFFE6FFF0FFFAFF03000C0012001572
:10308000001500130010000B000500FEFFF5FFEA1D
:10309000FFE0FFD5FFCBFFC0FFB5FFAAFF9FFF9664
:1030A000FF8EFF88FF83FF7FFF7CFF7BFF7DFF811B
:1030B000FF86FF8BFF8FFF94FF98FF9EFFA5FFAE5B
:1030C000FFB7FFBEFFC4FFC9FFCDFFD1FFD6FFDAB8
:1030D000FFDEFFE1FFE3FFE6FFE9FFEDFFF2FFF6B2
:1030E000FFFAFFFCFFFCFFFBFFF8FFF7FFF8FFFA1A
:1030F000FFFBFFFAFFF8FFF6FFF4FFF2FFEFFFEB35
:10310000FFE5FFDDFFD3FFCAFFC0FFB6FFADFFA2A3
:10311000FF93FF80FF6EFF5DFF4FFF43FF3AFF34D9
:10312000FF31FF32FF34FF35FF37FF39FF3CFF40EF
:10313000FF44FF48FF4BFF4CFF4AFF48FF45FF415C
:10314000FF3DFF38FF30FF25FF17FF06FFF1FEDAD6
:10315000FEC1FEA5FE88FE69FE48FE27FE06FEE6CD
:10316000FDCAFDB2FD9BFD84FD70FD5EFD4EFD447C
:10317000FD41FD44FD4EFD5EFD73FD8CFDA8FDC8C7
:10318000FDEDFD13FE37FE59FE78FE9AFEBFFEDE12
:10319000FEF6FE08FF15FF1DFF1FFF1FFF1AFF0FA2
:1031A000FFFEFEE8FECFFEB5FE9CFE87FE75FE65C7
:1031B000FE56FE4AFE44FE44FE4CFE5EFE78FE9342
:1031C000FEB0FECEFEEFFE13FF37FF57FF74FF8FFA
:1031D000FFA8FFBFFFD7FFECFFFDFF0C001F003172
:1031E0000043005600680079008B009D00AE00BFD0
:1031F00000D000E100F10002011201210131014083
:10320000014F015E016D017B0189019701A401B1AC
:1032100001BE01CB01D701E301EF01FB0106021161
:10322000021C02260231023B0245024E0258026194
:10323000026A0273027C0284028D0295029D02A53D
:1032400002AC02B402BB02C202CA02D102D802DF3F
:1032500002E502EC02F302F902000307030D031377
:10326000031A03200326032C03320338033E0344CE
:10327000034A03500356035C03610367036D037243
:103280000378037D03820387038C03910396039ADB
:10329000039F03A303A703AB03AF03B303B703BBAE
:1032A00003BE03C203C503C803CB03CE03D103D4BB
:1032B00003D603D903DB03DE03E003E203E403E602
:1032C00003E803E903EB03EC03EE03EF03F003F180
:1032D00003F203F303F403F403F503F503F503F535
:1032E00003F503F503F403F403F303F203F103F02E
:1032F00003EF03EE03EC03EB03E903E803E603E467
:1033000003E203E003DE03DC03D903D703D403D2D3
:1033100003CF03CC03C803C503C103BD03B903B581
:1033200003B103AC03A703A2039D03970392038C8D
:1033300003860380037A0373036C0366035E0357FB
:1033400003500348034003390330032803200317C5
:10335000030E030503FC02F302EA02E002D602CCEC
:1033600002C302B802AE02A4029A028F0285027B57
:1033700002700265025B02500246023B02300225E7
:10338000021B0210020402F901EE01E201D601CA99
:1033900001BD01B101A50198018C017F0173016696
:1033A0000159014D01410135012A011E0113010896
:1033B00001FD00F300E900DF00D500CB00C100B73C
:1033C00000AD00A4009A00900086007C00730069A4
:1033D00000600056004D0044003B003200290020F0
:1033E000001800100008000000F8FFF1FFE9FFE2FC
:1033F000FFDBFFD4FFCEFFC7FFC1FFBAFFB4FFAEB4
:10340000FFA8FFA2FF9CFF96FF91FF8BFF86FF8026
:10341000FF7BFF76FF71FF6DFF68FF64FF60FF5C5D
:10342000FF58FF55FF52FF4EFF4BFF48FF44FF413F
:10343000FF3EFF3AFF36FF33FF2FFF2AFF26FF2113
:10344000FF1CFF18FF13FF0EFF09FF04FFFFFEFA2A
:10345000FEF5FEF1FEECFEE8FEE3FEDFFEDBFED74E
:10346000FED3FED0FECCFEC8FEC4FEC1FEBDFEB93A
:10347000FEB5FEB2FEAEFEAAFEA6FEA2FE9FFE9B1B
:10348000FE97FE94FE90FE8DFE89FE86FE83FE80F2
:10349000FE7DFE7AFE77FE74FE72FE6FFE6DFE6AA2
:1034A000FE68FE66FE64FE62FE60FE5EFE5DFE5B22
:1034B000FE5AFE58FE57FE56FE54FE54FE53FE5270
:1034C000FE51FE51FE50FE50FE50FE50FE50FE5189
:1034D000FE51FE51FE52FE53FE53FE54FE55FE5663
:1034E000FE57FE58FE59FE5AFE5BFE5CFE5EFE5F16
:1034F000FE60FE61FE63FE64FE65FE66FE68FE69B8
:10350000FE6AFE6BFE6CFE6DFE6EFE6FFE6FFE7061
:10351000FE71FE71FE72FE73FE73FE73FE74FE7426
:10352000FE74FE74FE74FE74FE74FE74FE73FE730D
:10353000FE72FE71FE6FFE6EFE6CFE69FE67FE643B
:10354000FE61FE5EFE5AFE56FE52FE4EFE4AFE45ED
:10355000FE40FE3BFE36FE31FE2CFE26FE21FE1B0B
:10356000FE15FE0FFE08FE02FEFBFDF4FDEDFDE77D
:10357000FDE0FDD8FDD1FDCAFDC2FDBAFDB3FDAB36
:10358000FDA3FD9BFD92FD89FD81FD78FD6EFD652E
:10359000FD5BFD51FD46FD3CFD32FD27FD1CFD118F
:1035A000FD06FDFBFCF0FCE5FCDBFCD0FCC5FCBB38
:1035B000FCB1FCA7FC9DFC93FC8AFC80FC77FC6EB4
:1035C000FC65FC5DFC55FC4EFC46FC3FFC39FC33C5
:1035D000FC2DFC28FC22FC1EFC19FC15FC11FC0E29
:1035E000FC0AFC07FC04FC02FC00FC00FC00FC00E4
:1035F000FC00FC00FC00FC00FC00FC00FC00FC00EB
:10360000FC00FC03FC07FC0BFC10FC15FC1BFC2263
:10361000FC29FC30FC38FC41FC49FC53FC5CFC6799
:10362000FC71FC7CFC88FC93FCA0FCADFCBAFCC7E4
:10363000FCD5FCE3FCF2FC01FD10FD20FD30FD405B
:10364000FD51FD62FD73FD84FD96FDA8FDBAFDCC24
:10365000FDDFFDF2FD05FE18FE2BFE3EFE52FE656F
:10366000FE78FE8BFE9FFEB3FEC6FEDAFEEEFE0186
:10367000FF15FF29FF3CFF50FF63FF76FF89FF9C8A
:10368000FFAFFFC2FFD5FFE8FFFAFF0700100019E8
:103690000023002E00390043004D0056005F0067F4
:1036A000006E00740079007D008100850089008D26
:1036B00000920097009D00A300A800AD00B100B5E6
:1036C00000B700B800B900B900B900B900B800B837
:1036D00000B800BA00BB00BD00C000C300C500C8F0
:1036E00000CA00CC00CE00D000D200D400D700DB4E
:1036F00000DF00E400E900EF00F600FE0005010D28
:103700000114011B01210127012C01320137013C69
:1037100001420147014D01520158015D01610166FD
:10372000016A016D016F0171017301740175017608
:10373000017701780179017C017E01810185018891
:10374000018C018F019101930194019501960196DD
:1037500001970198019A019C019F01A201A601AA6B
:1037600001AF01B301B801BD01C201C801CD01D350
:1037700001D801DD01E201E701EC01F101F601FBF5
:1037800001010207020D0214021C0224022C023461
:10379000023D0246024F0258026002690271027A3B
:1037A0000283028C0294029D02A402AC02B302BA0C
:1037B00002C102C702CE02D602DD02E502ED02F42A
:1037C00002FB02010308030D03130319031F032562
:1037D000032D0334033D0346034E0357035F036881
:1037E0000370037803800387038D0394039A03A077
:1037F00003A703AD03B303BA03C103C803CF03D6C2
:1038000003DD03E303E803ED03F103F403F603F838
:1038100003FA03FB03FD03FE03FF0300040004FFA0
:1038200003FD03FA03F603F203EE03E903E403DE08
:1038300003D803D103CA03C203BA03B203AB03A480
:10384000039E03990394038F038C038803850382EB
:10385000037E037B037803750371036D03680364C0
:103860000360035C035903550352034F034C0348A1
:103870000343033E03380331032A03210319030FD3
:10388000030503FB02F002E402D802CC02BE02AF41
:1038900002A0028F027E026C025902460232021F0F
:1038A000020B02F701E401D001BD01AA01980186D3
:1038B000017501640153014201320120010F01FE33
:1038C00000ED00DB00C900B700A400920080006D8D
:1038D000005B0049003600250014000400F3FFE4FB
:1038E000FFD6FFC8FFBBFFAEFFA2FF97FF8DFF848F
:1038F000FF7BFF73FF6CFF65FF60FF5AFF55FF51B1
:10390000FF4DFF49FF47FF44FF43FF43FF42FF4393
:10391000FF43FF44FF44FF43FF41FF3EFF3BFF37B0
:10392000FF33FF2FFF2CFF29FF26FF23FF21FF1E60
:10393000FF1AFF17FF12FF0DFF08FF02FFFCFEF545
:10394000FEEFFEE8FEE0FED8FED1FEC8FEC0FEB7E8
:10395000FEAFFEA6FE9DFE94FE8CFE84FE7DFE76EE
:10396000FE70FE6BFE66FE62FE5FFE5CFE5AFE5857
:10397000FE57FE56FE56FE55FE54FE52FE50FE4EBB
:10398000FE4CFE49FE47FE44FE41FE3FFE3CFE3932
:10399000FE36FE32FE2EFE2AFE26FE23FE1FFE1CF3
:1039A000FE19FE16FE12FE0EFE0AFE06FE01FEFDCA
:1039B000FDF8FDF3FDEFFDEBFDE7FDE3FDDFFDDCD5
:1039C000FDD9FDD5FDD2FDCEFDCAFDC7FDC2FDBEB0
:1039D000FDBBFDB7FDB4FDB1FDAEFDAAFDA6FDA288
:1039E000FD9CFD96FD8FFD88FD82FD7CFD76FD71C1
:1039F000FD6DFD68FD61FD5BFD53FD4AFD40FD363B
:103A0000FD2BFD22FD19FD10FD08FD01FDFAFCF363
:103A1000FCECFCE4FCDCFCD3FCCAFCC0FCB6FCAC5B
:103A2000FCA1FC98FC8FFC87FC7FFC79FC73FC6E8E
:103A3000FC69FC65FC62FC5FFC5DFC5CFC5BFC5AA9
:103A4000FC5AFC5AFC5BFC5BFC5CFC5CFC5CFC5CBC
:103A5000FC5CFC5BFC59FC57FC55FC52FC4FFC4CDD
:103A6000FC49FC46FC42FC3FFC3BFC37FC34FC3090
:103A7000FC2CFC28FC25FC22FC20FC1EFC1DFC1C54
:103A8000FC1CFC1CFC1CFC1CFC1DFC1FFC20FC2268
:103A9000FC25FC28FC2CFC31FC36FC3CFC43FC4B9C
:103AA000FC54FC5EFC68FC72FC7DFC88FC93FC9E74
:103AB000FCAAFCB5FCC0FCCBFCD5FCE0FCEAFCF4A9
:103AC000FCFEFC08FD11FD1BFD24FD2EFD37FD4015
:103AD000FD49FD51FD5AFD62FD69FD70FD77FD7DDB
:103AE000FD83FD8AFD90FD98FD9FFDA8FDB1FDBA07
:103AF000FDC4FDCEFDD9FDE4FDF0FDFCFD09FE1782
:103B0000FE26FE34FE44FE53FE63FE73FE83FE94E7
:103B1000FEA5FEB7FEC8FEDAFEEDFE00FF12FF2690
:103B2000FF38FF4BFF5DFF70FF83FF94FFA6FFB7D9
:103B3000FFC7FFD7FFE6FFF3FFFEFF030017002BD1
:103B4000004000540068007D009100A500B900CD40
:103B500000E100F50008011B012E01410153016540
:103B600001770189019B01AC01BE01CF01E001F1A8
:103B70000102021302230234024402540265027558
:103B80000284029402A302B202C102CF02DD02EA61
:103B900002F802040311031D03280333033E034804
:103BA0000352035C0365036F03770380038903916A
:103BB000039903A103A903B103B903C003C803CF49
:103BC00003D503DC03E103E703EC03F003F403F89C
:103BD00003FA03FD03FE03FF03000400040004FFD7
:103BE00003FE03FC03FA03F803F603F403F103EF07
:103BF00003EC03EA03E703E403E203DF03DC03D996
:103C000003D503D203CE03C903C503C003BA03B46B
:103C100003AE03A703A0039803900388037F0376F2
:103C2000036D0363035A03500345033B033103262B
:103C3000031B0311030603FB02F002E502D902CEC7
:103C400002C202B602AA029D0291028402760269B1
:103C5000025B024E0240023202240216020802FAFD
:103C600001EC01DE01D001C201B501A7019A018D6D
:103C70000180017301660159014C014001330126A5
:103C80000119010B01FE00F000E200D400C500B6EE
:103C900000A700980089007A006B005B004C003D93
:103CA000002E001F0011000200F4FFE6FFD9FFCB39
:103CB000FFBFFFB2FFA6FF9AFF8FFF84FF7AFF705E
:103CC000FF66FF5CFF54FF4BFF43FF3BFF33FF2CBE
:103CD000FF25FF1EFF18FF11FF0BFF06FF01FFFC72
:103CE000FEF7FEF2FEEEFEEAFEE6FEE2FEDFFEDCA0
:103CF000FED9FED6FED4FED1FECFFECDFECBFECA4F
:103D0000FEC8FEC7FEC6FEC5FEC5FEC4FEC4FEC498
:103D1000FEC5FEC5FEC6FEC8FEC9FECCFECEFED167
:103D2000FED4FED8FEDCFEE0FEE4FEE9FEEFFEF48B
:103D3000FEFAFEFFFE05FF0BFF11FF17FF1DFF231D
:103D4000FF29FF2EFF33FF37FF3BFF3FFF42FF44BA
:103D5000FF46FF47FF47FF47FF46FF45FF42FF3F44
:103D6000FF3BFF37FF32FF2CFF25FF1EFF17FF0F22
:103D7000FF06FFFDFEF3FEE9FEDFFED4FEC9FEBE38
:103D8000FEB2FEA7FE9BFE8EFE82FE75FE68FE5B07
:103D9000FE4EFE40FE32FE24FE16FE07FEF9FDEA50
:103DA000FDDBFDCCFDBDFDADFD9EFD8EFD7FFD6F00
:103DB000FD60FD50FD41FD31FD22FD13FD04FDF6CA
:103DC000FCE8FCDAFCCDFCC0FCB4FCA8FC9DFC9338
:103DD000FC8AFC81FC79FC73FC6DFC68FC64FC6172
:103DE000FC5FFC5EFC5FFC60FC63FC68FC6DFC74CB
:103DF000FC7CFC85FC8FFC9BFCA8FCB6FCC5FCD6BF
:103E0000FCE8FCFBFC0FFD24FD3AFD51FD69FD8241
:103E1000FD9CFDB6FDD2FDEEFD0BFE28FE46FE64C8
:103E2000FE83FEA3FEC2FEE2FE03FF23FF44FF6407
:103E3000FF85FFA6FFC7FFE7FF08002800480068CE
:103E4000008800A700C600E40002011F013B0157E3
:103E50000172018D01A601BF01D701EF0105021A10
:103E6000022F02430255026702780288029602A4DA
:103E700002B102BD02C802D202DA02E202E902EF96
:103E800002F302F702FA02FB02FC02FB02FA02F75B
:103E900002F402F002EA02E402DD02D502CC02C220
:103EA00002B702AC029F02920285027602670257B5
:103EB000024702350223021102FE01EA01D601C2C5
:103EC00001AC01970181016B0154013D0126010FF5
:103ED00001F700DF00C700AF0096007E0065004CD0
:103EE0000033001A000200E9FFD0FFB7FF9FFF86F2
:103EF000FF6EFF56FF3EFF26FF0EFFF7FEE0FEC9F6
:103F0000FEB3FE9DFE87FE71FE5CFE47FE33FE1E85
:103F1000FE0BFEF7FDE4FDD1FDBFFDADFD9BFD8A6F
:103F2000FD79FD69FD59FD4AFD3BFD2DFD1FFD118C
:103F3000FD04FDF8FCECFCE1FCD6FCCCFCC2FCB9B9
:103F4000FCB1FCA9FCA2FC9BFC94FC8FFC89FC85C9
:103F5000FC81FC7DFC7AFC77FC75FC73FC72FC72C6
:103F6000FC72FC72FC73FC74FC77FC79FC7CFC80BA
:103F7000FC84FC89FC8EFC94FC9AFCA1FCA8FCAFA0
:103F8000FCB7FCC0FCC8FCD1FCDBFCE5FCEFFCF999
:103F9000FC04FD10FD1BFD27FD33FD40FD4DFD5BC9
:103FA000FD68FD77FD85FD94FDA4FDB4FDC4FDD441
:103FB000FDE5FDF6FD07FE19FE2AFE3CFE4EFE6005
:103FC000FE73FE85FE97FEAAFEBCFECFFEE2FEF566
:103FD000FE08FF1BFF2EFF41FF55FF68FF7CFF908F
:103FE000FFA5FFB9FFCDFFE1FFF2FF0200060009C8
:103FF000000D001000140017001A001E00210025FB
:104000000028002C002F003300360039003D00400E
:1040100000430047004A004E005100550058005C24
:10402000005F006200660069006D00700073007739
:10403000007A007E008100850088008B008F00924E
:1040400000960099009D00A000A300A700AA00AE62
:1040500000B100B400B800BB00BF00C200C600C978
:1040600000CD00D000D300D700DA00DE00E100E48C
:1040700000E800EB00EF00F200F600F900FC0000A1
:1040800001030107010A010E011101140118011BAE
:10409000011F012201260129012C013001330137C2
:1040A000013A013D014101440148014B014E0152D9
:1040B00001550159015C016001630167016A016DED
:1040C000017101740178017B017E01820185018902
:1040D000018C019001930196019A019D01A101A417
:1040E00001A801AB01AE01B201B501B901BC01BF2C
:1040F00001C301C601CA01CD01D101D401D801DB40
:1041000001DE01E201E501E901EC01F001F301F654
:1041100001FA01FD010102040208020B020E021263
:1041200002150219021C021F02230226022A022D76
:10413000023102340237023B023E0242024502498A
:10414000024C024F02530256025A025D02600264A0
:104150000267026B026E027202750279027C027FB4
:1041600002830286028A028D029002940297029BC9
:10417000029E02A202A502A802AC02AF02B302B6DE
:1041800002B902BD02C002C402C702CB02CE02D1F4
:1041900002D502D802DC02DF02E302E602E902ED08
:1041A00002F002F402F702FA02FE0201030503081C
:1041B000030C030F031303160319031D0320032429
:1041C0000327032B032E033103350338033C033F3E
:1041D000034203460349034D035003540357035A54
:1041E000035E036103650368036C036F0372037668
:1041F0000379037D038003840387038A038E03917D
:1042000003950398039B039F03A203A603A903AD91
:1042100003B003B303B703BA03BE03C103C503C8A6
:1042200003CC03CF03D203D603D903DC03E003E3BB
:1042300003E703EA03EE03F103F503F803FB03FFCF
:1042400003000000FC04FC07FC0AFC0EFC11FC153A
:10425000FC18FC1BFC1FFC22FC26FC29FC2DFC305E
:10426000FC33FC37FC3AFC3EFC41FC45FC48FC4B73
:10427000FC4FFC52FC56FC59FC5CFC60FC63FC6788
:10428000FC6AFC6EFC71FC75FC78FC7BFC7FFC829C
:10429000FC86FC89FC8CFC90FC93FC97FC9AFC9EB1
:1042A000FCA1FCA4FCA8FCABFCAFFCB2FCB6FCB9C6
:1042B000FCBCFCC0FCC3FCC7FCCAFCCDFCD1FCD4DC
:1042C000FCD8FCDBFCDFFCE2FCE5FCE9FCECFCF0F0
:1042D000FCF3FCF7FCFAFCFDFC01FD04FD08FD0B02
:1042E000FD0FFD12FD15FD19FD1CFD20FD23FD2612
:1042F000FD2AFD2DFD31FD34FD38FD3BFD3EFD4227
:10430000FD45FD49FD4CFD50FD53FD57FD5AFD5D3A
:10431000FD61FD64FD68FD6BFD6EFD72FD75FD794F
:10432000FD7CFD80FD83FD86FD8AFD8DFD91FD9464
:10433000FD97FD9BFD9EFDA2FDA5FDA9FDACFDAF7A
:10434000FDB3FDB6FDBAFDBDFDC1FDC4FDC7FDCB8E
:10435000FDCEFDD2FDD5FDD9FDDCFDDFFDE3FDE6A3
:10436000FDEAFDEDFDF1FDF4FDF7FDFBFDFEFD02B7
:10437000FE05FE08FE0CFE0FFE13FE16FE1AFE1DC5
:10438000FE21FE24FE27FE2BFE2EFE32FE35FE38D9
:10439000FE3CFE3FFE43FE46FE4AFE4DFE50FE54EE
:1043A000FE57FE5BFE5EFE61FE65FE68FE6CFE6F04
:1043B000FE73FE76FE79FE7DFE80FE84FE87FE8B18
:1043C000FE8EFE91FE95FE98FE9CFE9FFEA3FEA62D
:1043D000FEA9FEADFEB0FEB4FEB7FEBBFEBEFEC142
:1043E000FEC5FEC8FECCFECFFED2FED6FED9FEDD57
:1043F000FEE0FEE4FEE7FEEAFEEEFEF1FEF5FEF86C
:10440000FEFCFEFFFE02FF06FF09FF0DFF10FF147A
:10441000FF17FF1AFF1EFF21FF25FF28FF2CFF2F8C
:10442000FF32FF36FF39FF3DFF40FF43FF47FF4AA2
:10443000FF4EFF51FF55FF58FF5BFF5FFF62FF66B6
:10444000FF69FF6DFF70FF73FF77FF7AFF7EFF81CB
:10445000FF85FF88FF8BFF8FFF92FF96FF99FF9DDF
:10446000FFA0FFA3FFA7FFAAFFAEFFB1FFB4FFB8F5
:10447000FFBBFFBFFFC2FFC6FFC9FFCCFFD0FFD30A
:10448000FFD7FFDAFFDDFFE1FFE4FFE8FFEBFFEF1F
:10449000FFF2FFF6FFF9FFFCFF0000010104020636
:1044A00002070209020B020C020E02100212021392
:1044B000021502170218021A021C021E021F022114
:1044C0000223022402260228022A022B022D022F96
:1044D000023002320234023502370239023B023C1A
:1044E000023E024002410243024502470248024A9C
:1044F000024C024D024F025102530254025602581E
:104500000259025B025D025F0260026202640265A0
:1045100002670269026B026C026E02700271027322
:10452000027502760278027A027C027D027F0281A5
:1045300002820284028602880289028B028D028E28
:10454000029002920294029502970299029A029CAA
:10455000029E02A002A102A302A502A602A802AA2C
:1045600002AC02AD02AF02B102B202B402B602B8AE
:1045700002B902BB02BD02BE02C002C202C302C532
:1045800002C702C902CA02CC02CE02CF02D102D3B4
:1045900002D502D602D802DA02DB02DD02DF02E136
:1045A00002E202E402E602E702E902EB02ED02EEB9
:1045B00002F002F202F302F502F702F802FA02FC3C
:1045C00002FE02FF02010303030503060308030AB8
:1045D000030B030D030F0310031203140316031739
:1045E0000319031B031C031E0320032203230325BB
:1045F00003270328032A032C032E032F033103333D
:10460000033403360338033A033B033D033F0340BF
:1046100003420344034603470349034B034C034E41
:10462000035003520353035503570358035A035CC3
:10463000035D035F03610363036403660368036947
:10464000036B036D036F03700372037403750377C9
:104650000379037B037C037E03800381038303854B
:1046600003870388038A038C038D038F03910392CE
:104670000394039603980399039B039D039F03A050
:1046800003A203A403A503A703A903AA03AC03AED3
:1046900003B003B103B303B503B603B803BA03BC55
:1046A00003BD03BF03C103C203C403C603C803C9D8
:1046B00003CB03CD03CE03D003D203D403D503D75A
:1046C00003D903DA03DC03DE03DF03E103E303E5DD
:1046D00003E603E803EA03EB03ED03EF03F103F260
:1046E00003F403F603F703F903FB03FD03FE0300E2
:1046F00004000100FF00FC02FC03FC05FC07FC09B0
:10470000FC0AFC0CFC0EFC0FFC11FC13FC15FC1647
:10471000FC18FC1AFC1BFC1DFC1FFC21FC22FC24C9
:10472000FC26FC27FC29FC2BFC2DFC2EFC30FC324B
:10473000FC33FC35FC37FC38FC3AFC3CFC3EFC3FCF
:10474000FC41FC43FC44FC46FC48FC4AFC4BFC4D51
:10475000FC4FFC50FC52FC54FC56FC57FC59FC5BD3
:10476000FC5CFC5EFC60FC62FC63FC65FC67FC6856
:10477000FC6AFC6CFC6EFC6FFC71FC73FC74FC76D8
:10478000FC78FC79FC7BFC7DFC7FFC80FC82FC845B
:10479000FC85FC87FC89FC8BFC8CFC8EFC90FC91DE
:1047A000FC93FC95FC97FC98FC9AFC9CFC9DFC9F60
:1047B000FCA1FCA3FCA4FCA6FCA8FCA9FCABFCADE2
:1047C000FCAFFCB0FCB2FCB4FCB5FCB7FCB9FCBB64
:1047D000FCBCFCBEFCC0FCC1FCC3FCC5FCC7FCC8E7
:1047E000FCCAFCCCFCCDFCCFFCD1FCD2FCD4FCD66A
:1047F000FCD8FCD9FCDBFCDDFCDEFCE0FCE2FCE4EC
:10480000FCE5FCE7FCE9FCEAFCECFCEEFCF0FCF16E
:10481000FCF3FCF5FCF6FCF8FCFAFCFCFCFDFCFFF0
:10482000FC01FD02FD04FD06FD08FD09FD0BFD0D6B
:10483000FD0EFD10FD12FD13FD15FD17FD19FD1AEE
:10484000FD1CFD1EFD1FFD21FD23FD25FD26FD2870
:10485000FD2AFD2BFD2DFD2FFD31FD32FD34FD36F2
:10486000FD37FD39FD3BFD3DFD3EFD40FD42FD4375
:10487000FD45FD47FD48FD4AFD4CFD4EFD4FFD51F8
:10488000FD53FD54FD56FD58FD5AFD5BFD5DFD5F7A
:10489000FD60FD62FD64FD66FD67FD69FD6BFD6CFD
:1048A000FD6EFD70FD72FD73FD75FD77FD78FD7A7F
:1048B000FD7CFD7EFD7FFD81FD83FD84FD86FD8801
:1048C000FD8AFD8BFD8DFD8FFD90FD92FD94FD9584
:1048D000FD97FD99FD9BFD9CFD9EFDA0FDA1FDA307
:1048E000FDA5FDA7FDA8FDAAFDACFDADFDAFFDB189
:1048F000FDB3FDB4FDB6FDB8FDB9FDBBFDBDFDBF0B
:10490000FDC0FDC2FDC4FDC5FDC7FDC9FDCBFDCC8D
:10491000FDCEFDD0FDD1FDD3FDD5FDD7FDD8FDDA0F
:10492000FDDCFDDDFDDFFDE1FDE3FDE4FDE6FDE891
:10493000FDE9FDEBFDEDFDEEFDF0FDF2FDF4FDF515
:10494000FDF7FDF9FDFAFDFCFDFFFEFFFF0100FE96
:10495000FF0B002A001F003200240017001E003544
:10496000004D0033001300F7FF10001C002E00352F
:10497000001F000F00F5FF03001100140037003284
:1049800000020006003B00D400430173017A016875
:10499000013E012B016A01B302F60354026E00DCF2
:1049A000FE05FEEFFE66FFEAFE12FEAEFDB4FDB4AC
:1049B000FD98FD78FD5AFD6FFD6AFD56FD38FD2717
:1049C000FD33FD31FD42FD58FD64FD67FD6EFD8543
:1049D000FDACFDE8FD2DFE63FE8CFEA8FEB8FED109
:1049E000FE0DFF4AFF78FFB1FFEFFF22006800B61F
:1049F00000FC0036015F019301D30102022C025337
:104A0000027E029A02A602BC02C402D802F4020587
:104A1000031A0323031A031C03240333033F03462F
:104A20000346034403430334031D030203D902BEB8
:104A300002B602A40295028102700263023F0210D4
:104A400002DD01B6019901780164014E013A0126A7
:104A5000010501E900CB009F00700048002100FB28
:104A6000FFD0FFABFF7BFF49FF20FFF9FEDCFEB666
:104A7000FE90FE6EFE50FE31FE12FEF0FDC8FD9C63
:104A8000FD71FD4FFD31FD16FDFCFCE8FCD3FCB9CA
:104A9000FCA8FC9BFC94FC8DFC82FC82FC89FC93B2
:104AA000FC95FC93FC97FC95FC90FC93FCA1FCB757
:104AB000FCC8FCD6FCE6FCEEFCFEFC1BFD49FD72CE
:104AC000FD88FD96FDA2FDB2FDCDFDECFD06FE22AA
:104AD000FE3BFE5AFE85FEB2FEE3FE0FFF39FF5D90
:104AE000FF7CFFA2FFC8FFF8FF2D005D008F00C113
:104AF00000F60025014D0172019101B101D301EFD2
:104B00000110023102510271028E02B002C802D4B9
:104B100002DE02E902FB020503040303030803119A
:104B200003150311030803F902EF02ED02E802E2A4
:104B300002D802CB02B802A0028A027302620253B8
:104B400002400227020902E701C501A80196018976
:104B5000017C0169014F0134011501F000C800A674
:104B6000008E006F00460024000800E8FFC7FFAA7F
:104B7000FF90FF71FF4EFF2FFF16FF05FFF7FEE0CE
:104B8000FECAFEB2FE99FE79FE5EFE4BFE36FE1FA9
:104B9000FE09FEF5FDE3FDD8FDD7FDDDFDE2FDEBF1
:104BA000FDF0FDF1FDEEFDEEFDEFFDF0FDF6FD0289
:104BB000FE12FE23FE2EFE33FE3EFE4DFE60FE7410
:104BC000FE88FE99FEA9FEBDFED7FEF4FE0FFF296A
:104BD000FF40FF52FF5FFF6CFF77FF85FF96FFAB43
:104BE000FFC5FFE1FFFCFF1A003500530070009283
:104BF00000B600D800FD001E013D015A017101867A
:104C000001A101BE01D901EE0105021D02300241E0
:104C1000024B02520258025C02620266026602679E
:104C2000026802670263025B0255024E02420235CD
:104C300002240215020802FD01F301E601D901C7B1
:104C400001B3019C017F0165014E013D0130011D51
:104C5000010901F300D800BB009D008100640043FE
:104C6000002200FFFFE2FFC9FFB1FF9CFF89FF7731
:104C7000FF64FF4FFF39FF20FF06FFECFED2FEBBB3
:104C8000FEA6FE94FE84FE73FE63FE51FE3FFE31DF
:104C9000FE20FE0BFEF3FDDDFDCEFDC0FDB7FDAD3C
:104CA000FDA3FD98FD8BFD7CFD71FD6AFD67FD6533
:104CB000FD64FD63FD5EFD58FD54FD55FD5BFD5F2C
:104CC000FD5EFD5AFD53FD50FD4FFD54FD60FD6F2F
:104CD000FD82FD91FD9FFDAEFDBEFDCFFDE2FDF528
:104CE000FD07FE19FE2FFE44FE5AFE71FE86FE9C55
:104CF000FEB2FECFFEF4FE19FF3BFF5AFF77FF9591
:104D0000FFAFFFC7FFDFFFF4FF0A002000340048B9
:104D1000005B0073008E00AC00CF00F00011012E8C
:104D20000148015F01720185019901AE01C701E2ED
:104D300001FD0116022E0244025802680279028720
:104D4000029702A502AF02B802C102C902CE02D286
:104D500002D402D302CC02C402BA02B402AD02A849
:104D600002A1029A0293028A0282027D027A0277EB
:104D700002700265025602450230021B020702F26F
:104D800001DF01CE01BD01AB01980183016C01532C
:104D90000139011F010501EB00CF00B1009400763D
:104DA0000059003C0021000700EDFFD3FFB8FF9D34
:104DB000FF82FF66FF4CFF35FF1FFF09FFF3FEDC9C
:104DC000FEC5FEAEFE9AFE86FE75FE67FE5AFE4DDD
:104DD000FE41FE36FE2BFE22FE19FE0FFE02FEF500
:104DE000FDE7FDDAFDD2FDCCFDCCFDCCFDCDFDCE49
:104DF000FDCCFDC9FDC4FDBFFDBBFDBAFDB9FDBBCA
:104E0000FDBEFDC4FDCAFDD0FDD5FDDCFDE5FDEF19
:104E1000FDF7FDFDFD05FE10FE1DFE2DFE3EFE4DC7
:104E2000FE5BFE66FE6FFE79FE85FE93FEA4FEB974
:104E3000FECFFEE5FEF8FE0CFF20FF35FF4BFF62C4
:104E4000FF77FF88FF98FFA7FFB8FFCCFFE3FFFDC8
:104E5000FF1800310048005B006E007E008D009F4F
:104E600000B100C600DA00EF00040118012C014275
:104E700001590173018F01A901C201D801EE01039B
:104E80000212021F022902310238023F0246024C7E
:104E90000253025A0263026B02760282028C02956E
:104EA000029C029C0297029002890285028302837F
:104EB00002850287028A028A02880284027D0275C4
:104EC000026E0266025E02560250024A0243023A33
:104ED000022E021E020D02F901E601D301C001AE4D
:104EE000019C018B017A016A0159014701350122B8
:104EF000010E01F800E100C900B00096007D0064D9
:104F0000004B0033001A000200E9FFD0FFB8FFA1F8
:104F1000FF8AFF72FF5BFF43FF2CFF15FFFEFEE7DA
:104F2000FECFFEB9FEA5FE92FE81FE72FE63FE522A
:104F3000FE3EFE28FE12FEFCFDE8FDD7FDC4FDB3DB
:104F4000FDA3FD95FD87FD77FD68FD59FD4BFD3FF8
:104F5000FD33FD29FD21FD18FD10FD07FD02FDFDBE
:104F6000FCFBFCF9FCFBFCFFFC03FD09FD11FD173C
:104F7000FD1DFD22FD24FD25FD26FD27FD2BFD3118
:104F8000FD39FD43FD4CFD56FD61FD6FFD7CFD8946
:104F9000FD95FD9EFDA8FDB4FDC4FDD8FDEDFD020F
:104FA000FE14FE25FE36FE47FE5AFE70FE89FEA563
:104FB000FEC0FEDAFEF3FE0AFF22FF3AFF52FF6850
:104FC000FF7AFF8BFF9AFFA9FFBAFFCDFFE1FFF544
:104FD000FF0700190029003B004C005C006E0081B7
:104FE000009300A400B400C500D500E700FA000F4C
:104FF0000124013A01500167017D019401A901BD1D
:1050000001CF01DE01ED01FA010702140221022E97
:10501000023A02450251026002720285029702A61C
:1050200002B202BB02C102C502C802CB02CF02D447
:1050300002D902DF02E502E802EA02EB02EA02E735
:1050400002E302DF02DB02D702D502D302D102CB98
:1050500002C302B802AB029E029002830276026B88
:1050600002610258024E0245023C0233022A021E2D
:105070000210020202F301E301D201C001AE019C61
:1050800001890174015F014B01380124011101FF05
:1050900000ED00D900C300AD009600800068004F0D
:1050A0000035001D000700F2FFE0FFCDFFB8FFA3B1
:1050B000FF8CFF74FF5CFF46FF31FF1EFF0CFFF902
:1050C000FEE5FED1FEBCFEA7FE91FE7CFE68FE540E
:1050D000FE42FE30FE1FFE0BFEF9FDE7FDD3FDC3D1
:1050E000FDB0FDA1FD93FD87FD7CFD73FD6BFD63B0
:1050F000FD5CFD53FD48FD3DFD30FD25FD1BFD1311
:10510000FD0EFD0AFD08FD06FD06FD07FD09FD0B70
:10511000FD0BFD08FD07FD07FD0AFD0EFD13FD1843
:10512000FD1BFD1DFD1DFD1FFD23FD27FD2FFD3872
:10513000FD41FD4AFD54FD5FFD6CFD79FD87FD9449
:10514000FDA1FDACFDB8FDC5FDD4FDE5FDF8FD0CF0
:10515000FE20FE35FE4CFE63FE7AFE91FEA7FEBCED
:10516000FED0FEE4FEF7FE0CFF22FF39FF51FF697F
:10517000FF83FF9DFFB8FFD3FFEDFF06001E003346
:10518000004600580069008800A400BD00D600ED6C
:105190000004011A01300145015A016D018001939B
:1051A00001A501B601C701D701E601F40102021011
:1051B000021C02280234023E02480252025B0263D1
:1051C000026A02720278027E02830287028B028FD9
:1051D0000292029502960298029902990299029906
:1051E00002980296029502920290028D028A02862D
:1051F0000282027D02790274026E02680263025D1D
:105200000256025002490242023A0233022B0223A2
:10521000021B0213020A020202FA01F101E801DF95
:1052200001D601CD01C401BB01B201A8019F0196C5
:10523000018C0183017901700167015D0154014A0C
:1052400001410138012E0125011C01120109010053
:1052500001F700EE00E400DB00D200CA00C100B795
:1052600000AF00A6009D0094008C0083007A0072BD
:10527000006900610058004F0047003F0036002ED3
:105280000025001D0015000C000400FCFFF4FFEBDE
:10529000FFE3FFDBFFD2FFCAFFC2FFBAFFB2FFA9E5
:1052A000FFA1FF99FF91FF88FF81FF78FF70FF68E2
:1052B000FF60FF57FF4FFF47FF3FFF37FF2FFF27DD
:1052C000FF1FFF17FF0FFF06FFFFFEF6FEEFFEE7D3
:1052D000FEDEFED7FECFFEC7FEBFFEB7FEAFFEA8C6
:1052E000FEA0FE98FE91FE89FE82FE7AFE73FE6CA1
:1052F000FE65FE5DFE56FE4FFE48FE41FE3AFE3361
:10530000FE2DFE27FE20FE1AFE14FE0EFE08FE02F3
:10531000FEFDFDF7FDF2FDEDFDE8FDE3FDDEFDD94F
:10532000FDD5FDD1FDCDFDC9FDC5FDC0FDBCFDB95F
:10533000FDB6FDB3FDB1FDAFFDACFDAAFDA9FDA716
:10534000FDA5FDA4FDA3FDA3FDA2FDA2FDA2FDA25E
:10535000FDA2FDA3FDA3FDA5FDA6FDA8FDA9FDAB36
:10536000FDADFDB0FDB3FDB6FDB9FDBCFDC0FDC496
:10537000FDC8FDCCFDD1FDD6FDDBFDE1FDE6FDEC7C
:10538000FDF2FDF8FDFFFD05FE0CFE13FE1BFE22E7
:10539000FE2AFE32FE3AFE42FE4BFE54FE5DFE66E3
:1053A000FE6FFE79FE83FE8DFE97FEA1FEACFEB67B
:1053B000FEC1FECCFED8FEE3FEEEFEFAFE06FF12B4
:1053C000FF1EFF2AFF36FF43FF4FFF5CFF69FF759B
:1053D000FF82FF8FFF9CFFA9FFB7FFC4FFD2FFDF53
:1053E000FFECFFFAFF07001500220030003E004BE3
:1053F0000059006700740081008F009D00AA00B86A
:1054000000C500D200E000ED00FA00070114012100
:10541000012D013A01460153015F016B01770183C0
:10542000018E019A01A501B001BB01C601D101DBCA
:1054300001E601EF01F90103020D0216021F022825
:10544000023002380241024902500258025F0265EE
:10545000026C02730279027E02840289028E029338
:105460000297029B029F02A302A602AA02AD02AF0C
:1054700002B102B402B502B702B802B902BA02BA66
:1054800002BB02BB02BA02BA02B902B902B702B643
:1054900002B402B202B002AE02AB02A802A502A29E
:1054A000029F029B02970292028F028A028502806B
:1054B000027B02760270026A0264025E02570251A7
:1054C000024A0243023C0235022D0225021E021648
:1054D000020E020502FD01F401EB01E301D901D046
:1054E00001C601BD01B301AA01A00196018B018192
:1054F0000176016C01610156014B01400135012922
:10550000011D0112010701FB00EF00E300D700CBF2
:1055100000BF00B300A7009B008E00830076006AE6
:10552000005D005100450038002C001F00130007EB
:1055300000FBFFEEFFE3FFD6FFCAFFBEFFB3FFA7EE
:10554000FF9BFF90FF84FF79FF6EFF63FF58FF4DC5
:10555000FF42FF38FF2DFF23FF19FF0EFF05FFFB62
:10556000FEF1FEE8FEDFFED6FECDFEC4FEBCFEB3BD
:10557000FEABFEA3FE9BFE94FE8CFE85FE7EFE77B8
:10558000FE70FE6AFE64FE5EFE58FE52FE4DFE4751
:10559000FE42FE3EFE39FE35FE31FE2DFE29FE2680
:1055A000FE23FE20FE1DFE1AFE18FE16FE14FE133C
:1055B000FE11FE10FE0FFE0EFE0EFE0EFE0EFE0E85
:1055C000FE0FFE0FFE10FE11FE13FE14FE16FE1857
:1055D000FE1AFE1DFE1FFE22FE25FE29FE2CFE30B9
:1055E000FE34FE38FE3CFE41FE45FE4AFE4FFE54B0
:1055F000FE5AFE5FFE65FE6BFE71FE77FE7EFE8448
:10560000FE8BFE92FE99FEA0FEA7FEAEFEB6FEBE8B
:10561000FEC5FECEFED5FEDEFEE6FEEFFEF8FE0186
:10562000FF0AFF13FF1CFF25FF2EFF38FF41FF4B32
:10563000FF55FF5FFF69FF73FF7DFF87FF91FF9CB1
:10564000FFA6FFB1FFBBFFC6FFD0FFDBFFE6FFF009
:10565000FFFBFF060011001B00270031003C004744
:105660000052005D00670072007D00880092009D7E
:1056700000A700B200BD00C700D100DB00E500EFCD
:1056800000F90003010D0117012001290133013C3C
:105690000145014D0156015E0167016F0177017FF0
:1056A0000187018E0196019D01A401AA01B101B7F4
:1056B00001BE01C401CA01CF01D401D901DF01E358
:1056C00001E801EC01F001F401F701FB01FE010129
:1056D0000203020602070209020A020C020D020D71
:1056E000020E020E020E020D020D020C020B020946
:1056F000020702060203020102FE01FB01F801F4A7
:1057000001F001EC01E801E301DF01D901D501CF8E
:1057100001CA01C401BE01B801B101AB01A4019DE0
:105720000196018F01870180017801700168015F96
:105730000157014E0145013C0134012A01210118A4
:10574000010E010401FA00F100E600DD00D200C8FC
:1057500000BE00B400A9009E00940089007E007382
:105760000069005E00530048003D00330027001C24
:105770000011000600FCFFF0FFE5FFDAFFCFFFC4D9
:10578000FFB9FFAEFFA3FF98FF8DFF82FF77FF6D8C
:10579000FF62FF57FF4CFF41FF37FF2CFF21FF1730
:1057A000FF0DFF02FFF8FEEDFEE3FED9FECFFEC5C2
:1057B000FEBBFEB1FEA8FE9EFE95FE8BFE82FE782D
:1057C000FE6FFE66FE5DFE54FE4CFE43FE3BFE3267
:1057D000FE29FE22FE19FE12FE0AFE02FEFBFDF36A
:1057E000FDECFDE5FDDEFDD7FDD0FDCAFDC4FDBD30
:1057F000FDB7FDB2FDACFDA6FDA1FD9CFD97FD92A0
:10580000FD8DFD89FD84FD80FD7CFD79FD75FD72BA
:10581000FD6FFD6CFD69FD67FD65FD63FD60FD5F6E
:10582000FD5EFD5CFD5BFD5BFD5AFD5AFD5AFD5AB8
:10583000FD5AFD5BFD5BFD5CFD5EFD5FFD60FD6295
:10584000FD64FD67FD69FD6CFD6FFD72FD75FD7901
:10585000FD7DFD81FD86FD8AFD8FFD93FD99FD9EF9
:10586000FDA3FDA9FDAFFDB5FDBBFDC1FDC8FDCE8E
:10587000FDD5FDDCFDE3FDEBFDF2FDFAFD01FE0AC9
:10588000FE11FE1AFE22FE2AFE33FE3CFE45FE4DB0
:10589000FE56FE5FFE69FE72FE7BFE85FE8EFE9862
:1058A000FEA2FEACFEB6FEC0FECAFED4FEDEFEE9DF
:1058B000FEF3FEFDFE08FF12FF1DFF27FF32FF3D36
:1058C000FF47FF52FF5DFF68FF72FF7DFF88FF9378
:1058D000FF9DFFA8FFB3FFBEFFC8FFD4FFDEFFE9B7
:1058E000FFF4FFFEFF090013001E00290034003EF4
:1058F00000490053005D00680072007D0087009140
:10590000009B00A500B000BA00C400CE00D800E1A2
:1059100000EB00F500FE00080112011B0124012D1F
:105920000137013F01480151015A0163016B0174C4
:10593000017C0184018D0195019D01A501AC01B49B
:1059400001BC01C301CB01D201D901E001E601EDA7
:1059500001F401FA01000206020C02120217021DF4
:1059600002220227022C02310236023A023E024291
:1059700002450249024C0250025302560258025B91
:10598000025D025F026102630264026602660267F0
:1059900002680268026902690269026802680267B5
:1059A00002660265026302620260025E025C0259E4
:1059B000025602530250024D024902450241023D85
:1059C00002390234022F022A0225021F021A02148F
:1059D000020E0208020202FB01F501EE01E701E0FE
:1059E00001D801D101C901C101BA01B101A901A1C7
:1059F000019901900187017E0175016C0163015AD3
:105A000001500147013D01330129011F0115010B1F
:105A1000010101F600EC00E200D700CD00C200B8A1
:105A200000AD00A20097008C00820077006C00613E
:105A30000056004B00400035002A001F00140009EA
:105A400000FEFFF3FFE8FFDDFFD3FFC7FFBDFFB29E
:105A5000FFA7FF9CFF92FF87FF7CFF71FF67FF5C42
:105A6000FF52FF48FF3DFF33FF29FF1FFF15FF0BCC
:105A7000FF01FFF7FEEDFEE4FEDAFED1FEC7FEBE3B
:105A8000FEB5FEACFEA3FE9AFE92FE89FE81FE7973
:105A9000FE71FE69FE61FE59FE52FE4AFE43FE3C67
:105AA000FE35FE2EFE27FE21FE1BFE14FE0FFE0914
:105AB000FE03FEFEFDF9FDF3FDEEFDEAFDE5FDE171
:105AC000FDDDFDD9FDD4FDD1FDCDFDCAFDC7FDC471
:105AD000FDC2FDBEFDBDFDBAFDB8FDB6FDB5FDB311
:105AE000FDB2FDB1FDB0FDAFFDAFFDAEFDAEFDAE53
:105AF000FDAEFDAFFDAFFDAFFDB0FDB1FDB3FDB33C
:105B0000FDB5FDB7FDB8FDBAFDBCFDBEFDC1FDC4D0
:105B1000FDC6FDC9FDCCFDCFFDD2FDD5FDD9FDDD16
:105B2000FDE0FDE5FDE9FDEDFDF2FDF6FDFBFDFF10
:105B3000FD04FE09FE0EFE14FE19FE1FFE25FE2BBF
:105B4000FE31FE36FE3DFE43FE4AFE50FE56FE5D31
:105B5000FE64FE6BFE71FE79FE80FE87FE8EFE9572
:105B6000FE9CFEA4FEACFEB3FEBBFEC2FECAFED28D
:105B7000FEDAFEE2FEEAFEF2FEFAFE02FF0AFF1382
:105B8000FF1BFF24FF2CFF35FF3DFF46FF4FFF5754
:105B9000FF61FF69FF72FF7BFF84FF8DFF96FF9F10
:105BA000FFA8FFB1FFBAFFC3FFCDFFD6FFDFFFE8BD
:105BB000FFF1FFFBFF04000D00170020002A003357
:105BC000003C0046004F00580062006B0074007DEE
:105BD00000870090009900A300AC00B400BE00C78D
:105BE00000CF00D800E100EA00F300FB0004010C44
:105BF0000115011D0126012E0136013E0146014E0F
:105C00000156015E0166016D0175017C0184018B05
:105C10000192019901A001A701AE01B501BB01C22A
:105C200001C801CE01D401DA01E001E601EC01F185
:105C300001F601FC01010206020B02100215021915
:105C4000021E02220226022A022E02320235023AE5
:105C5000023D0240024302470249024C024F0251F8
:105C6000025402560258025A025C025E026002614D
:105C700002620264026402660266026702680268E7
:105C800002680268026802680268026802670266C7
:105C9000026602650264026302610260025E025CE7
:105CA000025A0258025602540252024F024C024952
:105CB000024602440240023D023902360232022FFD
:105CC000022B02270223021E021A02150211020CE5
:105CD0000207020202FD01F701F201ED01E701E214
:105CE00001DC01D601D001CA01C301BD01B701B079
:105CF00001AA01A3019C0195018E0187017F017812
:105D0000017101690162015A0152014A0143013BDB
:105D10000133012B0123011A0112010A010101F9CA
:105D200000F000E800DF00D700CE00C500BD00B4E1
:105D300000AC00A3009900910088007F0076006D00
:105D40000064005B0052004900400038002E00262D
:105D5000001C0013000A000200F8FFF0FFE7FFDD5F
:105D6000FFD5FFCCFFC3FFBAFFB1FFA8FF9FFF968F
:105D7000FF8EFF85FF7CFF74FF6BFF62FF5AFF51B0
:105D8000FF49FF40FF38FF30FF27FF1FFF17FF0FBE
:105D9000FF07FFFFFEF7FEEFFEE7FEDFFED8FED0B7
:105DA000FEC9FEC1FEBAFEB2FEABFEA4FE9DFE968B
:105DB000FE8FFE89FE82FE7BFE75FE6EFE69FE6230
:105DC000FE5CFE56FE50FE4AFE45FE3FFE3AFE34A5
:105DD000FE2FFE2AFE25FE20FE1CFE16FE12FE0DE4
:105DE000FE09FE05FE01FEFDFDF9FDF6FDF2FDEFEB
:105DF000FDECFDE8FDE5FDE3FDE0FDDDFDDBFDD9AE
:105E0000FDD6FDD4FDD3FDD1FDCFFDCEFDCDFDCC26
:105E1000FDCBFDCAFDCAFDCAFDC9FDC9FDCAFDCA4B
:105E2000FDCAFDCBFDCCFDCCFDCDFDCEFDD0FDD121
:105E3000FDD3FDD4FDD7FDD9FDDBFDDEFDE1FDE3A6
:105E4000FDE6FDE9FDECFDF0FDF4FDF7FDFBFDFFDA
:105E5000FD03FE07FE0CFE11FE15FE1AFE1FFE24BA
:105E6000FE29FE2EFE34FE39FE3FFE44FE4AFE5061
:105E7000FE56FE5CFE63FE69FE6FFE76FE7CFE83D0
:105E8000FE8AFE91FE98FE9FFEA6FEADFEB5FEBC0C
:105E9000FEC3FECBFED2FEDAFEE2FEE9FEF1FEF923
:105EA000FE01FF09FF10FF18FF20FF28FF31FF3818
:105EB000FF40FF49FF51FF58FF61FF69FF71FF7904
:105EC000FF81FF89FF91FF9AFFA2FFAAFFB2FFBAED
:105ED000FFC2FFCBFFD3FFDBFFE3FFEBFFF3FFFBD3
:105EE000FF03000B0013001C0023002B0033003BBA
:105EF0000043004B0053005A0062006A00720079B0
:105F00000080008800900097009E00A600AD00B4BD
:105F100000BC00C200CA00D100D800DE00E500ECE1
:105F200000F300F900000106010D01130119012021
:105F30000126012C01330139013E0144014A01507F
:105F40000155015C01610166016C01710177017C01
:105F500001810186018B01900195019A019E01A3A7
:105F600001A801AC01B001B501B901BD01C101C574
:105F700001C901CD01D001D401D801DB01DE01E26C
:105F800001E501E801EB01ED01F101F301F501F893
:105F900001FA01FC01FE01000202020402060208ED
:105FA0000209020A020C020D020E020F0210021177
:105FB000021102120212021202130213021302133E
:105FC00002120212021102110210020F020F020D40
:105FD000020D020B020A0208020702050203020177
:105FE00002FF01FD01FB01F901F601F401F101EFEE
:105FF00001EC01E901E601E201DF01DC01D901D593
:1060000001D201CE01CA01C601C201BE01BA01B668
:1060100001B201AD01A901A401A0019B019601916A
:10602000018D01880183017E01780173016E016891
:106030000163015D01580152014C01460141013BE0
:106040000135012E01290122011C01150110010950
:10605000010301FC00F500EF00E800E100DA00D4E4
:1060600000CD00C600BF00B800B100AA00A2009C8D
:106070000094008D0086007E007800700069006149
:10608000005A0053004B0044003D0035002E00260E
:10609000001F001800100009000100FAFFF3FFEBD9
:1060A000FFE4FFDDFFD5FFCEFFC6FFC0FFB8FFB1A5
:1060B000FFAAFFA3FF9BFF95FF8EFF87FF80FF795D
:1060C000FF72FF6BFF65FF5EFF57FF50FF4AFF4304
:1060D000FF3DFF36FF30FF29FF23FF1DFF17FF1194
:1060E000FF0AFF04FFFEFEF8FEF2FEEDFEE7FEE112
:1060F000FEDBFED6FED0FECAFEC5FEC0FEBAFEB571
:10610000FEB0FEABFEA6FEA1FE9CFE97FE92FE8EAA
:10611000FE89FE85FE80FE7CFE78FE74FE6FFE6BBF
:10612000FE67FE63FE5FFE5CFE58FE54FE51FE4DB0
:10613000FE4AFE47FE44FE40FE3DFE3AFE38FE3477
:10614000FE32FE30FE2CFE2AFE28FE25FE23FE2116
:10615000FE1FFE1DFE1BFE1AFE18FE16FE15FE1487
:10616000FE12FE11FE10FE0FFE0EFE0DFE0CFE0CCA
:10617000FE0BFE0BFE0BFE0AFE0AFE0BFE0BFE0BD9
:10618000FE0BFE0CFE0CFE0DFE0EFE0EFE10FE11B2
:10619000FE12FE14FE15FE17FE18FE1AFE1CFE1E51
:1061A000FE20FE22FE25FE27FE29FE2CFE2EFE31BD
:1061B000FE34FE37FE3AFE3DFE40FE43FE47FE4AF9
:1061C000FE4EFE52FE56FE5AFE5EFE62FE66FE6AFF
:1061D000FE6FFE73FE78FE7DFE81FE86FE8AFE90D7
:1061E000FE94FE9AFE9EFEA4FEA9FEAEFEB3FEB98C
:1061F000FEBEFEC4FEC9FECFFED4FEDAFEE0FEE522
:10620000FEECFEF1FEF7FEFDFE03FF09FF0FFF159A
:10621000FF1BFF21FF27FF2EFF34FF3BFF41FF47FE
:10622000FF4DFF54FF5BFF61FF67FF6EFF74FF7B55
:10623000FF81FF88FF8EFF95FF9BFFA2FFA9FFAFA5
:10624000FFB6FFBDFFC4FFCAFFD1FFD8FFDEFFE5E9
:10625000FFECFFF2FFF9FF000007000D0014001A29
:1062600000210028002E0035003B00410048004E70
:106270000055005B00620068006E0074007B0081C6
:106280000087008D00930099009F00A500AB00B12E
:1062900000B700BC00C200C700CD00D300D800DEAC
:1062A00000E200E800ED00F200F700FC000101064A
:1062B000010B010F01140118011D01210125012A03
:1062C000012E01320136013A013D014101450149EA
:1062D000014C014F015301560159015C015F0162FC
:1062E00001650168016A016D016F01710174017638
:1062F0000178017A017C017E0180018101830184A2
:106300000186018701880189018A018B018B018C3B
:10631000018D018D018E018E018F018F018F018F03
:10632000018F018F018F018F018F018E018E018DF1
:10633000018D018C018C018B018A018A0188018801
:106340000187018601850184018201810180017E2E
:10635000017D017B01790178017601740172017080
:10636000016E016C016A0168016501630160015EF3
:10637000015B0159015601530150014E014A014789
:1063800001440141013E013B013701340131012D3E
:10639000012A01260122011F011B01170113010F10
:1063A000010C0107010301FF00FB00F700F200EE02
:1063B00000EA00E600E100DC00D800D400CF00CA0B
:1063C00000C600C100BC00B800B300AE00A900A424
:1063D000009F009B00950091008C00860081007C4E
:1063E00000770072006D00680063005E0058005383
:1063F000004E00490043003E00390034002E0029C1
:106400000024001F001A0014000F000A000400FFFF
:10641000FFFAFFF5FFF0FFEAFFE5FFE0FFDAFFD646
:10642000FFD1FFCBFFC6FFC1FFBCFFB7FFB2FFAD7F
:10643000FFA8FFA3FF9EFF99FF94FF8FFF8BFF86AE
:10644000FF81FF7CFF78FF73FF6EFF6AFF65FF61CE
:10645000FF5CFF58FF53FF4FFF4BFF46FF42FF3DDE
:10646000FF39FF35FF31FF2DFF29FF25FF21FF1DDC
:10647000FF19FF15FF11FF0DFF09FF06FF02FFFEC9
:10648000FEFBFEF7FEF3FEF0FEEDFEE9FEE6FEE3A8
:10649000FEE0FEDDFED9FED6FED3FED0FECDFECB65
:1064A000FEC8FEC5FEC3FEC0FEBEFEBBFEB9FEB604
:1064B000FEB4FEB2FEB0FEAEFEACFEAAFEA8FEA783
:1064C000FEA5FEA3FEA2FEA0FE9FFE9EFE9DFE9CDC
:1064D000FE9AFE9AFE98FE98FE97FE96FE95FE9511
:1064E000FE95FE94FE94FE93FE93FE93FE93FE9320
:1064F000FE93FE93FE93FE93FE94FE94FE94FE950F
:10650000FE95FE96FE97FE97FE98FE99FE9AFE9BDC
:10651000FE9CFE9DFE9EFE9FFEA1FEA2FEA3FEA58A
:10652000FEA6FEA8FEAAFEACFEADFEAFFEB1FEB317
:10653000FEB5FEB7FEB9FEBBFEBDFEBFFEC2FEC489
:10654000FEC6FEC9FECBFECDFED0FED3FED5FED8E4
:10655000FEDAFEDDFEE0FEE3FEE5FEE8FEEBFEEE2B
:10656000FEF1FEF4FEF7FEFAFEFDFE00FF03FF075C
:10657000FF0AFF0DFF11FF14FF17FF1AFF1EFF2177
:10658000FF25FF28FF2BFF2FFF33FF36FF3AFF3D8C
:10659000FF41FF44FF48FF4CFF50FF53FF57FF5B95
:1065A000FF5FFF62FF66FF6AFF6EFF72FF76FF7A92
:1065B000FF7EFF82FF86FF8AFF8EFF92FF96FF9A83
:1065C000FF9FFFA3FFA7FFACFFAFFFB4FFB8FFBC67
:1065D000FFC1FFC5FFC9FFCDFFD2FFD6FFDAFFDF46
:1065E000FFE3FFE7FFECFFF0FFF4FFF8FFFCFF0025
:1065F00000050009000D001100150019001D002103
:1066000000250029002D003100350039003D0041F2
:1066100000440048004C005000530057005B005EEF
:10662000006200660069006D007000740077007AF7
:10663000007D008100840087008A008D0090009317
:1066400000960099009C009E00A100A400A600A94D
:1066500000AB00AE00B000B300B500B700B900BC9D
:1066600000BE00C000C200C400C600C700C900CB05
:1066700000CD00CE00D000D200D300D500D600D887
:1066800000D900DB00DC00DD00DE00E000E100E21C
:1066900000E300E400E500E600E700E700E800E9C9
:1066A00000EA00EA00EB00EC00EC00EC00ED00ED8D
:1066B00000ED00EE00EE00EF00EE00EF00EF00EF67
:1066C00000EF00EF00EF00EF00EF00EE00EE00EE55
:1066D00000EE00ED00ED00EC00EC00EB00EB00EA5A
:1066E00000EA00E900E800E700E700E500E500E473
:1066F00000E300E200E100E000DE00DD00DC00DBA2
:1067000000D900D800D600D500D400D200D000CFE8
:1067100000CD00CB00CA00C800C600C400C300C042
:1067200000BF00BD00BB00B900B700B500B300B0AA
:1067300000AF00AC00AA00A800A600A300A1009F23
:10674000009D009A0098009600930091008F008CA5
:1067500000890087008500820080007E007B007831
:10676000007600740071006E006C006900670064C0
:106770000062005F005C005A005700540052004F56
:10678000004D004A004700450042003F003D003AEE
:106790000037003500320030002D002A0027002588
:1067A00000230020001D001B00180015001300111D
:1067B000000F000B000900060004000100FFFFFCB1
:1067C000FFF9FFF7FFF4FFF2FFEFFFECFFEAFFE74F
:1067D000FFE5FFE2FFDFFFDDFFDAFFD8FFD5FFD3E4
:1067E000FFD0FFCDFFCBFFC8FFC6FFC3FFC1FFBF78
:1067F000FFBCFFB9FFB7FFB4FFB2FFAFFFADFFAA09
:10680000FFA8FFA6FFA3FFA1FF9FFF9DFF9AFF9890
:10681000FF96FF94FF92FF90FF8DFF8BFF89FF870C
:10682000FF85FF83FF81FF7FFF7DFF7CFF7AFF787D
:10683000FF77FF75FF74FF72FF71FF6FFF6EFF6CD4
:10684000FF6BFF6AFF69FF67FF66FF65FF64FF6319
:10685000FF62FF62FF61FF60FF5FFF5FFF5EFF5D42
:10686000FF5DFF5CFF5CFF5BFF5BFF5AFF5AFF5958
:10687000FF59FF59FF59FF58FF58FF58FF58FF585D
:10688000FF58FF58FF59FF59FF59FF59FF59FF5A49
:10689000FF5AFF5AFF5BFF5BFF5CFF5CFF5DFF5D24
:1068A000FF5EFF5FFF5FFF60FF61FF62FF62FF63EC
:1068B000FF64FF65FF65FF66FF67FF68FF69FF6AAA
:1068C000FF6BFF6CFF6DFF6EFF6FFF70FF71FF725C
:1068D000FF73FF74FF75FF77FF78FF79FF7AFF7B07
:1068E000FF7CFF7DFF7FFF80FF81FF82FF84FF85AC
:1068F000FF86FF88FF89FF8AFF8CFF8DFF8FFF9047
:10690000FF92FF93FF95FF96FF98FF99FF9BFF9CD7
:10691000FF9EFF9FFFA1FFA3FFA4FFA6FFA7FFA964
:10692000FFAAFFACFFAEFFAFFFB1FFB2FFB4FFB6EF
:10693000FFB7FFB9FFBBFFBCFFBEFFC0FFC2FFC375
:10694000FFC5FFC7FFC8FFCAFFCCFFCEFFCFFFD1F7
:10695000FFD3FFD5FFD7FFD9FFDAFFDCFFDEFFE073
:10696000FFE2FFE4FFE5FFE7FFE9FFEBFFEDFFEFED
:10697000FFF0FFF2FFF4FFF6FFF7FFF9FFFBFFFC6C
:10698000FFFEFF00000100030004000600070009ED
:10699000000A000C000D000F00100012001300157B
:1069A000001600180019001A001B001D001E001F11
:1069B0000021002200240025002600280029002AAA
:1069C000002C002D002E002F003100320033003447
:1069D0000036003700380039003A003C003D003EE8
:1069E000003F004000410042004300440046004692
:1069F000004700480049004A004B004C004D004E43
:106A0000004F004F005000510052005200530054FC
:106A100000550055005600560057005800580059C0
:106A20000059005A005A005B005B005C005C005C8F
:106A3000005D005D005D005E005E005E005E005F68
:106A4000005F005F005F005F005F0060005F00604C
:106A5000005F005F005F005F005F005F005F005F3E
:106A6000005F005E005E005E005E005D005D005C39
:106A7000005C005C005B005B005A005A0059005942
:106A80000058005800570056005600550054005456
:106A900000530052005100500050004F004E004D76
:106AA000004C004C004B004A00490048004700469B
:106AB00000460045004400430042004100410040C0
:106AC000003F003E003D003D003C003B003A003AE4
:106AD0000039003800370036003500350034003307
:106AE0000032003100310030002F002E002D002D2B
:106AF000002C002B002A002A00290028002700274C
:106B00000026002500240024002300230022002169
:106B100000210020001F001F001E001D001D001C82
:106B2000001C001B001B001A001A00190018001896
:106B300000170017001600160015001500140014A9
:106B40000013001200120011001100100010000FBD
:106B5000000E000E000D000D000C000C000B000BD1
:106B6000000A0009000900080008000700070006E5
:106B700000060006000500050004000400030003F1
:106B800000030002000200020001000100010001F8
:106B9000000000000000000000FFFFFFFFFFFFFFFC
:106BA000FFFFFFFFFFFFFFFEFFFEFFFEFFFEFFFEFA
:106BB000FF0200FDFF0700FEFF0A00BCFF16FF4EAC
:106BC000FF91FFA3FFA7FFA7FFBCFFDAFFFCFF03B6
:106BD0000016004E0074004B005A008900B400AC4F
:106BE00000AA00A800A8007A006F007D008700704E
:106BF000008300AF009E007A005800B3FFC4FE255A
:106C0000FECDFD1BFEF0FC62FD23FD00FC19FC0027
:106C1000FC0CFC00FC05FC00FC00FC15FCA3FC9A31
:106C2000FD7AFEE0FE43FFCCFF760014012301DC79
:106C30000189030004FA030004FC030004FD0300BF
:106C400004FE030004FF0300040004FF030004FE2D
:106C5000030004C8036203EF0277025402E5012037
:106C60000119004E00CF00CA0082002D00D7FFA6F8
:106C7000FF95FF60FF7CFF89FF9AFFFFFE8EFD6D91
:106C8000FC35FC00FC09FC00FC7CFC51FD6FFD7C2C
:106C9000FD76FC88FCA5FDE9FC0BFC15FCA9FC7A43
:106CA000FC02FC00FC6CFCEEFD97FEA1FE36FEBF74
:106CB000FDEBFDD6FD3EFDA5FC48FD01FF4CFF4967
:106CC000FE09FEFEFE3FFFE0FE4DFE0BFE5CFE7B7E
:106CD000FE3AFF70FF33FFE4FE9EFEAEFEEAFE0DBD
:106CE000FF13FF29FF32FF25FF93FFA5FFC7FF28F2
:106CF00000E3FF94FFAFFFCAFF2100D0004C011357
:106D00000147005C007000C9000F012F01E901BBC1
:106D10000202030C031F039203ED03D203B10358D5
:106D20000367038403EE03FF03F8030004FC03007E
:106D300004F403F403BF03C103ED03E003E1030024
:106D400004F103A503430368032203BE02BC02420D
:106D50000213020B02030253026E024D02F301BD45
:106D60000112022B02E601BF019001510152013BC9
:106D7000010F01D600B800B2007E003E000E004CAC
:106D8000FF8FFE31FE49FD1AFD4AFD0FFDE0FCB00C
:106D9000FC79FC63FC1FFC18FC34FC00FC0AFC3D85
:106DA000FC6CFC01FDEFFC22FC42FCAFFC9BFCBA3E
:106DB000FC49FC0DFC99FCD5FC90FDD4FDC0FD8C7C
:106DC000FD96FD17FD2EFC44FC6CFCB0FC10FDCBC9
:106DD000FD64FDACFC10FD23FEFBFE9FFE42FE4663
:106DE000FEBBFE6EFF6800ED006F00CE00AB00F64C
:106DF000FF8CFFB1FF44007E00B6001201C9014CB8
:106E000002ED017A0150023302A201B20153011EC8
:106E100001E1018202F601320137012C02B40215B0
:106E2000033C033E0237029A03FC036B0352028ABF
:106E300002CB035A031203E602FF02DD024A024CB0
:106E4000034B033202B601070267019A0097004024
:106E500000FC0077010E01E9FFEFFF3A0020008CF3
:106E600000BFFE27FE2CFFA9FF9EFF43FFF5FE2E6D
:106E7000FE4FFEF6FED5FF3BFFDAFEA7FEE3FDCE9A
:106E8000FD82FD87FDFDFCF6FD3BFEC9FD37FD469D
:106E9000FDC5FD80FD6FFD23FD29FD43FDA2FD66BF
:106EA000FD4BFEA0FE93FE4AFEDBFD3AFE87FE8709
:106EB000FEDEFE34FF3EFFCCFF1200F5FF0600A30E
:106EC00000AA003E005EFF7AFF7CFF88FF38004288
:106ED000009900FD00EE002800E7FF7A001100DFB6
:106EE000FF2E007B00D90096006BFFE0FE4DFFDC1B
:106EF000FF9D0084FFE2FF270094FF7BFFB7FFE9BF
:106F0000FF12007B018C002E004D00F0FFAC0092C0
:106F1000019B002D005A00C7FF5C006500F900C509
:106F200000CFFF9CFF0800D30036012601F600B712
:106F3000007E00F800C401D90188015001E900DF9A
:106F4000000D01A1005C003D002500B50024016199
:106F50000006007A004000EEFF4FFF53FF1700A429
:106F600000BA008F007DFFF5FD83FE35FFDEFEFBDE
:106F7000FF01006FFF96FFDEFECAFE59FF7DFF1383
:106F8000FFEBFE48FFEBFFB5FFC4FFA1FFB1FFA77A
:106F9000FF24FFD2FF72005400A7FFE1FFE4FFE6E9
:106FA000FF4DFF96FE22FFD8FFDDFFD4FF3900DA48
:106FB000FF6E00FCFF1CFF93FF54FF6EFF5D00E3BC
:106FC000FF81FF8DFF5FFF34FFCEFE29FEBDFDCAAE
:106FD000FECAFEA0FE52FE49FEDEFEBFFF7CFFC7DA
:106FE000FD88FEC4FE5EFECBFEA8FE98FF2A001EB2
:106FF000FFADFED9FFE40043009AFF6EFFA8FFC972
:107000000044011D00D8FF320089FFC8FF2700128D
:1070100000B70068014F00EDFF73004100C700B4E6
:107020000079005A00C300BD0031017F0114018BBB
:107030000095FF6D00AF015E012F010501EA001808
:1070400002F900400003014301B1012A01F000519F
:1070500001D1009A007300AD00DB0027018E01DD35
:107060000086FEE0FDB0FF2900FFFFE4FF8D00C1B8
:10707000FFAEFF67FFECFE53FF85FF4200B6002026
:107080000037FF8BFE5CFE7CFEAFFECFFFE8FFC744
:10709000000D0001FFFBFDEDFDAFFF60FFBAFFF348
:1070A000FF95FF31FF79FF81FF67FF2DFF8FFFE124
:1070B000FE7CFD87FE5FFF1BFFE8FE3FFF7BFFA01E
:1070C000FF04FFFDFE36FFD2FF30FF2C00570142C8
:1070D00000C9FF04FFE2FED3FF2100A7FF9E00BD11
:1070E000FF6EFFF0FFC1FF8CFF66FFD1FF8B007AC0
:1070F000FFFEFE94FF96FFC7FFA2FF4100A6FFA37D
:10710000FF45FFB8FF3400CAFF53FF05002B01DC29
:10711000FF8BFFA6FF4AFF41000A0134006FFFF119
:10712000FF8FFF3FFFC7006501FF00F6FFD3FFE8B9
:10713000FFC6FFA40061014201ED00DA0041000B2F
:107140000161019F008E00640092007F000F01EB3F
:107150000031004401A0011501F70004017D007316
:107160000088001E003F01DB017D018D0014002C12
:10717000018C0097FF6BFF35007C008DFF83FF843F
:10718000FF5200BB00BD0033007900340079FFCE10
:10719000FF0FFFCAFEAEFE72FF3A00C2FFF0FEC94B
:1071A000FEF8FEEEFE62FF45FF49FF45FFBDFE0C07
:1071B000FFE4FE25FFADFE56FF2600C1FFC5FF6CB4
:1071C000FFDBFFE3FF5AFF87FEAFFEBCFE41FF85FA
:1071D000FFF9FF82FF63FFC4FF0BFF4A00CDFF2EC4
:1071E000FFC8FE4EFE21FF0900B4008D005600F5D9
:1071F000FF0900EBFFBCFFC9FFFAFFE2FFC6FF1A61
:107200000057009100380091007F00A5FF88FFD84B
:10721000FFE1004301E1006D00F4FFEC001801857F
:1072200000B200F0005C01A601490158016F00CED8
:10723000FFBE009E002701D90038007A006E0020B2
:10724000003CFF1600050167001F00AAFF5FFFD486
:10725000FF17003A00DE00DA00790085FF4DFF8D50
:10726000FF8EFFCEFF64007E001B000E00BCFF4AB5
:10727000008C005E00DBFF96FF4FFF45FF8700B5E7
:107280000055FF92FFC1FFADFF81FFC6FF3C000C20
:1072900000080014FF5AFFD1FF14003D001300A79F
:1072A000FF67FFFCFF53001F00FCFF90FFBCFFA522
:1072B000FFDBFFFDFF9AFF8800CD00F6FF61FF2D89
:1072C000FF4CFFC2FFFEFF91FF0EFF96FF65FF26FA
:1072D00000270085FF1A00E4FF17FF47FF59FF2C26
:1072E00000DC00260067009EFF70FF80FF6400B393
:1072F000009D0089002300E7FFABFF53004800AF6B
:1073000000AE00D60066001B00380097000901C7D8
:1073100000320125013101920071005E00440069D4
:10732000004E005000CCFFA10032009CFF7B00AE5D
:10733000004E00E7FF2800F3FF1EFF7AFF4200E740
:10734000FF2C00B30086FF20FF66003600D9FF4304
:10735000FFF3FF350072FFD5FFFFFF8B00C100294F
:107360000066FFDAFFB7FF2800BDFF9BFFFEFFDBD3
:10737000FFFAFFE6FF29004A00570097FF81FFAEA2
:10738000FF0E00D4FFA6FFE8FF7000ADFF45FFC56C
:10739000FFACFFD8FFF8FFF7FFD6FF830084007B28
:1073A000002D0092FF6BFF92FFD7FF77FFE6FFD91A
:1073B000005201C00072002D004F005900D8FF5448
:1073C000004100FEFF9FFFC6FFDDFFBF00B5003498
:1073D0000069002400E0FF8CFF080072002000E03C
:1073E000FFAFFF9BFF50005A00380086007F009FD0
:1073F000FF51FF48FF37009500FDFF49001C0018B2
:1074000000A200B800ECFFD1FF04002200E6FFFD5F
:10741000FFAE00CD00FEFFEAFF74005800F6FF7BD0
:10742000FF130056003C009D00340002000C00F9E0
:10743000FF3300E7FF2100940082005B002100D4AD
:10744000FF30006D00CEFFC1FF1100D6FFC6FF3335
:107450000070003300E9FF81003700D3FF6EFF8426
:10746000FF5D00FDFF1F0010009CFFBCFF27001602
:107470000085FFDEFF4C003B00C8FF3EFFBAFFEB7C
:10748000FF5A00C90041001B00B6FF0F003B00CAB5
:10749000FFA3FFDDFF1400C8FF5F009D002500EB88
:1074A000FF7F00610086FFECFF7C004300F8FF26B1
:1074B0000069006000CEFF9FFFE1FF3D0067002AEA
:1074C00000540090004F009FFFA1FFF3FFE2FF1464
:1074D0000014001B0083FF28FFCBFF48006100E879
:1074E000FF0200B1FF47FF79FF7BFFF0FFA800B765
:1074F00000F2FF9CFF80FFF1FF1400E6FFE5FF7440
:10750000FFCDFF2E00E5FF51FF4DFF86FF2900B3A1
:1075100000D5FF0D0019008BFF46006500BFFFEA94
:10752000FF2E003900C100F000AC000B0024006207
:10753000008B003F002B007600A000A00019004443
:10754000003A005F003100E8FF290054003F006D61
:107550000078007B005C00F1FFF9FF98009A004E74
:1075600000FBFF15009F004B001200ABFF6A0054A8
:10757000001000BC007E004B00C1FFA0FF0B0053B9
:10758000003C0072FF3EFF8FFF6600A800FEFF3147
:107590000004006DFFAFFFDFFF8DFFD6FFBCFFC112
:1075A000FF2B003B000D00C8FFAFFF0100F1FFDD26
:1075B000FFFBFFA1FF87FF5DFFBCFFBFFFF7FF3CA5
:1075C00000B4FFE2FFC5FFB8FFD6FFE9FFEBFF64A1
:1075D000FFA0FFEFFF06001100E0FF81FF98FFD53D
:1075E000FFD2FFEFFFAFFFA2FFD4FFE9FFD7FFB14C
:1075F000FF380083003F00C3FF5BFF9CFF3E007C21
:10760000002C002E00DFFF3D00F2FFBDFF1B003A03
:10761000008300B500DA006D00FAFF9AFFF6FF372D
:10762000005F000E00E4FF21005500030074FFCE50
:10763000FF3A001D000C00EFFFA2FF34008300059D
:10764000003F005D00E0FFE3FF2600C100E7001AF5
:10765000009CFF3500B200FCFFAEFF22006C00E78B
:10766000001C006DFFE7FF1F000B00C4FF31006727
:10767000001400FAFF4C007F002300ADFF0400223D
:10768000004D0060002900910027002F006A0015BE
:107690000067FF52FFBBFFF3FF5D007700820073BE
:1076A00000400098FF74FF87FF27002D00B1FFAC5A
:1076B000FF7FFF88FF95FF4B004A00060013FFD8AD
:1076C000FED3FF4600D400DCFF50FF80FF76FFD8DA
:1076D000FFA0FFF2FF280066003F001200ACFFCEC3
:1076E000FE3DFF65FFB1FFCAFF9EFFC0FF35006C86
:1076F000001F00ACFF61FF80FFA4FFB3FFC9FF21A3
:107700000017001000220050004300FDFF0E00DBB8
:10771000FF3800610091FFC8FF4C0041004A003073
:1077200000190034006A0095004600AFFFF0FFAD7D
:10773000009A0079001100FCFF8B005B006000677D
:107740000041002A003F00450021007500FFFFEBCB
:10775000FF7C0070006A003B00F3FFD1FFF2FFDD09
:10776000FFAFFFF4FF1D005100770039002E0056D7
:1077700000F9FF5FFF97FF90FFEAFFE5FFECFF25B1
:10778000001F003800E8FFD4FF8CFFF7FF95FFF2E1
:10779000FFCE004300F9FFF9FF14002B0080FF63C8
:1077A000FFBBFFC6FFF5FFB7FF0F00E1FF95FFA18D
:1077B000FFDBFF0700F2FFBBFFBEFFB3FF51FFB3CC
:1077C000FF12000C00EEFFCDFFBCFFDCFF8FFF7A45
:1077D000FFF0FF0D00A9FFF3FFE0FF78FF9DFFD052
:1077E000FF93FF31FFE1FF1700E3FF9CFF86FFB42B
:1077F000FFEBFF0500D0FFD4FFD2FFBAFF4A004CD9
:1078000000CCFF2B001000E0FF2400E0FF55FF78C4
:10781000FF0A00B100C9000600D1FFD2FFDAFF1E47
:107820000076007F002700FCFF15007600B60056AA
:1078300000B9FFEDFF2C005D00340033001F00583D
:1078400000730053009D009000B10066000E003DE3
:1078500000870087007000370022000E0084004D72
:107860000011002E00F4FFFDFF88004600D6FF390E
:107870000039003F002B00EDFF39009700DDFFA429
:10788000FFA2FF38000600AAFFA7FF35005E0085B3
:10789000FFA5FFA1FFCBFFDDFFDEFFE1FF97FF6F3D
:1078A000FFE9FF97FF60FF6EFF89FF9CFF8BFFC022
:1078B000FF0B001A0069FF4BFF88FFF6FF1600F46C
:1078C000FFDDFFB5FFC9FFC5FF79FF69FFDDFF3BA6
:1078D00000E6FF71FFDAFFB1FF44FF5EFFC0FF600B
:1078E00000E9FF93FFA3FFA2FFDCFF90FF4AFF9692
:1078F000FF53008B000E0058FF6EFF0A00EDFF8063
:10790000FF59FF3800FBFF25FFC1FF32003D00019A
:1079100000FFFF480038001B000200040053007302
:10792000000600B6FF350035001C0066003A005026
:10793000003E000B006E007D000B00E0FF3F00AA40
:107940000097004200000079006B0016002D002A0D
:10795000006A0099005D007E009400070024004A40
:1079600000E4FF33004F005D00E600C4006200CD7C
:10797000FFE8FF190047007B001C00DBFFE4FFEB82
:10798000FFE4FFF7FFFCFF2D002200D6FFE0FFC45D
:10799000FFD7FFE1FFF7FF18009FFF81FF68FF8E11
:1079A000FFE6FFEEFF03009EFF3BFF66FF77FFBC95
:1079B000FFD3FFA4FF5DFF55FF83FFC5FFCBFFA5EE
:1079C000FF98FF88FF6DFF40FF65FF89FFCAFFCE6C
:1079D000FFC1FFA1FFC5FFFCFFD6FF39FF19FFAFB5
:1079E000FFD9FF1900DFFFA1FF9CFF63FFD1FF2B31
:1079F0000008002600F3FFB1FF07001400FAFF396A
:107A00000026000C00360096006400C6FF06003A0F
:107A1000005C006600490093004D000A000D00263E
:107A200000780094006E003200210014002400321F
:107A300000230005004600610006002A007200399C
:107A4000000A0028000F000A003900280029003B26
:107A50000010003B00E0FFA7FFDEFFFBFF45003A00
:107A60000044005B00FDFF95FFE2FFF4FFFFFFE72E
:107A7000FFDAFFEAFF050038001A001800B8FF7AA5
:107A8000FFE5FF0E00D4FF0E0057009100E1FF3725
:107A9000FF91FFC6FFE8FF35001F009AFF7DFF77CB
:107AA000FFB1FFA4FF94FFE8FF19002400BCFFA56D
:107AB000FFABFFCEFFB1FFC9FF0300B9FFA1FFCBB2
:107AC000FFEBFFE1FFE4FFCFFFEBFFC6FFB9FF0CC9
:107AD00000120008001500BCFFC1FFFCFFF9FFD930
:107AE000FFAEFFE0FF62006C0029000C00C0FFE663
:107AF000FFFEFF3D0078000300A6FFF2FF75006B5C
:107B00000077007F0020000E00FAFFFCFFF8FF0F57
:107B10000060008A007E004000160054003B000612
:107B2000002000D9FFFFFF69002400020034001B81
:107B3000001900F5FFE7FFF2FF00000C001E00EF48
:107B4000FF180056001B00E1FFBFFFF0FFBCFFAEB7
:107B5000FFD2FFFCFF3F000500B6FFC7FFD9FF03C0
:107B6000000800A3FFD7FF2300EAFFD8FFD7FFA537
:107B7000FFB6FFDFFFC2FFD7FFF5FFF2FFF7FF09F8
:107B800000E1FFC3FFD6FFA8FFA3FF26003F0028A8
:107B900000FBFFBBFFCCFF120060002B00E6FFBD27
:107BA000FF2700030002000E00A8FF1C009800A39E
:107BB00000F8FFCFFF590022002200550023005992
:107BC000001500CEFF21005D002F00070036005099
:107BD00000380005001C00370041005F0038001924
:107BE000000E0017001600250003000B002B0040BC
:107BF000003D00E1FFFBFF070035001700CEFFCD81
:107C0000FF2400170000001300F7FFC4FF82FFDC11
:107C1000FF24001000A3FFABFFE1FF03000000EF13
:107C2000FFB5FFCCFF2000DCFF9DFF7AFFB7FF12FE
:107C3000001E00DFFFB4FFE8FFE7FFCBFFD3FFD25A
:107C4000FFF7FF1B001B001200D4FFAFFFEFFF0484
:107C500000F7FF210039002300F3FFD3FFFCFF3DB5
:107C6000004E00040003004E001100E1FF02000A74
:107C70000056006E003100D7FFC8FF44007100209D
:107C800000EFFF06000D001000210041002000EB76
:107C9000FFFEFF3500ECFFDCFF12000F0046002F57
:107CA000002C002C001500ECFFFFFF420042003BBF
:107CB0000019003200260012000100D3FFD7FF2375
:107CC000005F002500080020004B0058002300132F
:107CD00000E2FFE3FF160010000D00350058001C05
:107CE000000400E8FF0000390015000A001F00230F
:107CF000001E00F1FF03000C00F3FFCBFFADFFF10E
:107D0000FF1700F7FFB1FFBDFFF2FF08000900D425
:107D1000FFADFFC2FFDDFFEBFFC7FFE6FFD8FFB7F8
:107D2000FFCCFFBAFFD3FFEEFFF1FFB5FFBEFFF6BA
:107D3000FF09000300D7FFD6FFDDFFE1FFE9FFECFD
:107D4000FF16002E001F0000000500CAFFE8FF27F5
:107D500000FAFF10001300FEFFF7FFFEFF1700FB05
:107D6000FFFEFF1200F2FF3A002D001E001B00155F
:107D70000017003F005E00040007001900430027C1
:107D800000FCFF0C00E6FF14005E00420032004AD7
:107D900000600025000900080027005D0032004156
:107DA000003E002F00050015004A0037001C002C83
:107DB000003D002C0047001600D6FFEDFF320034D6
:107DC000002C001A00E2FFD8FF0A00EEFFF4FF0BC0
:107DD00000D7FFF7FFEFFF0000F8FFF5FF190013D2
:107DE00000EEFFE8FF15000500FFFF0F00F3FFDACC
:107DF000FFD7FFFEFF0500F3FFF2FFEAFF140013B9
:107E000000F9FFF0FFE5FFE4FF11000500F2FF2A93
:107E1000000700F1FF0700E4FFDCFF01000D002A6E
:107E2000001100DDFFE8FF13001D000800FAFFF05D
:107E3000FFFAFF1A001300F3FF0300EAFFE1FF025D
:107E400000DFFFBEFFEDFF0500FBFF00000600E7BF
:107E5000FFEEFFFCFFE3FFF1FFE8FFDAFF0000E1C8
:107E6000FFC0FF12000B00F5FF0600C1FFBDFFF6CB
:107E7000FF15001D0026001600E5FFE5FFFBFF25AE
:107E8000001C00F5FF0600180018003D002A00E85D
:107E9000FFEBFFF1FFF4FF29003D0036000000E793
:107EA000FF17002100220024002B001A001B000BEA
:107EB00000290025003E0029001A003300FAFF1DAA
:107EC000000D000B000100370061001D00F3FF17DB
:107ED000001200FFFF2A002200FDFFE8FF11000B47
:107EE00000E6FFE1FF05001200FEFF01000900EFC0
:107EF000FFCEFFE1FFF0FFFEFF0D00F7FFE2FFD333
:107F0000FF00001200FBFFFDFFE9FF1A00FCFFFB72
:107F1000FF2A00150030002300E6FFDFFFF5FFF524
:107F2000FF0F00F2FFE5FF27000D001C00450007D2
:107F300000E9FFD7FFEAFF12001400E9FFFFFF2965
:107F400000FFFFF6FFDDFFC9FFD0FF03001700F8B9
:107F5000FFE9FFDDFFFFFFFFFFEBFFE9FFE6FFEDBE
:107F6000FFF6FFD1FFCEFFD2FFE0FFF3FFF4FFFAF1
:107F7000FFC5FFC3FFEEFF0000E4FFD3FFDBFFEE12
:107F8000FF0000FDFFEAFFDFFFD9FFE9FFEDFFFA89
:107F9000FF0D000D00F4FFE3FFFDFFECFFDFFFCE60
:107FA000FFFDFF0A00E6FFD6FFE4FFFBFF07000F1F
:107FB00000EDFFD0FFDFFFFEFFFBFFF7FFF9FF1A29
:107FC0000028001C0006000100090012000F001D1F
:107FD000004B00410026001D0009000C0026002077
:107FE00000260027003C004A004900290011002A11
:107FF000001600320012000600400040000C00E0B5
:10800000FFE6FFFCFF0F001E00240006000100FF3A
:10801000FF1500F7FFE5FFF3FFF1FF0200E8FFF9AE
:10802000FF1600EFFFD7FFE2FFFBFF090010001370
:1080300000F3FFD6FFD0FFE3FF0000FCFFD3FFD922
:10804000FFD2FFE0FFEEFFE2FFE1FFE2FFDEFFDB3A
:10805000FFE0FFCAFFCCFFCCFFD8FFE1FFDEFFEA65
:10806000FFF9FFCAFFB8FFE4FFF8FFE8FFE2FFE611
:10807000FFDCFFD7FFF2FF0A000B001600F9FFE359
:10808000FFD5FFE9FF0000F3FF0A0017000300F42B
:10809000FFEDFFE7FFD8FFEEFFF9FFFBFFF7FFE87B
:1080A000FFE0FFD3FFE5FFE5FFD7FFE0FFF9FFEFBC
:1080B000FFE3FFE7FFF5FFF9FFF2FFF8FF120017FC
:1080C00000FAFFE7FFF7FF0D001F00170003001283
:1080D000000900090005000600F4FF13002900262E
:1080E000001100F4FFFCFF0E002F0015000000E857
:1080F000FFF9FF19001E00FEFF0000090005001235
:108100000016001400FFFFF1FFF0FF16000F000043
:10811000000200F5FFFFFFEFFFE1FFF2FFEFFFFBC3
:10812000FFFAFFEAFFDFFFE1FFE2FFFEFF0700DDEE
:10813000FFE6FFE4FFE9FFE1FFD9FFE9FFEEFFFA09
:10814000FFEDFFDDFFD0FFCFFFEAFFEDFFE2FFE233
:10815000FFD4FFD8FFE4FFF2FFECFFCBFFC0FFE846
:10816000FFF4FFE8FFE7FFD4FFF2FF0600EEFFD5C4
:10817000FFEAFF0200FAFF0400FBFFEBFFF5FFFD43
:10818000FF11002100FEFFFAFFFEFFF9FF11001FA3
:10819000002A001E001A00240012000C0011002208
:1081A00000310032002F0024002A001B00170012AB
:1081B000000F002C0017001400070005001200FA41
:1081C000FF050013000800FCFF04000200F8FFF99F
:1081D000FFE5FFEAFFF6FFFCFF0100FEFFE5FFD829
:1081E000FFF0FFE9FFF4FFE9FFEAFFDFFFE4FFF440
:1081F000FFEEFFF9FFDCFFE2FFF7FFF4FFEEFFFF0A
:10820000FF15000500FDFF0800E7FFEDFFFFFF1071
:108210000025001B00FAFFEEFFF4FF00000A00FF3C
:10822000FF0D0009000E000A000600EFFFE6FFF850
:10823000FF18001800DCFFE4FFF5FFFFFFFFFFEF72
:10824000FFEFFFFBFF0B00FCFFE5FFE0FFFEFF0978
:1082500000FFFF0700FCFFEFFFF5FFF2FFE9FFF172
:10826000FFF5FFF2FFF2FFF8FFF8FFF1FFFFFF0657
:1082700000F3FFE4FFF6FFE8FFFEFF12000100FF3E
:10828000FFF2FF0200FFFFFDFFF6FFEAFF03001011
:108290000009000700160015000500F9FF07001788
:1082A0000011000A0002000F001E0028001700073E
:1082B00000180033003200160006001E002D002EAC
:1082C000003500180019001C0012000B0015001FDB
:1082D0000023001B0004000700040015001E000D11
:1082E00000FAFF0600090006000500FDFFF9FFF790
:1082F000FFFCFF000013001400FDFF040014001039
:10830000000A00F1FFF2FFFCFF02000B000300FD7A
:10831000FFF7FFF6FFF7FFEFFFF6FF02000C00018B
:1083200000E8FFF3FFF7FFFCFFF4FFF1FFF9FFFBAD
:10833000FFF8FFEAFFECFFF7FFFBFFFEFFF7FFE8A8
:10834000FFEBFFFEFFF6FFEFFFFDFFF9FFFCFFFE77
:10835000FFFCFFFCFF0B000A000000FDFF0500060C
:1083600000080010000100030009000300FCFFFEEC
:10837000FF090016000D00060006000A0013000D9C
:1083800000F3FFFCFF0800FFFF040004000300F8F7
:10839000FFF9FFF6FF06000B0004000500F9FFFAE5
:1083A000FFFCFFFFFFF8FFF6FFFDFF0500050000E3
:1083B0000007000500F9FFFCFF0700060013001589
:1083C000000500FEFF040010000F000D0015001B4B
:1083D0000009000900120024001B000D0018001CF9
:1083E0000025001E0024001A00190020001D0012A4
:1083F000001800230021001D001B00240011001D97
:10840000002200100008000F00190017000B0002E6
:10841000000500030004000A000A0006000A000A22
:10842000000200F9FF040008000600FBFFFBFF014B
:108430000005000D000F000B000A00FFFFF6FFFE15
:10844000FF0A00170010000A000000F7FFFCFF06FB
:10845000000000FCFFFDFF020004000200F3FFF13A
:10846000FF0200040006000F00FDFFF2FFFBFF010A
:10847000000B000C001000020002000500040006C2
:108480000006000A0005000700080010000A00F3BB
:10849000FFF5FF0100FDFFFFFFFEFFEFFFE9FFEB30
:1084A000FFF7FF0000FCFFEFFFE2FFDEFFEBFFF254
:1084B000FFF1FFF9FFF7FFEFFFF2FFF5FFF2FFF427
:1084C000FFF5FFFCFF04000200FEFF0000030007B1
:1084D000000B000E00080007001800200019000A19
:1084E000000E0012001400140015001500120014F4
:1084F00000190022001F001B001D001A0014001BA1
:10850000001D002200250015001E00270028002560
:108510000022001E001A001E00260032002C002B34
:10852000002F00200019001800140017001F00255C
:10853000002B001A000300FFFF01000C000E0003D7
:108540000003000B000400FCFFFAFFF7FFF2FFEF4F
:10855000FFF1FFEEFFF3FFF6FFF8FFEBFFE5FFE0B3
:10856000FFE0FFE2FFDAFFDAFFDCFFE7FFEAFFE30D
:10857000FFE8FFE6FFE0FFE7FFE7FFEDFFE9FFEDC4
:10858000FFF1FFEEFFF8FFF6FFFBFFF7FFF5FF023D
:10859000000100F8FFFEFF040002000300040007D2
:1085A000000900040002000900100011000C000E78
:1085B000000E000F00170016001100080006000E44
:1085C000000F0011000D0004000200FEFFFFFF037A
:1085D000000B000B00FFFFFAFFFEFFFEFFFDFF0098
:1085E00000FEFF07000E000000F5FFF3FFFCFF0C8C
:1085F000000E000600FFFFFCFF090010000C000A3F
:10860000000D00130010000E0006000800120011FB
:10861000000E000D000F0015001800120017000DCD
:10862000000C0015000F0005000C000E0007000AEA
:10863000000B000E001300160015001300100005BB
:1086400000FDFF09000D000C000B0007000200FAFE
:10865000FFFAFFFEFFFFFFF7FFF4FFFEFFFFFFF350
:10866000FFE9FFE5FFECFFF8FFF6FFEFFFEDFFEAA4
:10867000FFECFFECFFECFFEDFFF3FFF4FFF2FFEB8D
:10868000FFEAFFF1FFF6FFF4FFF0FFF3FFECFFE975
:10869000FFECFFEBFFE7FFEEFFEFFFF4FFFCFFF85F
:1086A000FFF5FFEFFFF0FFFCFFFDFFF7FFFBFF0013
:1086B0000001000100FFFFFCFF05000700060009A4
:1086C00000060008000100FCFFFCFF09000B00058C
:1086D00000070008000500F8FFFBFF03000200FE92
:1086E000FFF7FFFAFF03000400FEFFF4FFF8FFFAB4
:1086F000FFFEFF030000000100FCFF00000100007E
:108700000004000600010001000600040004000847
:1087100000090008000D000F00090001000200051B
:10872000000B000A000A000F000F000900060006F7
:1087300000FFFF07000E0015000C000200030003FD
:1087400000050009000900030001000A000C0005F3
:108750000008000600000009000D00060005000BDF
:1087600000080000000100FFFFF9FFFAFFFAFFFB1D
:10877000FFF7FFEAFFEAFFECFFE3FFE2FFE8FFE7B6
:10878000FFE8FFE1FFD9FFDDFFDFFFDBFFE3FFE3F2
:10879000FFDCFFDFFFE5FFECFFEBFFEAFFE6FFEEAC
:1087A000FFF2FFEFFFEEFFEDFFEFFFF6FFF7FFF643
:1087B000FFF4FFF6FFFDFFFDFFF6FFF3FFFCFFFFF9
:1087C000FF020002000000F7FFF7FF00000500FFB6
:1087D000FFFCFF0000FCFFFFFF000000000400079B
:1087E000000400FBFFF4FFFFFF07000D000C000872
:1087F0000007000C0011000E000B000A000B00091E
:10880000000A0008000B00120016000B000400090B
:1088100000070009000C00090005000B000F001103
:10882000000C00030007000800040005000000FE23
:10883000FF0000040005000100FDFFFEFFFEFFF940
:10884000FFF5FFF3FFF3FFF2FFF1FFECFFEEFFF2A6
:10885000FFF1FFECFFE7FFE6FFE8FFE7FFE0FFE5E2
:10886000FFE4FFE6FFE9FFE7FFEBFFE9FFE8FFE8D2
:10887000FFE7FFEAFFEEFFECFFEFFFF5FFFAFFF97E
:10888000FFF4FFEFFFEFFFF9FFFCFFF8FFF2FFF54A
:10889000FFFBFFFCFFFBFFF8FFFAFFFDFFF9FFF214
:1088A000FFF1FFF7FFFAFFF8FFF9FFF3FFF3FFF81F
:1088B000FFF7FFF4FFF4FFF4FFF7FFFAFFFBFFFE03
:1088C000FFFFFFFEFFFDFFFBFFFBFFFFFF010006B9
:1088D000000C0007000200040007000A000D000B56
:1088E000000C000F000D0010000F000E000D000E18
:1088F0000011000F000C000E000D000D00120015FD
:1089000000180012000F00100012001500140011D2
:108910000012001300130012000E000B000D000ED9
:10892000000D000B00070001000100020000000321
:1089300000FEFFF5FFF6FFF6FFF6FFF6FFF4FFEF90
:10894000FFEFFFEEFFEDFFEBFFF3FFF6FFF2FFEEB1
:10895000FFEDFFEFFFF0FFEEFFE9FFECFFECFFEDB7
:10896000FFF0FFF0FFEDFFEBFFEDFFECFFEBFFEAA9
:10897000FFE5FFE6FFEAFFE8FFE6FFE7FFE9FFEEBE
:10898000FFF1FFEAFFEAFFEDFFEEFFEFFFF2FFF975
:10899000FFFAFFF8FFF9FFFDFFFCFFFBFFFEFFFF03
:1089A000FF0300050007000500050005000500089D
:1089B000000600040006000C000D000D000C000C69
:1089C000000D000D000B000F001600150014001321
:1089D00000130015001400140012001200150017F7
:1089E000001A001A001A001700130011000D000AE7
:1089F000000B000E000E000B0009000C000D00091A
:108A0000000000FEFF000000000000FDFFFAFFFC78
:108A1000FFFFFFFDFFFEFFFDFFFDFFFEFFFFFF0469
:108A2000000300FFFF0100030004000300FFFFFC40
:108A3000FFFDFF00000000FEFFFBFFFCFFF9FFF859
:108A4000FFF5FFF3FFF2FFF3FFF3FFF0FFEFFFEFA0
:108A5000FFECFFE9FFE8FFE4FFE7FFE8FFE5FFE6E3
:108A6000FFEBFFECFFEBFFECFFEDFFEDFFEFFFEEA9
:108A7000FFEDFFEEFFF2FFF5FFF6FFF8FFFCFFFD55
:108A8000FFFCFFFAFFFBFF010005000600070008DE
:108A90000009000A0009000D000F000F001000116E
:108AA0000014001300120011001600190018001A1B
:108AB000001A001A0019001A0019001900190019EB
:108AC000001A001C001B001A0018001300110012ED
:108AD00000130011000E000D000D000B000B000B29
:108AE000000C000B00060006000400030004000256
:108AF00000FFFF0000040007000500FFFF03000364
:108B0000000000040004000300020004000A000842
:108B1000000300FFFF01000300FEFFFBFFF8FFFB67
:108B2000FFFDFFFBFFF9FFFAFFF8FFF7FFF6FFF489
:108B3000FFF4FFF3FFF3FFF4FFF6FFF6FFF3FFF0A0
:108B4000FFF2FFF3FFF1FFF3FFF9FFF9FFF7FFF586
:108B5000FFF7FFFCFFFBFFFBFFFAFFFEFF0000FF3C
:108B6000FF020001000200040006000500040005E9
:108B700000020007000B000A0006000A000F000EAA
:108B8000000D000E000D000B000C000E000C000D7F
:108B90000011001100100010000E00100012001350
:108BA0000012001000100013001400130012000E39
:108BB000000E00120012001200130010000E000E32
:108BC000000E001300150015001400160017001405
:108BD00000150016001400100012001300140015F8
:108BE00000130012000E000C000A00080009000823
:108BF00000080006000100FFFF0000FEFFFCFFFE72
:108C0000FFF9FFF7FFFAFFFAFFF7FFF6FFF8FFF9AA
:108C1000FFFDFFFCFFFAFFF9FFFBFFFCFFFCFFFF7E
:108C2000FF0100020004000500030003000200022F
:108C3000000400050003000300030005000200011A
:108C400000000001000100FFFFFDFFFBFFFCFFFA39
:108C5000FFFAFFFBFFFCFFFCFFFEFFFFFFFFFFFF34
:108C6000FF000000000400050004000700080007E2
:108C700000070008000600060009000B00070006B8
:108C80000009000A000C00080006000700090007A0
:108C90000004000700070009000B00090009000A92
:108CA000000600040003000500040007000B000B91
:108CB000000A000700030004000500030004000789
:108CC000000A000A000400FDFFFBFFFFFFFFFFFB9F
:108CD000FFFAFFFCFFFDFFFAFFFDFFFEFFFDFFFEB9
:108CE000FFFFFF0200030003000000030006000472
:108CF000000200020004000500070005000700094B
:108D000000080006000600070008000B000B000E1C
:108D1000000F000F00100010000F0010000E000DDB
:108D20000010001000110012001100130013000EBB
:108D3000000B000F0010000D000A000700070007DD
:108D4000000400010001000100010000000000011A
:108D5000000000FDFFF9FFF7FFF5FFF8FFFBFFFC48
:108D6000FFF9FFF9FFF8FFF5FFF5FFF3FFEEFFEC6A
:108D7000FFECFFEDFFEEFFF1FFEFFFEBFFEFFFF08A
:108D8000FFEFFFEDFFECFFEDFFEFFFF1FFF1FFF471
:108D9000FFF6FFF6FFF5FFF6FFF8FFF9FFFAFFF722
:108DA000FFF7FFFCFF010002000000FDFFFDFFFBDD
:108DB000FFFCFFFDFFFBFFFAFFFAFFFBFFFBFFFBE2
:108DC000FFFAFFFBFFF8FFF9FFFCFFFCFFFAFFFCD7
:108DD000FF00000100020003000400020008000A76
:108DE00000090007000500060008000D000D000D39
:108DF000000D000B0009000B000B000A000C000A1C
:108E00000008000A000C000C000900050003000423
:108E10000007000300000000000100020002000142
:108E200000020002000200FEFFFBFFFAFFFBFFFC56
:108E3000FFFBFFF9FFFAFFFCFFFAFFF6FFF3FFF37A
:108E4000FFF3FFF5FFF6FFF3FFF4FFF5FFF4FFF389
:108E5000FFF3FFF1FFF1FFF3FFF3FFF7FFF8FFF779
:108E6000FFF8FFF9FFF9FFF7FFF6FFF6FFF7FFFC4A
:108E7000FFFAFFF6FFF5FFF7FFF9FFF7FFF4FFF545
:108E8000FFF5FFF4FFF4FFF4FFF6FFF9FFFCFFFB33
:108E9000FFF8FFF9FFF7FFF7FFFCFFFDFFFEFFFD07
:108EA000FFFCFFFDFFFEFFFCFFFDFFFEFFFCFFFBE5
:108EB000FFFEFFFDFFF9FFFBFFFBFFFEFFFEFFFBD9
:108EC000FFFAFFF8FFF8FFF4FFF3FFF2FFF5FFF7FB
:108ED000FFF5FFF6FFF7FFF7FFF7FFF6FFF6FFF4EA
:108EE000FFF7FFF7FFF5FFF9FFFDFFFEFFFCFFFCBB
:108EF000FFFBFFF9FFFBFFFCFFFDFFFEFFFFFFFE97
:108F0000FF02000300000002000200020001000155
:108F10000001000400030003000000000002000341
:108F20000002000300040003000600040002000128
:108F3000000000FFFF02000300FFFFFEFF0000FF34
:108F4000FFFEFFFFFFFDFFFFFFFFFFFEFFFBFFF840
:108F5000FFF8FFFAFFFBFFFAFFFAFFF9FFF9FFFB4B
:108F6000FFFCFFFDFFFDFFFBFFFBFFFCFFF8FFF831
:108F7000FFF9FFFBFFFDFFFCFFFAFFF7FFF9FFFB27
:108F8000FFFAFFF9FFF8FFF9FFF8FFF8FFF9FFFA22
:108F9000FFF7FFF7FFF6FFF5FFF6FFF7FFF9FFF624
:108FA000FFF5FFF4FFF4FFF7FFF8FFF9FFF8FFF616
:108FB000FFF6FFF6FFF5FFF6FFF6FFF9FFFAFFF801
:108FC000FFF8FFFBFFFBFFFBFFFCFFFEFF010002C2
:108FD0000000000000000001000200040005000382
:108FE000000200020003000400020002000100026F
:108FF0000002000200000000000200020002000166
:109000000003000400030001000000FEFFFFFFFF5B
:10901000FFFEFFFEFF0000FFFFFFFFFFFFFEFFFD63
:10902000FFFDFFFEFFFEFFFEFFFEFFFDFFFFFF0057
:1090300000FEFFFDFFFEFFFEFFFDFFFDFFFBFFFC4F
:10904000FFFFFFFFFF0000FFFFFDFFFDFFFDFFFC37
:10905000FFFBFFFBFFFCFFFDFFFDFFFEFFFFFFFD32
:10906000FFFDFFFEFF0100010000000000FFFFFE0A
:10907000FFFEFFFEFFFEFFFFFF00000000FFFFFE00
:10908000FFFFFF000001000100FEFFFDFFFFFF00EA
:1090900000FFFFFFFF0000000000000000FFFFFFD7
:1090A000FF010000000000FFFFFFFFFFFF010001C4
:1090B000000000FFFFFFFF000001000200020001AE
:1090C000000300020002000200030003000200028D
:1090D0000003000300030002000100010001000181
:1090E0000001000100010002000200020002000273
:1090F00000010001000000FFFFFEFFFEFFFFFFFF79
:10910000FFFFFFFFFFFFFFFFFFFEFFFEFFFEFFFD74
:10911000FFFDFFFDFFFDFFFDFFFDFFFDFFFEFFFE6D
:10912000FFFFFFFFFFFEFFFEFFFFFFFFFFFFFF0050
:109130000001000100010001000100010002000225
:109140000002000300020001000100010001000113
:109150000001000100010001000100000001000108
:1091600000010001000100010000000000000000FB
:1091700000000001000100010001000000000000EB
:1091800000010000000000000000000000000000DE
:1091900000000000000000000000000000000000CF
:1091A00000000000000000000000000000000000BF
:1091B00000000000000000000000000000000000AF
:1091C000000000000000000000000000000000009F
:1091D00000000000000000000000000000F1FF118E
:1091E00000EDFF1500E9FF1900E4FF1000DDFF218D
:1091F00000CDFF2A00A8003CFF55FD3FFD91FF0D6B
:10920000FDAE023402130093002AFFD2004801B2DF
:10921000020900C501F200070086FF25028C003319
:10922000011301C8FE99009BFF74018CFFD3FF3826
:10923000FE6A010C01ADFDAFFFB5001A007A001EF9
:10924000008BFE53FFA2FFC3FFD0FF8EFE04FFF58D
:10925000FF58FF9FFE2BFDFCFF250062FF59FF21F9
:10926000FF160065FFB5FFE8003EFFD9FF170110AC
:10927000FF6C00950065008FFF61FFF600CB00E8F2
:10928000018CFD9801930026FE57012FFF95FEA744
:10929000FFBF00D6FE7F0174FE8B016C003800FC1E
:1092A00001B9FED1030EFF6401E4FF8FFFAE021B84
:1092B000FF1601F3FFF5FF9DFEF600F3FD14FECE51
:1092C000FF470081FF77FFFF00CAFE66FF4BFF8468
:1092D00000CC01810023FFBF009301E50115FFA928
:1092E0000041019600A1006001B1FEE7FEB8004612
:1092F00000B9FFE90048016BFF9E020BFF8EFE5193
:1093000001BFFF17FF1CFE1500DDFEC5FE700071DA
:10931000FFB4FFC8FEF3FF2FFC18007A0095FD4450
:10932000FF10005A02A7FF62FFFDFFC2014BFF08BA
:1093300001DFFF63FFFF01D0FEDAFF70FF7C011D3C
:10934000FE810191FFBCFE6300B7FD2800F9FDAB73
:1093500000DAFF6400F1FFC5FF5C010902C3FE43B0
:10936000FF7101B00126FFC500EE0154FFA6006F9A
:10937000FF220197FEF201A7000DFDDC00FB006B50
:10938000FF5BFE7000A4FF1B00090138FE70FF8B1D
:1093900000CAFF56FFFE00E500720161FF83FD5F1A
:1093A00002A4002800E0FFD8FE0401C30146FF58D4
:1093B000FFE1FF2DFFEEFFC2FF4C00D3FFE0FFB047
:1093C000009B012E01E8FF9CFF49FFB30018FF8FAF
:1093D000FF3E0128FF930036FF1F028DFEC1FFDA1A
:1093E000FF5EFF4EFF54FF9F00DAFFBB02AEFC3171
:1093F000010200540053001700E90065FF49005BBB
:10940000FF8800020067FE9AFF90FF87FF8FFE8BA8
:10941000FE7FFF630037018DFEFC0073FD230166B4
:1094200001C400580039FFB802C901D5FF5E0033FE
:1094300002DFFFD0001AFFA0FF4B001100AFFE3388
:10944000FEABFFFCFF37005FFE6F003FFFE6FF2132
:109450000175FE5D008201DEFFCEFE9401A9FF2FA3
:1094600000DF0157FE60FF5E01AE01B2FE88FEE53F
:109470000047FFB901B2FE5900670118FFC900019A
:10948000FFC0FF60FFBC00ABFE1D0187FE3600651C
:109490000083FFD8FF0C00990149FF81019BFEA1C9
:1094A0000079FFC20162FF03008E00F0FC0C02A1F4
:1094B000FF7601170065FE76FFD8FFD4014EFEDA75
:1094C0000010FEF3FF5801D9FE9601D3FE30FF3E97
:1094D000FFE00175FEFE00B0FF10FF9A01E0FF689B
:1094E0000121FF0D01D000440089FF0D00FEFE9513
:1094F00000B800D0FFDFFEDD00020121FF41FFC9FF
:10950000FFB600DEFF6F00B3FE71003CFF04006396
:10951000011700BFFF1EFEDDFFE801CEFEC7FF2BD7
:1095200000C1FF1A0002019DFF20FE53014B0051B4
:1095300000E1FF2D0059FF41FFB800A00046FF27C2
:1095400000E4018DFEBBFF4601D4FE77FF380139F0
:1095500000D30022FFEE00EBFF7EFF920286FE8723
:1095600000B2FF78012300F2FE1E003BFF6400DD25
:10957000FF17FFEAFF0200D3FF760065FEC7FF3F3B
:109580000067FF86FFA300460069FF7AFE80006542
:10959000FFD500FA00ECFE5000F2008400ECFE5F04
:1095A00001D300C4004900D7FFA50117FE91009622
:1095B000018FFE5E00B6FF5DFFCAFF39002AFE85FF
:1095C00000A0FE44000300F4FE4F00FBFEEF002667
:1095D000000800E0FDD4006700ABFF94001800888D
:1095E000FF1D01920062FF21FF2C01C4FE430047D2
:1095F0000172FEED00D0FEED01AFFEF701CFFEDF00
:10960000004D0055FFB300A8FF7C007EFE08031A42
:10961000FD890201FF270188FFA6FF4400F5FF63D3
:109620000125FE690292FDA3008900F7FF82FFB5C4
:109630000051FF0CFF06FFCCFFC600CFFE22009BAF
:10964000FF35FF1A0192FF4DFEC4009F00F7FF8E09
:10965000FF4001E6FE7501AC00F4FF0301F6FE5C7D
:1096600002ECFFA9FF56010200B200A1FF0A00753B
:10967000006CFFC0FF8DFF3A00DCFEA900D5FED4D0
:10968000FEBD00A3FFABFE29FF0A01E1FF05FF09B4
:1096900001CFFFCEFE4D0228FF380156FEC301B3B5
:1096A0000086FE5701BCFF60FF89FFDC0103FFC29B
:1096B000FF1D004F00090064FF6200CCFFA800619D
:1096C0000150FDD3016300A5FF8100FDFE7E01096D
:1096D000005AFF570090FFA80097FF8FFF35019BAE
:1096E000FE6BFFCCFEDFFF06FF58001C004EFEAFF6
:1096F000FFC40050008800210121FF2000B601288E
:10970000002D00BBFE8300BE0176FFD5002400457E
:10971000FF8900FAFFE1FEEA0014FF3F00A2003BD0
:10972000FF1B0192FE760030005300EDFFE3FF25A2
:109730000140FFBB00ACFEAE0156FF74FFD000023B
:10974000FFDEFEF8FFB3FF67FFFE0030FF4AFF0FAA
:10975000003C006100FFFF60FE910138FF74009D36
:10976000007EFFAEFF35012F0122FE8800C000B54C
:10977000FFCCFFC4004D007DFFF8FF3B0140FF1709
:10978000006300B7FF62FF0A00940009FFAAFFA16F
:10979000FE860185FF65FFFCFFDEFE7601CCFEB490
:1097A0000065FF34FF4001C9FF5600A1FF9A010E7A
:1097B000FFCA000E0085FEBA0230FFE5FFC4FFD9E4
:1097C000FE8D00F00093FEDA0054FF0CFF6501559A
:1097D000FF5B0089000BFE8F000501FEFF7A010987
:1097E000FFECFFFFFFE70164FFD0FFBEFFA3FF0C0C
:1097F00001FEFFBAFFA3FFCDFFA8003D00FFFEC2A0
:109800000057FF91FFF2FF5A00DFFF6400C2FF79AB
:109810000075FF1A006901B4FE52005E006E00B9C7
:10982000FE2E00D4016FFE7D003F0066FF9600888B
:10983000FF3C0196FE5500A900EEFF5F00F3FEFD20
:10984000FF2A009F00E0FEE40086FEF2FF7B001C82
:10985000FFB4FFCEFE7600B4002AFF1800970093F5
:10986000FE6C018900770062FFEBFFD1FF87006784
:1098700000EBFEE4019BFE920068005DFF510018C2
:1098800000F0FF81FFC9FF2600C300B2FECD00AE8D
:1098900000DBFFF0FE0500F3FFB6FF3A0059FE04BF
:1098A0000111018FFF350084FF2E00D0015BFFB84E
:1098B000FF5F002D005B0076001AFFC0FFF700215C
:1098C000FF7D01D3FEE1FF9EFF62FFF000FEFEAAD6
:1098D000000C004100FFFED0003A00E1FE5100B64E
:1098E000FF49017400A1FEF400A4FFB800D300EE0C
:1098F000FE920031007400CBFFD0FE93FFD300EF47
:10990000FE9E0069FF09FF00003DFF6200F2FE2F8E
:10991000006900ABFFEC00D1FFD900BFFFA2FFF14F
:10992000001000D40045FFD200C100290074FFCC14
:1099300000BAFFB7FF620005FFF9FE5500CFFF3602
:10994000FF16012AFE4900B1FFEDFF75FFE3FF0995
:10995000007700D700ACFF910014FF8E01E9FFEB08
:10996000FF2E012CFF1C00E7FF1A001400ABFF754F
:109970000035FF40001F002100ABFF1DFFCF00DAC4
:10998000FF4F003201FBFFBFFF91008BFF34001A35
:10999000006EFFB20085FF1A0082005CFF22004AC1
:1099A0000097FFD9FE8F01E9FF78FF1B0111FF949B
:1099B000001100BDFF3F00A7FFBDFF0400ECFF89C1
:1099C0000071FF5900BEFFB6FF810044FFCFFFE6E4
:1099D000FEA30093FF2B00E0FF76FFAF002A0028D4
:1099E000004000E3FF9EFF8B010FFFC50095FF8540
:1099F000FFB401DDFD3200FCFF5E001FFF75FFCCF0
:109A00000087FF530088FFBE0079FFD6FFC7FF1015
:109A1000006C000B01EAFF6FFFD200F3FFFCFEE2D7
:109A200000360045FF47018CFFCD0088FF7800819C
:109A3000FF130063005BFE6C0012001E00A7FF64B2
:109A400000D5FF0900440003FF9100E2FF9EFF994B
:109A500000270098FF7D0098FF3500B70057FF5F93
:109A600000360072FF680012002B00C000A8FE360E
:109A7000010300170088FFF9FFEDFF09003E0027F2
:109A8000FF010127FFAB00E7FFA4FF2B000BFFE660
:109A900000460001FF21005600350099FFBF00A5D8
:109AA000FEC4003300FCFEBB00EBFE4100FDFF2ABC
:109AB00000ACFF9FFFC2FFC7FF0A00CF0055FF1D8C
:109AC00000BA000C005B0066FF5700D6FFE8FFC13C
:109AD000FF360050FFF9FFF3FF38006900A0FF0ECA
:109AE00000A3FFC7000E0036003300FBFFBE007C62
:109AF00000C0FF9A00C9FFC6FFA20087FFC0FF7D1C
:109B0000001C0002009FFF77FF670029008EFF9A6C
:109B1000FF980073FF5500580008FF4E0107FF54DF
:109B2000008500D8FF4A002AFFA400A6FEF000042A
:109B300000A1FF83FFCAFF0C0163FF220034FF482E
:109B400001C4FFEDFFC2FF84FFC00092FF26004565
:109B5000FFF10024000D000C00CDFFAC00AFFFB6FC
:109B6000FFF6FFF5FFCAFF6FFF4C002400240047FB
:109B700000C3FF18007AFF4E01C7FF82FFCBFF2C06
:109B80000061004F00DCFEAFFF9C003FFFD5FF628D
:109B9000004D0045FF44019FFE09017EFFE5FFDD0A
:109BA000009AFF650033FF9F007CFF6E007CFFEA98
:109BB000FF220088FF7100FAFFFBFFD9FF17004466
:109BC00000F9FF3E0041FFD20097FFE2FF8200EF65
:109BD000FEC700A6FFA100E6FF270093FF0700CD08
:109BE000000CFFA40031FFCC005B00ECFF0E004C2A
:109BF000005000CBFF6A00F6FFC5FF2A00FEFFF50C
:109C0000FF55001CFFD2004CFF0200240039FF6406
:109C100000A4FFD90045FFB0FF4D00C5FEE400B22F
:109C2000FF5E001F0047FFA9002C0003004000A7B3
:109C3000FF190017004C00D7FFF3FE20011DFFBFE6
:109C400000FDFFD2FE7C01AEFFB3FFD40015FF1470
:109C500000580082FFAA00D0FFD5FF020087005005
:109C6000FF7E00000089FFF4FF3700B100BFFECC8B
:109C7000005DFF4D009BFFD7FF460034FF0F01A999
:109C8000FF98FFBCFF4B006000AAFFFBFF5400CD14
:109C9000FFB000DCFFC9FF5000360002001B001CB3
:109CA00000ABFFAC00B6FF74007C0042FF4000E652
:109CB000FF5F00EBFFB6FF600099FFF9FF6600EF62
:109CC000FF0100BEFF1800CFFF1D00C8FF65FFB3F6
:109CD00000D2FF2E0052FFF2FF560089FF1400272A
:109CE00000ADFFFFFF6300F3FFA4FFA500B1FF82FB
:109CF000FFA300C5FFF6FFC5FFDAFF630011009860
:109D0000FF5900AFFF6000630074FF9CFF3D00D36C
:109D1000FFA8FFC00081FF7EFF7A00F3FFF7FF3F3F
:109D200000E3FFC1FF50009F00B2FF9CFF23002A09
:109D30000067009FFF9900CCFFB3FF4C008EFFB57A
:109D4000FF5F0023003CFFF70051FF5800B4FF38CD
:109D5000000E00BBFFD60004FFBD00F4FFD9FF9941
:109D60000077FFE7FF65001F00480062FF6700F013
:109D7000FF340097FFE4FF6400AEFF340054FF3768
:109D8000000E003100BDFF73007AFF0D006200512C
:109D900000DCFFBBFFC600EAFF2700060051007A87
:109DA000FFB300CAFFA4FF4F00F8FFDBFFF2FF2460
:109DB00000160090FFBBFF3700ECFF1B0086FFF290
:109DC000FFC7FF5BFF2900020078FFF2FF38006940
:109DD000FF5B00FFFFB6FFDF00B9FFC2FF2200708C
:109DE00000E4FF6F00F7FF6F00070016001700790F
:109DF0000083FF09004900D8FFAC0065FFE400685C
:109E0000FFB5FF7600FFFF73FF8BFF5000B5FF002B
:109E1000002D0061FFF7FF0C0000009CFFEEFF1318
:109E200000DAFFF2FF5700330002002F005300B9A1
:109E3000FFDAFF6600D1FF2B00E8FF7F0072FF1BF7
:109E400000670097FF4000E0FFAAFF69006600EB93
:109E5000FFF2FF150038000900CEFFD6FF3000FBEF
:109E6000FF11001A00A8FFF4FFDCFF0200EEFF84E0
:109E7000FF01009DFF80FF7200720088FF250069CE
:109E80000083FF20003900D7FFD5FF1600390040BE
:109E90000086FF66002700AAFF5A00B4FF5700FAA9
:109EA000FFF9FFCFFF1F00A6FF480066008BFF00F1
:109EB00000E0FF9F000B00EEFF210086FFD50004AD
:109EC0000081FF9DFF1E008D004CFF6F00ECFF6ABC
:109ED000FF2D00B3FF0200DFFFB1FF0900BBFFB899
:109EE00000C4FF5400ABFFB0001E00FCFFD90044CB
:109EF000FF8700F3FF7400CBFFF7FFEDFF2200F1B7
:109F0000FFD3FFE4FFB5FFA4FF4600B5FF090052F1
:109F100000BBFFF4FF0C00760072FF25007FFF7E80
:109F200000D3FF74FFAA00E0FF97FF1A005A00BA9F
:109F3000FFD0FF42007800D7FFC1FF6D00C4FFF5DE
:109F4000FF5E00A9FFFDFF08000800C9FF4800C62A
:109F5000FFFAFFECFF110044009BFF4400A5FF4CFB
:109F600000E7FF3700F3FF10001800D8FF100016BD
:109F7000005900B2FF29000F000400E1FF4500B7BF
:109F8000FFEFFFE2FF0800F4FFA9FFFDFF2700DC61
:109F9000FF3400DAFF40006200D0FF4300EFFFA56E
:109FA000009AFF54002900C1FFAE005AFF5800B6C6
:109FB000FF90FF4C00F6FFE9FF4CFFA20026FF6573
:109FC00000D6FFF1FF3E00B9FFF4FFDBFF8300AED8
:109FD000FF3F00AAFF7200FCFFF9FFBFFF83006C88
:109FE000FFF5FFE6FF10003E0022FFB80091FF39A9
:109FF000001200ECFFFFFF31000B00D0FF76007372
:10A00000FF2200DFFFEEFF67007BFF3300D6FF0E6D
:10A0100000FDFF1000CDFF15000400C8FF8800BF41
:10A02000FFF3FF8700DCFF2900B4FF29005E00A3D7
:10A03000FF6F00A0FF9900FDFFD5FF0E000700E9AC
:10A04000FFD9FF4400D6FF4100C1FFEAFF11002EF7
:10A05000002900B8FFE3FF170034003100D2FFFAF7
:10A06000FF05001F001800B6FF240005000500CB07
:10A07000FF00000B00E5FF53002DFF4200D8FFC991
:10A08000FF630056FF5B00E8FFF8FF1A00FCFF319A
:10A0900000C1FF23009DFF840034009CFF1700AE29
:10A0A000FFA800D7FF2900E9FFC9FF2B00570030A8
:10A0B00000A5FFF4FF19001700D8FF2A0091FF2226
:10A0C00000E9FFE6FFE4FF1100E3FFD6FF1B00E518
:10A0D000FF3500EBFF3F00E4FF08006600F0FF0FD4
:10A0E000000200C9FF33000300F0FF0A001A00D885
:10A0F000FF09000D00DAFF1E00E0FF1B00C0FFDCBF
:10A10000FF76000B00D1FF1B00AAFF19005800AF1B
:10A11000FFE5FFFFFF5900F9FFDCFF0C00D6FFD67B
:10A12000FF4C000100A3FF410001002900E1FF02F4
:10A13000002600D5FF1C001A00F1FFEAFF1400D32F
:10A14000FFF5FF0300FEFF2400FCFFB8FF4F00C037
:10A15000FFEEFF2A0017001D00BCFF1B00AEFF51E1
:10A16000000B00EEFFEBFFE2FF2B003D00C6FFF609
:10A17000FF1500D9FF5900CCFFDFFF25001B009C15
:10A18000FF27000100F6FF2700CBFF3D000200FD86
:10A19000FF1700D8FFFAFF4E00D7FF0F00F6FF1B96
:10A1A00000F4FFF5FF0200CEFF4000C1FF0C00F0FD
:10A1B000FF060005000B00FBFFDCFF270030001846
:10A1C0000001000500E5FF6100E5FFCCFFFFFFF6A1
:10A1D000FFF2FFBDFF4F00C2FF2100EEFFE3FF458E
:10A1E00000C5FFEBFFE1FF4B00D2FF14003500FD7F
:10A1F000FFD9FF3700E2FFE8FF2500DEFFEEFF2179
:10A20000003300E5FF2200C8FF2200F6FFFDFF0932
:10A2100000E2FFF4FF2500DFFFEEFF1F000600193C
:10A2200000E4FFCEFF1B004300FAFFCFFFE2FF1167
:10A230000008003900BCFF0500EFFF05001500D144
:10A24000FF17000100FAFF11002800EFFF1C00F5C6
:10A25000FFFEFF1D001F00E8FFFCFF060001000CD1
:10A2600000F7FF1400F3FF2700ECFF0D00E7FF2FBE
:10A27000000B00EDFF0E0011000800D1FF2400A428
:10A28000FF2400FEFFF1FFF7FFFEFF0B00D0FF1AD7
:10A2900000CAFF2200EEFFCFFF25001000D5FFF01F
:10A2A000FFEDFFF7FF0500FFFF0400B1FF2F00F5F2
:10A2B000FF0900D6FF3500DEFFF9FF5D0099FF635F
:10A2C00000EDFF1200F8FFE0FF4D00F5FF1000DA8F
:10A2D000FFF9FF3A00CAFF3600DBFF01000F00FC68
:10A2E000FF2000E4FF1300A2FF3F00FCFFF4FF2665
:10A2F00000DFFF240008000700F1FF05000800212F
:10A3000000F0FFF5FF3500DDFF0000FEFFEFFF3737
:10A31000000F00DEFFDDFF09003000DFFF2300BB80
:10A32000FF04002C00F0FFFBFF0E000F00EBFF0FFF
:10A330000001002300FFFF2400E3FF0A00050001E5
:10A3400000DBFFE8FFD8FF2F00DDFFCDFFEEFF159C
:10A35000000C00DBFFE6FFE9FF4900ECFF2300C72C
:10A36000FF50001000F8FFF3FF0800FDFFFCFF297D
:10A3700000C9FF1F00EEFFD5FF0C001800C0FF1D35
:10A3800000F2FFF3FF0C00EEFF5A00D0FFF5FF478D
:10A3900000EAFF2E00DAFF1C000F00F0FF2200F0A1
:10A3A000FF0300DAFF1E00D1FFF7FFF3FFE1FF120A
:10A3B000000000D7FF1D002C00E6FF2300F3FF0381
:10A3C0000013002000F0FF2300FCFF0700EEFF2633
:10A3D000001F00B2FF2F00EBFFF7FF1900F7FFEEA1
:10A3E000FFE0FF28001900CFFF0100BDFFFDFFF3D4
:10A3F000FF2500F1FFA8FF6300F7FFEDFF08000253
:10A4000000FDFF0D000F00DFFF1900F5FF18000031
:10A4100000CEFF1000E2FF2000F3FFF0FFF6FFF098
:10A42000FF400004001100FAFFD7FFFDFF3F0005C9
:10A4300000F1FF0D00EFFF3B000F00D3FF0400DA37
:10A44000FF1E00EFFF1500F3FFE2FF3600EDFF0FE8
:10A4500000D4FF21000600D3FF03000200DFFF2726
:10A46000001F00CFFF18002A00FAFFE1FF0D00F9DE
:10A47000FFEEFF07000B000600E7FFD4FFF4FF101C
:10A48000000100FBFFF2FFFCFF04001D000700E4D9
:10A49000FF12000E0037000200EFFFF8FFF5FF3853
:10A4A00000E3FFEEFFFDFF10002700B4FF120007DE
:10A4B00000E9FF3300DBFF18000000F9FF0700F799
:10A4C000FF0600ECFF2600EBFF0900140001000B63
:10A4D00000F5FF02001B000F00DDFFEBFF3A00FB61
:10A4E000FFE8FF1400C7FF3E001200D0FF0E00F689
:10A4F000FFF3FF2F00E2FFE7FF1C00D5FF2300F171
:10A50000FFE7FF1D00EDFF0800F6FFFAFF1200074E
:10A5100000F2FFFCFF3700F5FFE7FFFCFF13000828
:10A5200000F8FFFFFFEBFF10001900CFFFEEFF1D4B
:10A5300000F6FF1700EBFFFFFF0400F9FFF1FF0437
:10A5400000F4FFFBFF1200F2FFF7FFF3FF1600DB42
:10A55000FF1200FAFF22000000D4FF02001500FFE6
:10A56000FFEDFF3800C9FF1F000400F7FF0300E400
:10A57000FF2700EEFF02000200F9FF00000700FCC9
:10A58000FF0200EFFF11001800D5FF35000600069E
:10A59000001300F7FF05000B001100C9FF210000A8
:10A5A00000F5FF0C00E7FF1500CFFFECFF1500EFF3
:10A5B000FFFEFFFBFF1000F8FF07001F00F3FF0F77
:10A5C000000C00F4FF1C000500FDFF0B0009000457
:10A5D000000A00FFFFF6FFEEFF0500EAFF0D000690
:10A5E00000DDFF010009000600C9FF2C00F2FF0694
:10A5F00000E7FFFDFF2A00F5FF0A00E5FF0F00EE70
:10A60000FF2200DEFFFBFF0E0001000B00F7FFF151
:10A61000FFF1FF1300E6FF1E00F4FF10000900EA3F
:10A62000FF0D000B000D001300D8FF07001C00E514
:10A63000FFE8FFF0FF2A00D9FFFAFFF9FF0300FA55
:10A64000FFF6FFFEFFEDFF2C00F3FFF2FF1200F715
:10A65000FFFFFF17001000E5FF040018000600F5DB
:10A66000FFFDFF1B00FEFF1700F7FF14000D00EEBB
:10A67000FF0B00E8FF0B000900F6FF070003000FC7
:10A6800000DAFF0D00180001000700ECFF210002B6
:10A6900000F6FFFCFF0D00FEFFFAFF0000F9FFECE3
:10A6A000FFF2FF12000200F0FFFBFFF6FFFAFF17B8
:10A6B00000CDFF02002300E8FF000009000300EBCB
:10A6C000FF1600FCFF01000A00DFFFFDFF0C002267
:10A6D00000F9FFECFF11000100FFFF0000F3FFF69F
:10A6E000FFFCFFF8FFFBFF0700F6FF0200FFFFF98A
:10A6F000FF0300F6FF2000F9FFE5FF1D00FDFFF15D
:10A70000FF1200FFFF07001200E1FFFDFF19000C20
:10A7100000DEFFF5FFFFFF1500FDFFE9FFFFFF046F
:10A7200000FAFFF7FF1400FFFF09000A002800EB02
:10A73000FF08000B000D00FBFFEFFF1600E9FFFE16
:10A74000FFEFFF0900FFFFD4FF1D000A0006001BFA
:10A7500000DDFF0C002800E5FFF2FF0A00EBFF1709
:10A76000000200F5FF0B00F5FF0E000E00FEFF08D3
:10A77000000200E4FF13001C00ECFF1500F1FFF5E0
:10A78000FF0C00FEFFFDFFE7FFF2FF1100FFFFF1EE
:10A79000FFF4FFEFFF2B00EEFFEAFF1400FEFF0DBA
:10A7A000000500F1FF02000C00EAFF1400F1FFFBBE
:10A7B000FF0500DFFF06001100F9FFF4FF0F00F2B4
:10A7C000FF05001300F0FF0000150004000300F275
:10A7D000FFF0FF11000500E4FF020014000200F981
:10A7E000FFF5FF1E000100F1FF07000300FAFF1B49
:10A7F00000E7FF02002100E6FF1800F8FF0F00F954
:10A80000FFFCFF0000F0FF0A0003000100EDFF075E
:10A81000000E000100F9FF1F00FAFF0A00FFFFFE13
:10A82000FFF8FF0D001D00E7FF0B00FDFF0B00FD13
:10A83000FFF5FFEFFF1400E9FFE8FFF9FF05000354
:10A8400000F9FFFBFFEDFF1300FAFF1300EAFFF42E
:10A85000FF160004000800FDFFF3FF0900E9FF08F0
:10A8600000F9FFECFF1E00EDFFF4FF05000500F20C
:10A87000FF0400F2FFF7FF110002000700060005C9
:10A8800000FDFF0F000C00FFFF01000800FFFFF5B7
:10A89000FF1700F3FFF5FFF9FFFFFF1B00F0FFFBC1
:10A8A000FF1200FCFF1D00F5FFF6FF1000F5FF0D85
:10A8B00000FCFF0A000200F8FFFDFFF1FF1300009B
:10A8C00000F5FF0D00DFFFFCFFFDFF020006000B9F
:10A8D00000F6FFF4FF1800E3FF1B000200F3FF0681
:10A8E00000FEFF1500F4FFEDFF09000A001300F25F
:10A8F000FFEDFF1100F8FF0400F7FF1000E2FF007A
:10A90000001700F2FF1500F8FFE5FFF6FF0400074F
:10A9100000F5FFFAFF1200F1FF04000F000300131F
:10A92000000A00EBFF1000FDFF01001700D8FFF048
:10A93000FF1F000F00EBFFECFF0600FDFF0A00FF0A
:10A94000FF080006000A000200F2FF1C001800F9D0
:10A95000FFF4FF080001001300EEFF09000200F5FC
:10A96000FF14000C00F1FF00000B00DEFF1000F9E7
:10A97000FFEEFF0200EEFFF1FF0800FAFF0900ED15
:10A98000FFECFF1B00F4FF0800E9FFFCFF0F00F9DC
:10A99000FF090008000000E8FF17000900ECFF199C
:10A9A00000F7FFEEFF0C0001000600EFFF0B0003B5
:10A9B00000EBFF02000F00F7FFF4FF0800F8FF0FA5
:10A9C000000300F1FFF1FF090009001700F1FF0487
:10A9D000000D00F1FF2400F9FF1D00FFFF09000238
:10A9E00000E7FF1000FEFF0400E9FF000002000C7A
:10A9F00000ECFF03000000F1FF0D00FDFFFEFFF47F
:10AA0000FF0D00FAFF04000800FFFFF2FF0700003F
:10AA1000001700F6FF02000C00EAFF0B0010000315
:10AA200000E4FF2000E5FFF9FF0000F5FF0700F359
:10AA3000FFF6FFFFFFFFFFF1FF1600F3FFF5FF102A
:10AA400000FCFFFEFF0900EDFF0C000A000B0008F0
:10AA500000F4FF0C000600FEFF0E000600FAFFF9EE
:10AA6000FFF4FF08000500FBFFF5FFF8FFFFFFFF05
:10AA7000FFFCFF0200E8FF0B00F2FFFCFF0B0002EF
:10AA800000FFFFF6FF1A00EEFF040015000900F5B5
:10AA9000FF040019000200F6FF05000F00FBFFFF96
:10AAA000FF1000F3FFF5FFFEFFF6FF0500050005B0
:10AAB000000300F6FFF8FF0900080001000500068A
:10AAC00000F6FF1E00F8FFFBFF0E00EFFF0800FD81
:10AAD000FF0300FFFFF9FFFCFF0C00000004000271
:10AAE00000ECFF0400F2FF03000400FCFF0300EC95
:10AAF000FF04000D0003000400F3FFFEFFFEFF0B48
:10AB000000FAFFF6FFFCFFF0FF0F00FAFF0100FE66
:10AB1000FF0400F9FFF3FF04000800EEFFF3FF0A53
:10AB20000004000B00E9FF01000C00F0FF1600FB21
:10AB3000FFF3FF1000F0FFFEFF05000C00FEFF0E0C
:10AB4000000200FAFF000009000C00FAFF050009EE
:10AB5000001100F6FF0900FEFF0600F8FF060003E3
:10AB600000F3FFF8FFFBFF0600FCFF0B00F6FFF908
:10AB7000FFF3FF08000000F6FF11000000F5FF0FD3
:10AB800000F9FF0E000C00FFFF0100FAFF1800FEA5
:10AB9000FFFBFF090006000400FAFFF8FF0800EEC3
:10ABA000FFFBFFFEFFFEFFFAFFFEFFF3FFF9FF0AC8
:10ABB00000040003000100F4FF050010000700047A
:10ABC00000F0FF0F00F3FF09000800F6FF0000018E
:10ABD00000F7FF07000600FBFF0500ECFF0300FB8A
:10ABE000FFFEFFFEFFECFFFDFF0D00FDFFFFFF037B
:10ABF00000FDFFF9FF07000C00FCFFEFFF0300085A
:10AC000000F6FF0C00FAFFFCFF12000100F6FF1532
:10AC10000000000C000000F0FF0D000700FDFFFD2C
:10AC2000FFF3FFF4FF1500F2FF0300FFFF03000432
:10AC300000F7FF0800FDFF0200000003000700FC12
:10AC4000FF03000B00F2FFF7FF0B0008000200F803
:10AC5000FFF2FF040001000400FFFF0500FCFFFFFE
:10AC6000FF0A00F9FF06000A00F1FFF4FF0A00FDE9
:10AC7000FF0900FCFFEFFF0A00FCFFFDFF070001DA
:10AC80000009000A00F6FF1100F9FFF7FF0A00F0C3
:10AC9000FF13000000FAFFFCFFFDFFFCFFFBFF0AB3
:10ACA000000400FDFFF1FF02000700FBFF0400109D
:10ACB00000FBFFF8FFF8FF0A00FAFF08000200029D
:10ACC00000010000001200ECFF0B00F1FF07000C78
:10ACD00000F4FFFEFF0000FEFF02000A00F2FF0684
:10ACE00000FDFFEEFF02000500FFFF0300FCFF0375
:10ACF00000020001000700ECFFFBFF0D000100FC5B
:10AD0000FF03000400FFFF0000F6FF0900FBFF0C3B
:10AD1000001400E4FFFFFF1700F2FFF4FFFFFF0144
:10AD2000000B00EFFFFFFFFDFFFFFF040006000721
:10AD300000F5FF0E00F1FF06000400FDFF1900F30F
:10AD4000FFF2FF0900FEFF08000200F5FF180008EF
:10AD500000F8FFF3FF12000100F7FF0500060008EE
:10AD60000000000900FDFFFDFF09000600FEFF04D2
:10AD700000FCFFFCFFFFFF0200FEFFF1FF02000AE4
:10AD8000000200F8FFF5FF010000000600F8FF01D7
:10AD900000FDFF00000800FDFF040002000500FEAA
:10ADA000FFFFFFF7FFF8FFFCFFFBFF0B00FBFFF6C9
:10ADB000FF0000F2FF02000700F7FFFFFF0100069F
:10ADC000000700F4FF0000080008000C000500F573
:10ADD000FFF5FF08000600F6FFF8FF1000FBFFEF8D
:10ADE000FF0100F4FF0B00F9FFFDFF0300F9FF0373
:10ADF000000400070007001000EFFF150005000D1C
:10AE0000000A00F6FF0D00F1FF100006000100FB34
:10AE1000FFFEFFFEFF0300FFFF01000000FDFF0635
:10AE200000EDFF03000400F9FFFDFFFCFFFBFF0F37
:10AE300000F2FFFAFFF9FFFDFF0D0005000200FB25
:10AE4000FF070004000800F5FF1100F4FFF9FF03FD
:10AE500000F9FFFDFFFFFFFDFFF6FF0400050009FD
:10AE600000F4FFFDFF03000A00FFFFFDFFFCFFFFF2
:10AE7000FF0C00050004000000F7FF0500FFFF00C5
:10AE8000000100EFFF0D00F7FFECFF03000300F6E9
:10AE9000FF0300F9FFFBFF0C00FEFF0400FAFFFCBC
:10AEA000FF00000500000002000000010000000D8E
:10AEB000000200020005000800000003001A00EA7A
:10AEC000FFFFFFFBFF0E000A00F1FF0500FEFF0879
:10AED0000003000400FDFF0900F7FFF8FF0F00FA70
:10AEE000FFF9FFFFFFFEFFFEFFFFFFF9FF0A00F47F
:10AEF000FFFEFF0B0001000400F9FF0600F3FFFE58
:10AF0000FF060003000400F4FFF7FF0000FFFF0B43
:10AF100000FCFFFAFFF5FF00001300F7FF0300023B
:10AF200000070007000F00FCFFF9FFFEFF0E000501
:10AF300000F4FF0500F5FF0000F6FF0100FDFFF340
:10AF4000FFFFFF0600FFFFFBFF06000100FDFF05FE
:10AF500000FBFF0600010008000A00F5FFFFFFFEEE
:10AF6000FF100002000200F9FFF0FF0E000500F3E1
:10AF7000FF0400EFFF0D000F00EAFF0000F1FF01EA
:10AF8000000400F6FF02000200F4FFFBFF08000AC5
:10AF900000FEFF07000400FFFF050009000E00F09F
:10AFA000FF06000B00F6FF0500030004000200F698
:10AFB000FF0300F8FF06000E00F1FFFBFFF9FF1092
:10AFC00000FEFFF7FF0500F2FF0C00F8FF0700FF8F
:10AFD000FFFDFF0A0001000900FEFFFCFF01000960
:10AFE00000F9FF09000000F1FF0400FEFFFFFF0170
:10AFF00000F4FFF9FF09000200FAFFFCFF01000660
:10B0000000FBFF0200FFFFFAFF03000700F9FFFC4F
:10B01000FF0800F2FF07000400EFFF0B000600002E
:10B020000003000300030006000100F8FF0D00FD0F
:10B03000FFFFFFFFFF0000FFFFF4FF01000000FC27
:10B04000FFFFFF0300FBFF0400060002000000FCFE
:10B05000FF060002000800000000000200060008D1
:10B0600000FBFF0800F8FF0E00FAFFF0FF100000E1
:10B070000001000800F3FFFCFF020000000100F1E6
:10B08000FF0C00F6FFFCFF0000F7FF0100FFFF00D0
:10B0900000FEFF0700060000000200070005000E8A
:10B0A00000FEFFFCFF010003000900FBFFEDFF07AE
:10B0B000000000EEFF0000FAFFF3FF0100FEFFF9C1
:10B0C000FF0400FFFF0A00FCFFFCFF0B00FDFF0B6D
:10B0D000000600F8FF0B00FCFF01000200FCFF036C
:10B0E00000FAFF0700F7FFF6FF0B00F9FFFDFFFF77
:10B0F000FFFEFF0800F7FF0100FCFF060009000645
:10B1000000FEFFF8FF0E0000000100FEFF07000434
:10B110000005000500EBFF09000200F9FFFAFF023D
:10B1200000FFFF0300FEFF0400020001000800F121
:10B13000FF0B00FEFFFAFFF8FF03000400FFFFFF14
:10B14000FFFEFF090009000600FBFFFAFF0B0006E7
:10B1500000F9FF0000FAFF02000900FBFFF9FF03FE
:10B16000000300FDFFFAFF0800F3FFFDFF0500FBF1
:10B17000FF08000300F8FFF5FF0F00FDFFF4FF0DCF
:10B1800000F9FF0200FEFFFFFF0100FCFF0E00F6CA
:10B19000FF0800FAFF06000300FEFF0600F4FF07A9
:10B1A00000F9FF0600FFFFFDFFF8FF0700010003A5
:10B1B00000FDFFF5FF0D00FDFF07000000F9FF0592
:10B1C00000090000000200FEFFFDFF040002000570
:10B1D00000FEFF0A000000FAFF0700F6FF0600FA73
:10B1E000FFF7FF0300FBFF08000000F4FF0000056D
:10B1F00000000001000000FFFF03000500FFFFF951
:10B20000FF0C00FFFFF5FF0700F9FF0B00FFFFFA3F
:10B21000FFFDFF03000700F8FF0800F3FF0000FF39
:10B22000FFFEFF0A00FCFF0300FDFF050003000610
:10B2300000FDFFFCFF0500FDFF08000100F1FF011C
:10B24000000700FBFFFDFFF2FF0400FFFFF9FF070F
:10B2500000F9FF08000500F8FF02000300000007E6
:10B26000000900FDFF01000100000000000100FED8
:10B27000FFFCFFFCFF02000300F6FF0100FBFF00E4
:10B28000000B000400F7FFF7FF15000600F8FF01B0
:10B290000004000300FDFF04000400FCFFFEFFF5B6
:10B2A000FF03000500FBFFFCFF01000400FBFFFFA4
:10B2B000FF0400FAFFFBFF0C00F5FF03000200FD96
:10B2C000FF01000500040002000B00FAFF0300016B
:10B2D00000000002000100FAFF04000400F6FF0075
:10B2E000000800FDFFF8FFF4FF0C000200F3FF016F
:10B2F00000FAFF0500FEFF01000B00F9FF03000844
:10B300000005000000FDFF0000FBFF0D00FFFFFF38
:10B31000FFF9FFFDFF0500FBFF0C00F8FFF9FF0739
:10B32000000500F8FF05000900FDFF0B00F9FFFF15
:10B33000FF0E000000FAFFFBFFFDFFFFFF0200020F
:10B3400000FCFFF8FFF8FF08000800F9FFEFFF011D
:10B35000000900FAFF0100FFFF0200FAFFFEFF0AEA
:10B36000000100FCFFFEFF04000900FFFF0000FEDB
:10B37000FF06000900F2FF010003000400FDFFFBCF
:10B38000FF0500FBFF0200FFFF0600FEFF00000DAF
:10B3900000FBFFFCFFFFFF0400FFFF0800FFFFF9B9
:10B3A000FF0300FAFF030000000700F8FFF7FF02A9
:10B3B0000006000200F6FF0600FBFFF8FF0100FD9B
:10B3C000FFFCFF0100F8FFF9FF0800030001000087
:10B3D0000000000500000006000300FDFF0500005E
:10B3E000000700FDFFFEFFFBFFFFFF0100F8FF0964
:10B3F00000FFFFFFFF0300FDFF0E000500FAFF073F
:10B4000000FFFF03000900F5FF06000300F4FF063C
:10B4100000FFFFFBFF0200F9FF01000500F4FF033E
:10B42000000300F9FF04000900FBFF03000200FA1B
:10B43000FF0700FDFF0100010005000200F4FFFA14
:10B44000FF06000400F6FF00000400F6FFFBFF000B
:10B450000000000200FDFF040000000200000005E3
:10B4600000050003000600FFFF0900FCFF0900FCC7
:10B47000FFFBFF0700F6FF04000800FDFFF5FF04D7
:10B4800000FFFFFDFF0200F3FF0500FDFFFCFF0AC8
:10B4900000F9FF0B00FCFFFCFF0C00FCFFF9FF01B3
:10B4A000000900FBFFFDFFF9FF0A00FEFFF4FF119A
:10B4B00000FDFFFAFF0700FFFF01000000FEFF078D
:10B4C000000700FEFF0100010001000200FBFFFC7D
:10B4D000FF0800FDFFF9FF0A000300FFFF0100FB6A
:10B4E000FF07000800F5FF02000000FCFF02000358
:10B4F00000FFFFF8FF0000F9FF01000000F7FF0365
:10B5000000020004000700FCFF0700FAFFFCFF0B2D
:10B510000001000600FFFFF5FFFDFFFFFFFDFF0438
:10B5200000FBFF0100FDFF02000100FFFF03000020
:10B5300000FFFFFFFF0500FDFF0400F9FFF8FF0714
:10B54000000200FFFFF6FFFFFF0500FCFF0200FE08
:10B55000FFFDFFFEFF0200030001000100FEFF06E9
:10B5600000020008000400FFFF0500FFFF010003C8
:10B57000000300FEFF01000000FDFF02000100FECD
:10B58000FFFDFF0000FFFFFDFF0500F8FFFDFF06C8
:10B5900000FDFF0400FEFFFEFF0300FBFF030006AB
:10B5A00000FFFF00000300FAFF04000300FAFF069B
:10B5B00000FCFF03000400FDFFFEFFFEFFFEFFFF97
:10B5C000FFFFFF0200FEFF0000FFFFFDFF03000181
:10B5D000000500FDFF000004000000FDFF0500FE67
:10B5E000FFFDFF0200FDFF0400FEFFFDFFFDFFFE6B
:10B5F000FF0200FEFFFEFF00000000FDFF0200034F
:10B600000000000000010002000100010001000034
:10B6100000FFFF0400000000000000FCFFFFFF032C
:10B6200000FFFF0000FFFFFFFF0200FDFF02000020
:10B6300000000000000000010005000000FFFF0303
:10B6400000FEFF00000000000000000100FFFF01FD
:10B650000001000000FFFFFFFF01000100020000E9
:10B660000000000000010001000000FFFFFFFFFFDD
:10B67000FF0100FFFFFFFF0000FEFFFFFF0200FED3
:10B68000FF00000000FEFF01000100FFFF010001BC
:10B6900000FFFF01000000000001000000010001A8
:10B6A0000000000000FFFF0000FFFFFFFF0100019E
:10B6B0000000000000000000000000000001000089
:10B6C0000000000100000001000000000001000077
:10B6D000000000000000000000000000000000006A
:10B6E000000000000000000000000000000000005A
:10B6F000000000000000000000000000000000004A
:10B700000000000000000000000100000001000037
:10B710000000000000010000000100000001000026
:10B720000001000000010000000100000001000015
:10B730000001000100010000000100010001000201
:10B7400000FBFFE8FFD3FFEBFF08000800EDFFD48C
:10B75000FF6FFFD1FE6EFE6CFE5DFE1FFEDAFDC3C5
:10B76000FDD9FDDAFDD7FDCAFDBAFD9BFD82FD982E
:10B77000FDF3FD4EFD7AFDE3FD20FD38FD80FC0765
:10B78000FC79FCB7FCBEFCB4FCEFFC84FDF3FDF8D7
:10B79000FEBCFE9BFE92FE79FD5BFFD2FFCBFFDC81
:10B7A000FF54013D011500C202320110007E0298D3
:10B7B000032002D3FE8BFF910212034703E603C36B
:10B7C00003AB03DD030004F903A203DE03B1039519
:10B7D00003F1030004970340034503D30243020D22
:10B7E00002AE0275035302640278013A00C4001AE3
:10B7F00000B700E5004D01720009FFD6FDA6FCDD93
:10B80000FC20FD5FFD2FFDAEFC6AFCAEFC05FD1EBD
:10B81000FD08FD34FD9FFDF2FDBBFD39FE49FEA68E
:10B82000FE65FE14FDD3FCF0FD87FF06FE50FD9B78
:10B83000FED3FE3CFED5FDFCFD4FFE6CFEDCFD6440
:10B84000FEACFE3EFE5CFE25FE7BFEC2FEA7FE9B1E
:10B85000FFF10089011701F00031017E01E801B21A
:10B86000012F0122018B0195016A013B0161015702
:10B8700001B400A4009B0086004D016F01D100B807
:10B88000FF63FF33004900630003012E01D8000D60
:10B8900001B9007C00C700C00020017701BA008F09
:10B8A000008801CD010E02BB01EB00EC00B501BE2A
:10B8B0000145015001F600F2000B01E2000B0114FA
:10B8C000013B01EF013C02F10196017A010302758F
:10B8D00002FC015201E101DD02E602DF02D40207AF
:10B8E000031603C402C30213034C03260309030017
:10B8F00003FD02D902D502BA02E602FE029E025000
:10B90000023502420246020402EC01C101820181B9
:10B91000017A0198017501DE001500E7FF0700C6F6
:10B92000FF38FFECFEDAFEF8FEADFE1EFEE3FDCFB3
:10B93000FDDBFD17FE2BFECDFD88FD5BFD79FD983F
:10B94000FD7FFD56FD67FD8DFD78FD63FD73FD9A5E
:10B95000FD7CFD43FD3CFD63FD7DFD5FFD30FD2372
:10B96000FD42FD47FD22FD04FD01FD19FD1DFD12F7
:10B97000FD1BFD1CFD1AFD06FDE7FCC9FCEAFC5E93
:10B98000FDBBFDD6FDF8FD5BFE8DFE9CFEE9FE686D
:10B99000FFC0FFDAFFC4FFF9FF61000801A2019AAE
:10B9A00001A201A801BA01CD01CD01BC01B001BFC6
:10B9B00001C401AF01A401A901BF01ED010B0226E1
:10B9C0000234022C021802220237024E02520251A5
:10B9D0000264026B0267027F0299029E029E029F2E
:10B9E00002A102A902C202B502C102E102E702D02D
:10B9F0000284025E0258023A023A022C020202104B
:10BA000002F601E201E101D301D901B10187015B35
:10BA100001040106011D01BA0038001C007F005816
:10BA200000D5FF96FFAFFF94FF0AFFB0FE9BFEB369
:10BA3000FE5AFEEBFDD4FDC1FDC6FDE0FDDCFDBB05
:10BA4000FD9BFD94FD88FD87FD7FFD78FD72FD79EE
:10BA5000FD96FD8CFD7DFDA0FDEDFDFEFDC9FDC249
:10BA6000FDEEFD12FE16FE29FE5EFE57FE1EFEC80E
:10BA7000FDF5FD42FE03FEC1FDDFFD1CFE00FEBA2A
:10BA8000FDBDFD09FE56FE77FE53FE66FE8AFE678B
:10BA9000FE54FE41FE23FE20FE62FEE1FE50FF96B4
:10BAA000FFFCFF3B002800F6FFA4FF9FFFCEFFF145
:10BAB000FF0C000E002C005F0079009D00D80014E0
:10BAC000013A0166019601B701AA01560150018CA5
:10BAD00001B601EA01FB01F201FF01F401EB01F8FB
:10BAE00001100226021702FD01FE010C021B022DAD
:10BAF000023102260235024F025C026B02660273BB
:10BB0000029802B202AB029B02BD020103F902ECF1
:10BB100002D602E60207031903EC0277026D02481F
:10BB2000020B02CE01A20177012701C6007900773E
:10BB300000A800890011009FFF2AFF11FFCAFE59CB
:10BB4000FE2EFE0AFE06FE14FE1DFE06FEFBFDFE98
:10BB5000FD04FEFAFDDEFDD2FDE0FDFDFDF1FDCDB3
:10BB6000FDC0FDC3FDB2FDAAFDB0FDC4FDCFFDC407
:10BB7000FDC3FDC5FDB9FDB1FDABFD9BFD92FD8291
:10BB8000FD7CFDA6FDD9FDACFD9FFDA5FDADFDF441
:10BB9000FDF8FDE0FDCAFDD9FD0AFE2EFE61FEBFE7
:10BBA000FEC6FE8EFE82FEC1FE05FF15FF1FFF4B87
:10BBB000FF4AFF56FFA6FFD1FF1000250058008561
:10BBC000006F006E00A300F2000C01EF00E3002202
:10BBD000017A01BE01BD01A3019201B201EE01197A
:10BBE00002F701D001F90133024302FF01AF01B4B2
:10BBF00001F9010202F501EB01F6010202FC01FB71
:10BC000001E101E001DE01A3019A01AC01B901D615
:10BC100001DE01040212022102230237024F025602
:10BC2000023D020C0213021A020E02FF0100020082
:10BC3000020102FA01EA01CB01CB01A7016B01422B
:10BC40000124011E01E800C200AE00920060000E57
:10BC500000F6FF0500E7FFBFFF8DFF7AFF60FF29B9
:10BC6000FF1DFF34FF33FFFCFEC3FE97FE89FE86F7
:10BC7000FE75FE4FFE22FE10FE17FEF2FDCBFDC943
:10BC8000FDBCFDB7FDADFDACFD9FFD86FD89FD94BE
:10BC9000FDA0FD8AFD71FD82FD83FD70FD60FD5EEE
:10BCA000FD62FD5AFD56FD3FFD38FD45FD51FD5736
:10BCB000FD53FD52FD48FD50FD6DFD96FDB5FDB3F4
:10BCC000FDDDFD38FE89FEBAFEB5FED7FE09FF4751
:10BCD000FF82FF94FFB3FFF3FF42006D00890095E0
:10BCE00000BE0011015201640171019A01DE01FCE4
:10BCF00001FE011402220232023302320232023801
:10BD0000024A025A025A0251024B023C0227022600
:10BD1000022202EC01DD0103020F02F601CD018FC8
:10BD2000018101C401EE01E801C701C901EB010174
:10BD30000209020A02230222021402F901EA01198D
:10BD4000024B023502FA01C2019801890183019870
:10BD50000178015D01660143012201FB00D800BFAB
:10BD600000B700C200A80088006400300027002C43
:10BD700000F4FFA2FF88FF6EFF34FFF2FECBFEC08F
:10BD8000FE7CFE30FE27FE1DFE07FE03FE01FE0EBA
:10BD9000FE09FEDCFDC3FDDEFDEDFDCFFDBFFDD5E3
:10BDA000FDE4FDD9FDD3FDCBFDD4FDD4FDBEFDC129
:10BDB000FDDDFDFFFDFEFDDAFDBBFDB0FDA2FDA832
:10BDC000FDC3FDCFFDC9FDD0FDFCFDFBFDDDFDED9F
:10BDD000FD2EFE5FFE5DFE51FE5CFE80FE9AFEC8FB
:10BDE000FEF3FE0EFF11FF06FF19FF25FF15FF1AD8
:10BDF000FF44FF51FF45FF51FF85FFC1FFF9FF33AE
:10BE0000006B009500B100C400D000D300F7002201
:10BE1000011D011201230122010E012E01430169BE
:10BE20000178017201A301C801D501CA01CA01CE7E
:10BE300001D401DF01060227020D02170236025863
:10BE40000242022A02330246025D024D02530257A9
:10BE50000263024C0235024C026F02750262024C10
:10BE6000022F02270239022C02F301EE01FD0136F6
:10BE700002560236021A020C02E701B60182015490
:10BE800001410124010101CC009D005100E6FFA405
:10BE9000FF84FF4FFF0AFFE4FECAFE9FFE74FE4EC2
:10BEA000FE3FFE26FEFCFDF3FDF5FDF1FDDAFDC6CD
:10BEB000FDC5FDC1FDA7FD9EFDA2FDA2FD9EFD9756
:10BEC000FD8BFD85FD85FD95FD9FFD93FD9FFDA6E9
:10BED000FDA9FDD9FD1EFE44FE1CFEF1FD16FE4B24
:10BEE000FE54FE47FE5BFE8AFEA8FE98FE89FE9F7A
:10BEF000FEB8FEBAFE8FFE79FE97FEAEFEB2FEBB26
:10BF0000FEC7FEC3FECAFECEFED6FEFCFE17FF37FE
:10BF1000FF61FF82FF93FFA4FFC3FFC8FFC6FFE3DB
:10BF2000FF0D0027002A0027001F003D0077008F2B
:10BF300000A500D100F7002001210119012E0151B7
:10BF40000181019901AB01BA01CA01D701EA01FFE0
:10BF500001F101E101E301F5011D021402F501FC0B
:10BF6000011502260213020B020D0204020102FE59
:10BF700001E901E301F20111020E02DD01CE01F837
:10BF800001150216020602E401DD01E701D401BC3D
:10BF900001BF019C01870184017201650157014EB7
:10BFA000013D0139012B011601EE00AD008900723F
:10BFB000005C0038001700FDFFF7FF0500F5FFBC2F
:10BFC000FF74FF4DFF33FF0DFFD4FEACFE94FE5E09
:10BFD000FE39FE35FE31FE22FE11FE03FEFCFD00A1
:10BFE000FEF4FDE8FDE2FDD7FDB7FDA2FDA4FDA531
:10BFF000FD9DFD91FDA5FDBDFDE0FDEBFDDBFDD44F
:10C00000FDC7FDCCFDD6FDC5FDC5FDBCFDC2FDEAED
:10C01000FDFCFD04FE0AFE0BFE2CFE4FFE51FE4B06
:10C02000FE56FE5FFE5EFE6FFE84FEA3FEBBFECBF1
:10C03000FEE2FEE9FE05FF23FF2DFF31FF4DFF7AF3
:10C04000FF8AFFA9FFD8FFF9FF0E003300560063F7
:10C05000008A00BB00D300DF00FC002A0152016708
:10C06000017C01AC01D801E701F4010C02120209C4
:10C070000200020B0214020802FF0103020902F58A
:10C0800001E901EC01F4010202FD01F001E401E02B
:10C0900001EF01FF01F601E101D901EA010702F513
:10C0A00001D401C601C401CB01B501B001B101BB8E
:10C0B00001B801A801A801B601C501C001BE01A5D2
:10C0C00001870177016701520143011801E800D19E
:10C0D00000C800BA008000420024001800F1FFCB25
:10C0E000FFBEFF9CFF5CFF27FF1AFF13FFF3FED587
:10C0F000FED1FEC3FEADFE96FE71FE5AFE41FE3637
:10C10000FE2EFE17FE12FE09FEFEFD10FE15FE17A6
:10C11000FE0AFEEFFDF5FDF3FDE6FDF3FDFEFDF28B
:10C12000FDE7FDDFFDE9FDFAFD00FE06FE18FE223B
:10C13000FE39FE4EFE43FE32FE2EFE32FE3AFE5C1D
:10C14000FE5CFE4AFE58FE7CFE94FE9FFEA9FEBAEF
:10C15000FECDFEDDFEF0FE0DFF22FF38FF57FF6B28
:10C16000FF6FFF72FF8DFFADFFC2FFBCFFC8FFF383
:10C17000FF1A0027002A004A0067008700A700B8BE
:10C1800000DC00EE00E500E000EF00FE00FA00F742
:10C190000005011F011C011701280136014301554B
:10C1A0000171018801870180019A01A901AF01C0D5
:10C1B00001C601C801B301B301BD01C001D001CD69
:10C1C00001C001D001E501E901F001EF01E6010242
:10C1D0000222021B021F021D02110207020E021B95
:10C1E000020302CE01AB01BA01C801B4018F015EA6
:10C1F000014701530142011901FB00E200DA00C7C7
:10C2000000A5008700580033000C00E1FFC6FFB610
:10C21000FF9FFF73FF53FF37FF1AFFFAFEF5FED8AB
:10C22000FEA4FE7FFE79FE89FE6AFE42FE1BFE0131
:10C23000FE0CFE07FEE6FDDEFDEFFD00FEFCFDEF61
:10C24000FDFBFDFAFDE6FDE6FDDBFDBAFDA1FDAE61
:10C25000FDD6FDEDFDF1FDF2FDFAFD0DFE1CFE1615
:10C26000FE21FE3DFE47FE58FE53FE4DFE55FE5B91
:10C27000FE70FE90FEABFEA5FEA1FEBDFEE6FEFB3F
:10C28000FE03FF18FF36FF45FF36FF36FF4EFF5710
:10C29000FF52FF5EFF7DFF95FFA8FFA6FFA8FFC12D
:10C2A000FFDDFFF8FF100029003A0047005C00772F
:10C2B000009D00C200D200C800D400F9000C011B90
:10C2C0000118012B015B017A0183016F017A01A33F
:10C2D000019F019F01B901C901DA01EE01040206C3
:10C2E0000206020902150214020B0210021B0221AF
:10C2F000021802210226021002010206020C0204A8
:10C3000002FF0104020202F901EE01F301F201E66B
:10C3100001D301BB01A70189017F017D0176015392
:10C3200001420150014B0135010B01DE00B900A8AB
:10C33000009B007B0050001F00E8FFCDFFBEFFA563
:10C34000FF80FF57FF43FF30FF12FFDFFEBBFEAA57
:10C35000FE9BFE83FE64FE56FE4EFE4DFE49FE2E03
:10C36000FE24FE25FE22FE17FEFEFDFEFD03FEF36B
:10C37000FDEDFDF1FDFAFD06FE03FEF6FDF5FDFE09
:10C38000FDEFFDFBFD0CFEFDFD03FE0CFE09FE0FA7
:10C39000FE13FE0BFE17FE31FE3AFE37FE4AFE6A22
:10C3A000FE7CFE7BFE78FE87FE9EFEAEFEAEFEAFFE
:10C3B000FEC0FEC1FEBFFED1FEEDFE0EFF15FF1456
:10C3C000FF32FF55FF77FF9DFFBBFFD1FFE6FFEF79
:10C3D000FF0D002A0039004F00650082009900AA75
:10C3E00000C000DB00FB001501230129013A014ACE
:10C3F000015401650171016C015C016C018E01A8A1
:10C4000001AB01AB01C101CC01CD01CF01D201DDF6
:10C4100001E501D901D301DE01F201E401D301D626
:10C4200001D301D901E601EF01D901BB01A601AB9E
:10C4300001B601A7018B0190019C018F0197019C1E
:10C440000192018C01870183018501780158013C2B
:10C45000013301340120010801E900D000CF00CDF3
:10C4600000C200AB008C007A006700410035002C50
:10C47000000A00E0FFB5FF91FF7AFF61FF4CFF2447
:10C48000FFFFFEEBFEE9FEF6FEE5FEB2FE88FE8350
:10C49000FE77FE59FE3BFE3AFE2EFE1DFE0CFEFC14
:10C4A000FDF6FDEDFDE5FDE3FDEFFDF4FDFBFDFA21
:10C4B000FDF3FDF2FDF0FDF0FD0AFE15FE10FE0796
:10C4C000FE0DFE15FE11FE1FFE20FE20FE25FE368F
:10C4D000FE48FE54FE4AFE45FE59FE7CFE8EFE9945
:10C4E000FEAEFEC0FED5FEE6FEEBFEF3FE09FF1D2E
:10C4F000FF2EFF35FF4BFF72FF96FF98FF91FFA2C3
:10C50000FFBDFFE0FFFCFF00000300120038005FEA
:10C5100000700078009300B400CD00DD00EE001143
:10C5200001210135014D01660175017D018B01A4D9
:10C5300001B901B501B401C501CF01C401BA01C2FD
:10C5400001DB01E501E401E201EA01EE01F001F4A1
:10C5500001F7010102FA010102F801E301D901D357
:10C5600001CC01BF01BC01BF01C401B901AB01A2F3
:10C57000019F018B017F017E017801740165015EDD
:10C58000015A014E013A012C01220117010901044F
:10C5900001EC00B9009B0093007C005B00350019A2
:10C5A000001400F6FFD6FFBDFF9FFF81FF68FF4F1D
:10C5B000FF32FF20FF0FFFF0FED5FEC6FEBAFEAB36
:10C5C000FE88FE6EFE75FE84FE6AFE40FE3AFE3672
:10C5D000FE24FE11FE18FE27FE19FE06FE17FE2899
:10C5E000FE31FE2AFE20FE2BFE2DFE37FE3FFE4CC6
:10C5F000FE50FE52FE5BFE6BFE7FFE7BFE63FE4C3A
:10C60000FE61FE82FE93FE99FEA1FEB8FECBFED631
:10C61000FEEAFEF5FEFDFE0FFF21FF2CFF35FF2F8A
:10C62000FF24FF39FF4DFF66FF6FFF71FF8CFFA2F4
:10C63000FFA9FFA7FFA8FFBCFFDEFFF2FF0100FC80
:10C64000FFFBFF140025002E003300430054005F61
:10C6500000730085008D009A00A100AE00C400D0D8
:10C6600000D900E300F6000E012001300141014332
:10C670000144014F016A0181017F017B0183018A2D
:10C68000019A01A901A601AC01B501B601BA01CD1B
:10C6900001D201DA01DC01D501D401DE01DF01DACA
:10C6A00001DD01E101DB01CE01C301BF01C701BF13
:10C6B00001BD01BE01B6019701830179016F015AE5
:10C6C000014701340122011B010301F300CF00B433
:10C6D00000B00099007C005A003C002D001700F1CA
:10C6E000FFC7FFA6FF8AFF70FF4CFF2DFF13FFF768
:10C6F000FEF1FEE1FEC9FEB8FE9EFE75FE5EFE5333
:10C70000FE51FE45FE29FE19FE10FE12FE17FE1A0E
:10C71000FE1CFE18FE11FE13FE0AFE02FE0FFE16A0
:10C72000FE09FE0FFE1EFE2AFE2BFE22FE1EFE1C32
:10C73000FE1FFE36FE53FE5EFE60FE68FE82FE8F2A
:10C74000FE83FE7CFE91FEA8FEB9FEC0FED7FEF879
:10C75000FE09FF0EFF26FF45FF48FF46FF5EFF7AFA
:10C76000FF7BFF7BFF80FF96FFA6FFB0FFBAFFC6EF
:10C77000FFD8FFF4FF0A0015002C004F006500767B
:10C78000008C009200A800C300C200BC00C600D00C
:10C7900000E100F200FF000D011D01240121013024
:10C7A000013E013E014401490146014B015F016721
:10C7B0000162016101620164016B016F0171016F2E
:10C7C000016A0162015F01720176015D015A015E39
:10C7D000015D015F01610165015E015D0155014E71
:10C7E000015401630160015F01630165016701613B
:10C7F0000161016001600159013A011B011E011232
:10C8000001FA00E700D100C600BB00A00087007C51
:10C81000006100470042003D002800FAFFE0FFD21F
:10C82000FFBFFFAFFF8FFF7CFF64FF3AFF0FFFF9F1
:10C83000FEEFFEDDFED0FEC5FEA9FE91FE94FE9A3F
:10C84000FE92FE7AFE64FE65FE6CFE6FFE60FE5593
:10C85000FE59FE55FE53FE5CFE64FE5CFE57FE670D
:10C86000FE62FE5AFE62FE6AFE6EFE73FE6AFE5FA6
:10C87000FE67FE69FE6EFE77FE8EFEA0FEA1FEA69E
:10C88000FEB3FEB5FEC4FEDDFEDDFEDAFEEFFE0DFC
:10C89000FF14FF11FF18FF3AFF55FF5DFF69FF739B
:10C8A000FF7EFF87FF95FFAFFFB9FFC9FFE0FFF2F3
:10C8B000FF02000B00200036004B00630076007F73
:10C8C0000087008F009D00AE00BD00C100C000C504
:10C8D00000CE00DC00E500F000F7000401080113C1
:10C8E000011F011901160120012A012A0125011F3A
:10C8F00001210129012F012401200127012C0126FA
:10C90000012B0142014B01430146014E014A0148FE
:10C91000014001350135014101490153015D0156D5
:10C920000150014C01470149014801470145013EC1
:10C93000013E013501220121012C011F010B01F7EC
:10C9400000D900CB00CF00DF00DC00BE00A30094C4
:10C95000008C007D0059003700290026001000F4EB
:10C96000FFD9FFBEFFAAFF96FF86FF6BFF53FF456F
:10C97000FF3AFF32FF0BFFDFFED5FED1FEC5FEC43E
:10C98000FEBAFEA8FEA0FE9BFE9EFE95FE7DFE6208
:10C99000FE62FE63FE60FE49FE3AFE3BFE3AFE4248
:10C9A000FE37FE34FE42FE61FE72FE6CFE6FFE7BC1
:10C9B000FE7FFE91FEA0FE8EFE82FE8AFE96FEA9FE
:10C9C000FEA9FEA8FEB1FEBAFECFFEE2FEEFFEFD1E
:10C9D000FE0CFF1AFF26FF32FF44FF4FFF5AFF6B8A
:10C9E000FF85FF93FF99FFA9FFB6FFC7FFD4FFDEC6
:10C9F000FFF3FF090010001E002B0030003700403D
:10CA00000052006B007C00880098009D009E00A9E9
:10CA100000B500C300D500DA00D600D800EA00FA5D
:10CA2000000401000103010C01120116011901208B
:10CA30000124013201300126012E013F0143014151
:10CA4000013A01340133014301590164015B015B87
:10CA5000016801700173016F016E0175017001625F
:10CA600001600160016401680165016301680160A2
:10CA70000157014601310133012E011F0116010446
:10CA800001F200DE00CE00C700BC00AA00950089BC
:10CA9000007F0078005D00390028001A00F8FFE2EE
:10CAA000FFD6FFC6FFB4FF99FF86FF6EFF4BFF382E
:10CAB000FF2CFF20FF0AFFFAFEF1FEE5FEE3FED5A4
:10CAC000FEB4FEAFFEB5FEA8FE95FE7EFE75FE6CC2
:10CAD000FE6EFE70FE6DFE6CFE6BFE6AFE74FE7BEB
:10CAE000FE73FE64FE57FE5BFE65FE7CFE85FE80E7
:10CAF000FE7AFE81FE8CFE93FEA1FEA5FEB6FEBF71
:10CB0000FECBFED7FEE2FEE4FED3FEDEFEF8FE0C18
:10CB1000FF04FF00FF04FF12FF20FF2EFF3DFF4434
:10CB2000FF49FF51FF5EFF71FF86FF89FF94FF956C
:10CB3000FFA9FFCBFFDAFFE8FFF5FFF8FF020019BE
:10CB40000028003B004B004E005A006E0073007935
:10CB50000084009100A100AC00B800CB00D300D944
:10CB600000E000E700FA000B010C01180121011F91
:10CB70000125012F013301370147014F01590156AA
:10CB80000156015B01570162017101760176017F57
:10CB9000017F01770169016101630166016E01781E
:10CBA00001760170016E016D017201720161015720
:10CBB000015F015D014B012F0132013D0141013A4D
:10CBC0000120010B01FA00F000E800E500D100BDF2
:10CBD00000B0009A00800072006F0058003C002BEB
:10CBE000001900F9FFE0FFD8FFBFFFA4FF8EFF6F21
:10CBF000FF51FF54FF4FFF31FF20FF0DFF00FFE803
:10CC0000FED1FEB6FEABFEA6FE91FE87FE7DFE7453
:10CC1000FE6DFE52FE32FE30FE3AFE38FE33FE3925
:10CC2000FE47FE3FFE31FE2FFE39FE40FE40FE472E
:10CC3000FE4FFE4FFE4CFE55FE5FFE6AFE74FE7E0A
:10CC4000FE81FE91FEADFEB9FECAFED1FECEFEDF34
:10CC5000FEF4FE00FF05FF18FF1EFF25FF3BFF4D02
:10CC6000FF5AFF63FF73FF76FF81FF95FFA7FFBAAF
:10CC7000FFCCFFE3FFF5FF03000F0021003A004D5A
:10CC80000056005C0061006F00870098009B00A2C6
:10CC900000A800A900B000CA00D200D100D900DC71
:10CCA00000E100E500F800FC00FA00F100F80010D7
:10CCB000011C012301160117011D012B012C012D5F
:10CCC00001300135012B01200129013001390130EA
:10CCD000012C012D01260129012E012E013A0136D8
:10CCE000012E012E012F01290124012A01290130E1
:10CCF00001360136013701330123011B0117010EF3
:10CD0000010B010401F700FF000001F000D500C68F
:10CD100000BB00A6009E008F0084006B00620057DD
:10CD200000400035002A00270021000E00F7FFDC3C
:10CD3000FFBFFFAAFFA3FF90FF75FF61FF4EFF3B00
:10CD4000FF1BFF04FFE5FED1FECEFEC8FEC0FEB015
:10CD5000FEA7FEA9FE9FFE7CFE82FE7EFE77FE827F
:10CD6000FE84FE81FE74FE62FE66FE66FE61FE6368
:10CD7000FE59FE5CFE60FE71FE80FE82FE78FE784B
:10CD8000FE8CFE99FEA0FE9CFE9BFEA5FEB8FECD8D
:10CD9000FED5FEDAFEE3FEECFEF8FE04FF11FF21F5
:10CDA000FF2EFF3BFF4BFF4FFF69FF85FF92FF9D6B
:10CDB000FFB3FFC7FFC8FFD2FFE0FFF1FF01001084
:10CDC0000016001200210037004400590069007865
:10CDD00000870089008F0091009C00AB00C400CF49
:10CDE00000C100C100C800D100CE00D000E200E9BF
:10CDF00000E000DA00DC00E400EC00EB00EE00FCF8
:10CE000000FD00FB000001080117011301150119C5
:10CE100001190113010D011A0113010C010D011774
:10CE2000011B0119011E011D011B01170111010F39
:10CE3000011701170119011901180110010E011044
:10CE40000107010601FC00F000F700F300E900EC27
:10CE500000E500D500C800BD00B000A4009F009907
:10CE6000008D007C006400550045002A0026001A51
:10CE700000FFFFF7FFF5FFF5FFE2FFBAFF97FF9412
:10CE8000FF93FF7CFF65FF57FF50FF42FF36FF28EF
:10CE9000FF16FF03FFF3FEF6FEFAFEEFFEE0FEE1F3
:10CEA000FECCFEB8FEBFFEBEFEADFEA3FE9FFEA7FB
:10CEB000FEB5FEADFEAFFEBAFEB9FEB2FEB4FEB7E1
:10CEC000FEB1FEADFE9EFE96FE9BFEAFFEBDFEAC2D
:10CED000FEA6FEB5FEBEFEC0FEC8FECEFED6FEE439
:10CEE000FEEBFEF6FE0BFF18FF0EFF11FF2DFF4BB2
:10CEF000FF4DFF4BFF5CFF71FF8BFFA0FFA7FFA45F
:10CF0000FFA7FFBBFFD1FFD3FFD6FFD9FFF0FF0381
:10CF10000007000F000C00130028003D00500057D0
:10CF20000061007500850090008D008B008D008EE3
:10CF3000009600A900B300B500C000C000C000CF3B
:10CF400000DF00E200DD00DC00EE00F500F500FA95
:10CF5000000001F700F300000104010401FD00FEE0
:10CF6000000F011D012F01330123011F012A013888
:10CF7000013C012E012E0129012701360143013A0E
:10CF80000120011E011F0114011A012101150111C7
:10CF90000107010E0122011501FE00F800ED00E875
:10CFA00000E100D500C600B800A10084008C008913
:10CFB000007200660054003600250018000700F8D3
:10CFC000FFEAFFE9FFE1FFD1FFB9FFA2FF94FF8372
:10CFD000FF77FF6EFF6DFF54FF33FF2BFF2AFF2EFD
:10CFE000FF23FF1BFF0BFFF3FEE3FEDCFEDFFEE291
:10CFF000FEDCFED8FED9FED3FED1FECEFEB7FEACDF
:10D00000FEB7FEB9FEBDFEB6FEAAFEA6FEA2FEA4B7
:10D01000FEADFEB4FEB3FEA6FEA2FEA4FE9DFEACD7
:10D02000FEBBFECDFED4FED8FEDAFEDAFEE5FEFE45
:10D03000FE0FFF0CFF06FF09FF13FF1CFF3DFF481B
:10D04000FF41FF44FF4CFF62FF73FF73FF77FF8BCD
:10D05000FF99FFA5FFADFFB1FFC0FFCBFFE4FFFBD2
:10D06000FFFDFFFEFF0A001A002A003A00440050AC
:10D07000005000590065007500810077007C009524
:10D0800000A700B100B700B000BD00CB00CF00D9B1
:10D0900000D400CE00DA00F5000201FF00FD00061A
:10D0A0000111011901150117012A0136012E01286C
:10D0B000013601490152014E01510152014C014C0E
:10D0C000014F0143013B01310130013C0138012F87
:10D0D000012C011E011B01220117011E0115011067
:10D0E0000112010401FB00F400E500D200C500C0FC
:10D0F00000C400B5009F009C009D00880071005F87
:10D100000055004900410031001C000E00FBFFECFF
:10D11000FFE2FFD3FFB9FFACFFA1FF9AFF94FF89A5
:10D12000FF83FF78FF67FF57FF4BFF3EFF31FF2B69
:10D13000FF17FF07FFF7FEE6FEE2FED3FEC9FEC2C1
:10D14000FEB9FEAFFEB1FEA6FE8FFE88FE8FFE94F6
:10D15000FE8EFE92FE9FFE93FE86FE99FEA3FEAB20
:10D16000FEB2FEACFEAAFEB9FEBAFEB7FEB8FEC124
:10D17000FED3FED2FECDFEDCFEF0FEFBFEFAFEFF8D
:10D18000FE0AFF08FF16FF25FF35FF47FF4FFF5937
:10D19000FF63FF6EFF77FF85FF91FF96FFA6FFB647
:10D1A000FFC7FFCFFFD3FFDBFFE5FFE8FFF9FF0677
:10D1B000000B001E003000400040003F00490069A5
:10D1C000007A0070006B0085009C009C0096009423
:10D1D00000A500B000B400B900BD00BE00C700D07B
:10D1E00000D800E500DF00DA00E500E900EF00EE1E
:10D1F00000EA00F700FD00EF00F000F100F100018F
:10D20000010201FB00FC00070105010B01140118DC
:10D2100001200118011501290125011E0111010735
:10D22000010D010C010B01070106010201020102BF
:10D2300001FF00F500F000EF00F500F200E700DE6E
:10D2400000D000C900B300A600AA00A000870075A6
:10D25000005C004C0045003A002D001E0014000D3B
:10D26000000D000B00F8FFE5FFE6FFDFFFD4FFC471
:10D27000FFAEFF99FF97FF9AFF85FF6CFF5EFF549B
:10D28000FF43FF39FF3AFF35FF21FF13FFF5FEE1B2
:10D29000FEE1FEE1FEECFEE5FECCFEBCFEBBFEC305
:10D2A000FEBFFEA8FE9DFEA7FEADFEAEFEA0FE9553
:10D2B000FE9DFE9FFEA1FEA7FEA5FEA2FEA6FEAE5F
:10D2C000FEAFFEA9FEB5FEC8FECEFED6FEDAFEE833
:10D2D000FEFAFE07FF11FF13FF18FF26FF3BFF4872
:10D2E000FF55FF59FF53FF67FF85FF90FF8CFF93AA
:10D2F000FFAAFFA8FFA6FFB0FFC8FFE9FFEEFFF4FB
:10D30000FFF7FF0400070000000B001C002F002F98
:10D31000002B00380047004A0050005700610068A9
:10D3200000700079008D009C00A2009D009700977E
:10D330000095009D00AD00B600B900B000AD00BA88
:10D3400000BF00C500DC00EB00F200F800F100EFC8
:10D3500000F700FE00030109010F011E012201195F
:10D36000011E012F013B013C0141013E013201360A
:10D370000140013E01440146013B01320134013CC0
:10D38000013B01350130012301150120011E01057A
:10D3900001FE00FF000401FE00F000E600D900D00D
:10D3A00000C600BA00A7009F008E007B0074006AD0
:10D3B0000061004C0030001D00110009000600F65D
:10D3C000FFD1FFBBFFBBFFB0FF9CFF87FF6FFF627A
:10D3D000FF5FFF4EFF35FF24FF1EFF13FFF5FEDD4D
:10D3E000FED3FED0FEC1FEACFE99FE94FE95FE8DEE
:10D3F000FE83FE71FE6CFE6CFE66FE65FE69FE62DB
:10D40000FE5DFE68FE73FE75FE66FE63FE6EFE7ACE
:10D41000FE75FE72FE74FE78FE85FE91FE99FEA1F9
:10D42000FEA2FEA7FEBDFEBFFEC4FEDBFEF3FEFCB9
:10D43000FE01FF0BFF21FF36FF3CFF42FF50FF5470
:10D44000FF60FF75FF7FFF92FF9CFFA8FFAFFFBA51
:10D45000FFC7FFC9FFD5FFDBFFEEFF08001B002A57
:10D460000033003C003D0042005100640072007136
:10D4700000760088009300A300AD00AC00A900B7BF
:10D4800000D100D600D700DD00E100E800F400FF85
:10D490000006010501110123012101240133013D91
:10D4A0000141013C01490153016601770165015CBD
:10D4B000016701750178017B0177017B017C017CAB
:10D4C000017E017B0181018A017F017A017A017865
:10D4D00001700164015A01470149014A0151014E9D
:10D4E000014501410138012A011C010D01F500ED42
:10D4F00000EA00D600BA00AA009900950078005E04
:10D50000004B002C001C000900FAFFE8FFC4FFA537
:10D51000FFA1FF9AFF92FF7DFF5DFF42FF33FF2FC8
:10D52000FF22FF0DFFF5FEF0FEE9FECFFEB7FEA2E3
:10D53000FE98FE84FE6DFE6AFE5DFE54FE4EFE4BBE
:10D54000FE44FE3BFE32FE31FE33FE22FE14FE0E92
:10D55000FE16FE1DFE2CFE2DFE24FE1BFE23FE31BC
:10D56000FE3EFE46FE4EFE67FE6FFE7BFE8BFE9B82
:10D57000FEA3FEAEFEBBFECDFED7FEDBFEE7FEF653
:10D58000FE05FF17FF29FF32FF3DFF50FF64FF6CD0
:10D59000FF79FF8DFFA6FFB0FFBAFFBFFFD0FFE40A
:10D5A000FFEDFFFCFF0700170024002E0038004BA2
:10D5B00000550067007F0086008C0095009B00AB43
:10D5C00000C200CE00D000D600E500F400FC00F35D
:10D5D00000FE000F0119011D012001250132013A51
:10D5E000013F013D013C0146014501550153014BFD
:10D5F0000156015D01640163016001620167016818
:10D600000168016B01760179016F016201640168B3
:10D61000015E0156015D01680165015C014D014D2E
:10D62000014A014401440143013D012B012001183D
:10D630000113010A01FF00EF00E300D700B900AABF
:10D6400000A2009400850076006300530047002F7D
:10D650000016000600FCFFEFFFDEFFD0FFBBFFA4BB
:10D66000FF85FF72FF69FF57FF46FF36FF2EFF154C
:10D67000FFFEFEF4FEEFFEDAFEC5FEC2FEBAFEB409
:10D68000FEA7FE94FE82FE79FE7CFE81FE75FE659D
:10D69000FE56FE57FE5BFE54FE4FFE4CFE4FFE57FD
:10D6A000FE58FE56FE58FE5CFE61FE6EFE79FE766A
:10D6B000FE7DFE8BFE8FFE94FE96FE9BFEABFEABC8
:10D6C000FEB2FEC0FEC7FED5FEE2FEEDFEFEFE0E81
:10D6D000FF1CFF2AFF35FF47FF5DFF6FFF83FF94AD
:10D6E000FF9CFFAAFFB8FFC9FFD8FFE1FFF1FFF8D9
:10D6F000FF01000A001C00270032004900500055BD
:10D7000000630072007400810090009B00A700A5D8
:10D7100000A900B500B500BC00C400CB00D000D209
:10D7200000D400DB00E400DF00EA00F80003010C95
:10D73000010D0113011701160116011A011E01271F
:10D74000012D012E0127012A01360140013F013937
:10D75000013C014701460134013701460146013CC5
:10D760000141014501420140013301320133012AE7
:10D77000011E011501160114010A010201F600F54E
:10D7800000F000E500E500DB00CE00C600BB00AF06
:10D7900000A2009A0097008E007D006B00580048A0
:10D7A000003E0030002400160010000400EEFFDFF1
:10D7B000FFCFFFC4FFC1FFB5FF9DFF85FF6CFF5C7E
:10D7C000FF54FF4AFF3AFF26FF15FF04FFF8FEEF64
:10D7D000FEE4FED3FEBCFEB3FEA9FEA1FE98FE91C0
:10D7E000FE8DFE85FE7DFE77FE73FE75FE7AFE776A
:10D7F000FE6FFE6FFE78FE76FE70FE69FE6CFE76B2
:10D80000FE75FE7BFE83FE8BFE95FE9AFEA5FEB0A6
:10D81000FEB9FEBEFECFFEE5FEEFFEF3FEF3FE0216
:10D82000FF18FF2AFF33FF39FF4BFF58FF64FF6EDD
:10D83000FF7EFF96FFA9FFB6FFBDFFC7FFD1FFE048
:10D84000FFEEFFFCFF07000A000E001F002C003A4D
:10D85000003D003E004200490058006A0077007514
:10D860000077007F009100A300A800AD00B600C2C1
:10D8700000C600C900D000D700DB00DE00E100E6F2
:10D8800000ED00F100F400F100F600FD0006010DCE
:10D89000010C010A010F011201180118010F0111F9
:10D8A00001140119011801150116011E01170110BB
:10D8B000011601190116011601230123011D01158D
:10D8C00001090108010201FD0000010001F700EB60
:10D8D00000E400DF00DD00D900D400C800BE00C4B1
:10D8E00000BC00AC00A0009C009200870084007B7C
:10D8F000006B005D004E0046003F00270017000D42
:10D90000000500F8FFE3FFD7FFC9FFC0FFB2FFA08B
:10D91000FF91FF89FF82FF6DFF5CFF57FF4CFF3BCC
:10D92000FF33FF31FF2BFF18FF07FF04FFFEFEF759
:10D93000FEEFFEE3FED8FED0FEC7FEC0FEBDFEB881
:10D94000FEB2FEB5FEBCFEB8FEB0FEABFEAEFEB54E
:10D95000FEB6FEAFFEACFEB5FEB9FEBCFEC4FECE0A
:10D96000FED3FED7FEDCFEDEFEE3FEE9FEF2FEF9AC
:10D97000FE00FF0BFF16FF1DFF22FF2FFF3BFF4B9B
:10D98000FF55FF5CFF67FF7AFF8EFF99FFA2FFB58F
:10D99000FFC0FFC6FFD0FFE1FFF4FFFDFF0500164B
:10D9A00000220026002F003B004B0057005E006560
:10D9B00000720079007D007F0083008C008F00934F
:10D9C000009C00A900AC00AB00AD00B200B200B4F6
:10D9D00000B700BA00BC00BA00BD00C400C300BF5D
:10D9E00000BF00C400CA00CE00CF00CA00CA00CFEA
:10D9F00000D200D300D400D200CF00CE00CF00D0A0
:10DA000000D000D200D100CB00C700C900CB00CDB0
:10DA100000C700C000BE00BF00BE00B700B400B821
:10DA200000B500AB00A400A100A100A100990092E4
:10DA3000008E008C008D008A00850081007D0076BC
:10DA4000007200700069005F0055004C0048004AF9
:10DA500000400031002B0024001A000E000200FAE2
:10DA6000FFF5FFECFFE3FFD6FFC8FFBDFFB4FFAB40
:10DA7000FFA0FF97FF8EFF87FF81FF78FF69FF5EA2
:10DA8000FF53FF4EFF49FF3BFF35FF2EFF22FF18DC
:10DA9000FF12FF0EFF0CFF0CFF03FFF8FEF8FEF96C
:10DAA000FEF9FEF8FEFAFEFBFEF7FEF4FEF9FE02BA
:10DAB000FF03FF05FF0BFF0DFF14FF1BFF23FF26D6
:10DAC000FF2AFF31FF39FF3FFF44FF4DFF55FF5E47
:10DAD000FF66FF6CFF71FF7BFF83FF8CFF97FFA04A
:10DAE000FFA9FFAFFFBAFFC3FFC9FFCFFFD6FFE219
:10DAF000FFECFFF0FFF9FF000007000D000F00181A
:10DB000000200027002B00300038003E003D004080
:10DB10000045004B0053005600560059005D00625E
:10DB20000065006A006B006C00720074007700777B
:10DB3000007000700075007C0080007F007F008115
:10DB400000830084008300800085008A00870081B4
:10DB5000007F008500890088008400830086008C97
:10DB60000090008F008F0091009500970096009420
:10DB700000940098009800960096009400950093F9
:10DB80000090008F008F008E008C00860084008241
:10DB9000007C0079007A007A0076007100690067E5
:10DBA0000065005D005700540052004C0044003CEA
:10DBB0000034002F002A002100150010000B000681
:10DBC000000000F9FFF1FFE9FFE2FFDCFFD4FFCA2C
:10DBD000FFC4FFBEFFB4FFAAFFA3FF9DFF95FF8C0C
:10DBE000FF83FF7EFF78FF73FF6AFF62FF5FFF5ACC
:10DBF000FF58FF55FF52FF4EFF49FF47FF46FF44C6
:10DC0000FF40FF3EFF3CFF3AFF3BFF3CFF3CFF4035
:10DC1000FF43FF44FF46FF49FF4BFF50FF54FF58AF
:10DC2000FF5EFF62FF65FF69FF6EFF76FF7AFF7E92
:10DC3000FF84FF89FF8EFF93FF9AFF9DFFA0FFA740
:10DC4000FFAFFFB3FFB7FFBDFFC4FFCBFFD2FFD7CE
:10DC5000FFD9FFDEFFE2FFE7FFEBFFF1FFF5FFFA81
:10DC6000FFFCFFFDFF0000030007000A000E001389
:10DC7000001400150017001B001F00230028002CB3
:10DC8000002E00310037003B003D004000440049B9
:10DC9000004E0050005100540058005D00610065C6
:10DCA0000068006A006E0071007400750079007CE5
:10DCB000007D007E00800085008B008B008A008B39
:10DCC000008F0092009200930097009900980096B0
:10DCD0000095009500940094009500960097009799
:10DCE00000950093009300930090008C00890086BB
:10DCF00000840082007F007D00780070006B006966
:10DD00000067005F00570050004D0047004000389A
:10DD10000033002D0024001B0014000D000600FF3E
:10DD2000FFF8FFF2FFEBFFE5FFDEFFD6FFD0FFCBF2
:10DD3000FFC4FFBDFFB8FFB4FFADFFA6FF9FFF9775
:10DD4000FF91FF8EFF87FF82FF7FFF7CFF75FF71D2
:10DD5000FF71FF6DFF68FF67FF67FF63FF5FFF5C99
:10DD6000FF5AFF58FF55FF52FF52FF52FF51FF521B
:10DD7000FF53FF55FF58FF59FF5CFF5FFF61FF63D3
:10DD8000FF65FF68FF6EFF72FF77FF7BFF7DFF81FE
:10DD9000FF84FF8AFF8DFF90FF94FF9AFF9FFFA5EE
:10DDA000FFADFFB2FFB5FFBAFFC3FFCCFFD2FFD775
:10DDB000FFDAFFDEFFE6FFEAFFECFFF1FFF7FFFC13
:10DDC000FFFEFF000006000C001100150018001EE9
:10DDD00000230028002C002F00320035003A003CC0
:10DDE000003E004200470049004A004B004D004FF2
:10DDF00000530058005D006100630067006B006E17
:10DE0000007200750079007D007E007E007F00803A
:10DE100000830085008600870087008800880088CE
:10DE2000008700850084008600860082007F007FD6
:10DE3000007E007B0078007500730070006E006C3F
:10DE4000006B006800650062005E005A00550051DA
:10DE5000004D004A00450041003D003900370032C6
:10DE6000002C002800260023001F001A00170014B1
:10DE70000010000C0007000200FEFFFAFFF5FFEFA4
:10DE8000FFE8FFE4FFE0FFDBFFD5FFD1FFCDFFC8D8
:10DE9000FFC3FFBEFFB9FFB6FFB1FFACFFA7FFA1F5
:10DEA000FF9DFF9CFF99FF94FF91FF8FFF8EFF8CDA
:10DEB000FF8AFF89FF87FF87FF86FF86FF85FF8632
:10DEC000FF86FF85FF85FF86FF87FF87FF88FF8A24
:10DED000FF8BFF8DFF8EFF90FF92FF95FF98FF9BBA
:10DEE000FF9EFFA1FFA4FFA6FFA8FFACFFB0FFB4F9
:10DEF000FFB6FFB7FFBCFFC0FFC3FFC7FFCBFFCF1D
:10DF0000FFD3FFD6FFDBFFE1FFE5FFE8FFE9FFED11
:10DF1000FFF1FFF5FFF8FFFAFFFEFF010004000725
:10DF20000009000B001000120016001B001E00204C
:10DF30000022002300260028002B002C002F003098
:10DF400000330036003800390039003B003E003F06
:10DF5000004100420044004500440045004600479F
:10DF60000048004900490049004B004B004B004D60
:10DF7000004F00500050004F004E004D004C004C30
:10DF8000004E004D004B004A004A0049004800473F
:10DF90000047004600450046004500430041004060
:10DFA000003D003A00380036003500330031002FC4
:10DFB000002E002B00290026002500240021001F30
:10DFC000001D001B0018001500130010000D000CB0
:10DFD000000B0009000600040002000000FEFFFB29
:10DFE000FFF8FFF5FFF2FFEEFFEDFFEBFFE8FFE6C6
:10DFF000FFE2FFE0FFDDFFDCFFDAFFD8FFD5FFD156
:10E00000FFCFFFCEFFCCFFC9FFC8FFC7FFC5FFC2D0
:10E01000FFBFFFBDFFBCFFBBFFBAFFB8FFB7FFB636
:10E02000FFB6FFB4FFB3FFB2FFB2FFB2FFB2FFB360
:10E03000FFB4FFB5FFB5FFB5FFB6FFB8FFBAFFBC31
:10E04000FFBDFFBEFFBFFFC1FFC3FFC5FFC7FFC9C5
:10E05000FFCBFFCDFFCFFFD1FFD3FFD6FFD9FFDB33
:10E06000FFDDFFDEFFE1FFE2FFE4FFE5FFE7FFE9A1
:10E07000FFEAFFEBFFEEFFF1FFF4FFF7FFF9FFFB15
:10E08000FFFEFF010003000500070009000C000D62
:10E09000000F0011001100130013001400160018E7
:10E0A0000019001A001B001D001E001F0021002285
:10E0B0000023002500270029002A002B002B002C1C
:10E0C000002D002D002E002F0030003000300030D9
:10E0D00000310031003000300030002F002E002DC4
:10E0E000002D002C002C002B002B002A00290029D9
:10E0F00000290029002900280029002A00290028D9
:10E1000000290029002800270027002800270027D1
:10E11000002600250024002300220021001F001EED
:10E12000001D001C001A0019001700160014001230
:10E130000010000F000E000D000B00090007000684
:10E1400000050003000100FFFFFDFFFBFFF9FFF7E3
:10E15000FFF5FFF4FFF1FFEEFFECFFEBFFE9FFE758
:10E16000FFE6FFE5FFE4FFE2FFE1FFDFFFDEFFDCAC
:10E17000FFDBFFDAFFD9FFD8FFD7FFD6FFD5FFD5EA
:10E18000FFD4FFD3FFD3FFD2FFD1FFD1FFD1FFD107
:10E19000FFD1FFD1FFD1FFD1FFD1FFD2FFD2FFD2FC
:10E1A000FFD2FFD3FFD3FFD3FFD4FFD5FFD6FFD7D6
:10E1B000FFD8FFD9FFDAFFDCFFDEFFDFFFE1FFE37F
:10E1C000FFE4FFE5FFE5FFE7FFE9FFEAFFECFFED16
:10E1D000FFEEFFF0FFF1FFF3FFF5FFF7FFF8FFFAA7
:10E1E000FFFBFFFCFFFEFFFFFF0000010002000439
:10E1F0000006000700080008000A000B000C000DD4
:10E20000000E000E000F001000100011001200128E
:10E210000013001400150015001500160017001754
:10E22000001800180018001800190019001A001A28
:10E23000001A001A001A001A001A001A001A001B0D
:10E24000001B001C001C001C001C001C001C001CEF
:10E25000001C001B001B001B001B001A00190019EA
:10E2600000190018001800170017001600150015F7
:10E270000014001400140013001200120012001108
:10E2800000100010000F000F000E000E000D000C1B
:10E29000000B000A000A000900080007000600063B
:10E2A0000005000400030001000100FFFFFEFFFD68
:10E2B000FFFDFFFBFFFAFFF9FFF8FFF7FFF6FFF6A0
:10E2C000FFF5FFF4FFF3FFF2FFF1FFF1FFF1FFF0C5
:10E2D000FFEFFFEEFFEEFFEDFFEDFFECFFECFFECDD
:10E2E000FFECFFECFFEBFFEBFFEBFFEBFFEBFFEADD
:10E2F000FFEBFFEBFFEBFFEBFFEBFFEBFFEBFFEBCE
:10E30000FFEBFFECFFECFFEDFFEDFFEDFFEEFFEEAF
:10E31000FFEFFFEFFFF0FFF0FFF1FFF2FFF3FFF37E
:10E32000FFF4FFF4FFF5FFF5FFF6FFF7FFF7FFF847
:10E33000FFF8FFF9FFFAFFFBFFFBFFFCFFFDFFFD0E
:10E34000FFFEFFFEFFFFFFFFFF00000000010001D6
:10E3500000020002000200030003000400040004A5
:10E360000005000500050006000600060006000680
:10E370000007000700070007000700070007000765
:10E380000007000700070007000700070007000755
:10E39000000700070006000600060006000600064B
:10E3A0000005000500050005000400040004000449
:10E3B0000004000400030003000300030003000343
:10E3C000000200020002000200020002000200013E
:10E3D0000001000100010001000100010001000036
:10E3E00000000000000000000000000000C5FF5712
:10E3F00003AEFE00FC19FC14FC00FCB6FEB300A347
:10E4000000090231007B025F018301D3007900071C
:10E41000010100DFFF1003000400047801F5FF0E86
:10E42000FF57FE4AFF19FFF4FF8501D1014F013A62
:10E4300000F9FD99FFC2FFD7019201990089FF629F
:10E44000FE00FD04FD85FD77FD47FE91FEB3FEDE77
:10E45000FEDBFF61FFFCFF00022F01BC01870311FF
:10E460000364032201A3002D00BAFFEFFF3C00C2AA
:10E47000FFC4FE21FF5CFF4C008A00D2FFCAFEEE03
:10E48000FEF9FEF4FE0BFE47FD34FEB4FEF4FE6A18
:10E49000FFDCFF4C006B00F900F8010A023B02DDD3
:10E4A00001BD0060008D003500E4FF72FFF1FFED5B
:10E4B000FF6EFFD4FF19001D00E6FE58FFFDFEC8E9
:10E4C000FE6FFF68FFA5FF97FFCDFF4A00E500B98B
:10E4D00000CD008100F0FFEDFFBFFFADFFCCFF13CB
:10E4E00000CAFF5FFFC2FFCDFFBBFF54006A001CE4
:10E4F000002600C9FFE4FF0400DDFFC2FFF4FF17A0
:10E5000000E8FFECFFD5FFFAFFCBFF080000000F8B
:10E51000001D000F00D9FFD9FFF1FF0000FBFF6EC7
:10E52000FFA5FF81FF92FFE6FF1B00510069004835
:10E53000004000DFFF94FFADFFE7FFFCFFE5FFE9D0
:10E54000FF18006C0034001D0017000200F2FFB835
:10E55000FFB1FFACFFC7FF0500E1FFF1FF1600248C
:10E56000001B00FAFF06001D0027001B00EEFFD86D
:10E57000FFC4FFB8FFADFF8FFFCAFFE2FF0F0031FE
:10E5800000200039000D002300F4FFD8FFE7FFF062
:10E59000FFF9FF0500F9FF1B001400FBFFFFFFC19F
:10E5A000FFC0FFB6FFE6FFFBFFE2FFDBFFEDFF036F
:10E5B000001500F2FF2700FCFF0900D9FFDCFFC4B3
:10E5C000FFF9FFD9FFF7FFEFFF0C0001001E000F5E
:10E5D00000140019000B003A0005007E00A5FD2B79
:10E5E000038D02A9FD14FD00FC4DFC00FC43FC8BD7
:10E5F000FCA0FF01020004FD03E003F403B70331B4
:10E600000140FD3CFEEAFD00FC28FCEEFCABFC9466
:10E61000FE4801AE02E203B303C9038B03EA02DD45
:10E620000116FF9FFEFCFC01FD0DFE48FEC3FD4FE1
:10E63000FF6F016D00ED00D1FFB4016B0118FE8882
:10E64000FD0FFFACFEE2FF5B02EE01E00226003CA4
:10E65000FFFDFF47FF59FFB400C6010FFF75FD7BAB
:10E66000FE89FF3F001A018901CC009301F9005196
:10E67000004C0087FF41FFF0FF1900110047FF0029
:10E68000FE70FFC7FE6DFE4AFFA5FF1EFEF7FD48A8
:10E69000FF0A0093004A016F01FD00D5016F019B45
:10E6A000014C0240029D01B400AEFF9FFE8CFEB201
:10E6B000FDC0FC4DFDF0FDF7FE2DFF8BFF9500C961
:10E6C00001A4010601C6001C00A4FFC2FF64009A59
:10E6D00000EAFFA8FF9C0044010F01220053FF67DE
:10E6E000FFEEFFA4FFF6FFBFFF9AFFD5FFB2FF3199
:10E6F000003200BCFF35FFFAFE34FF76FFBFFFC9D2
:10E70000FFDDFF6800BC00880018000500DDFF2B5E
:10E71000007400920079008D009900C8FF5EFF62CE
:10E72000FF51FF45FF9DFF03004F00F6FF0300610F
:10E73000009D007A006D005100ECFFE4FFD9FF0757
:10E7400000E0FF0C000000F2FFC5FFFBFF1F00D33D
:10E75000FFDCFFA8FF6DFF16FF82FFFFFFEDFF0547
:10E76000002800300075006900F9FF350042002BD9
:10E77000002100D6FFE9FFB6FF8AFF3AFF88FFDDE0
:10E78000FFEDFF1C0042007B0064003900D3FFF165
:10E79000FF02004100540060003F00DFFFD4FFAEE5
:10E7A000FFDBFFE1FFCBFFC3FFD7FFCDFFA0FFDB08
:10E7B000FF110025001A001F005A005B0059005B82
:10E7C000000D00E9FFBEFFD2FF0100FFFF1500EBC7
:10E7D000FFB6FFC2FF9DFF9FFFADFF92FFBAFFB7DD
:10E7E000FFD0FFBFFFB7FF90FFB8FFD8FF0900269B
:10E7F00000450047007500780096009C0093006A71
:10E80000002300F0FFBFFFB9FF98FFCDFFB3FFD299
:10E81000FFA4FFE3FFB1FFE4FF86FF010078FF2EB6
:10E8200000A3FE0BFC00FCB1FC7DFEA10000040077
:10E83000049B03810051FD810194026501BE03A484
:10E84000020004880070FDBCFE6EFF46FEFCFD75F4
:10E85000FE3BFECEFD00FCA3FDD8FF35FFAD00E67C
:10E8600000EF003A02250044FEB1001503F2FD6EF0
:10E87000FE09FF16FEFE000B029F00630072FFF808
:10E88000006D011E0266035602E603F202B2011B8E
:10E89000FED6FC2FFC00FC0DFC83FD07FEA80053F8
:10E8A000FFC3FD84FF11FFDAFFEE020004B903B7D6
:10E8B0000350007A01A6001801F3003AFFE5FE615B
:10E8C000FECBFD15FEC6FE0DFF42005B00A6FF2736
:10E8D000FF68FE7DFDDAFEB7FE660047000700D543
:10E8E0000044005901200267017B016601120231D8
:10E8F0000250005DFFC3FF9BFFCDFDC9FE3BFFB98A
:10E90000FE28FE01FF0EFF94FFED005E001C00B824
:10E91000FF1E00DA00E4009DFFA3FFCAFF9B006A10
:10E9200001F0003301C8006600F2FF07FFC1FEFAE4
:10E93000FE21FF5AFFF0FE21FF12FFDBFE9AFF6F60
:10E94000FF69FF7FFFD4FFD1FF8D00FC00CF009750
:10E9500000F2FF3E002800BBFFEBFF6E00D5FF8DED
:10E96000FFDBFFFCFFA8008A0051009B00620072E1
:10E97000006E007900DA00AF000800AEFF6FFFFE06
:10E98000FE3AFFF3FFC5FFA3FFAEFFD9FF69004DBD
:10E9900000430046003D001B00E1FF91FFB4FFB6BD
:10E9A000FF88FF2AFF1DFFF9FEDBFE21FF24FF8CFD
:10E9B000FFE6FF2200670065009600C400C6008CD9
:10E9C00000A000B4009E00470029002600E3FF4994
:10E9D0000027002A0003001C00F7FF1D0082FFC172
:10E9E000FF50FF76FF88FE58FC00FC51FC01FC0B39
:10E9F000FEB30300048F030004B0030004D201E758
:10EA0000FE7E0286FF2E00A1027C00C0FE22FEAA2E
:10EA1000FC66FE97FEE7FFA503A601B4FF27FC10E6
:10EA2000FC8DFDF4013702E5004AFE39FF00012AA2
:10EA3000020C033200B200DBFE7BFE6AFF64FE4B79
:10EA4000FDD5FEBBFEC8FEC4FE8AFF6902D50300E9
:10EA5000044202290177006B00FBFF56FC8DFCF29B
:10EA6000FC47FDEF000301E300C30043FFC2FD8547
:10EA7000FDB4FF5EFE63FCBBFCC3FFD600F0FFB835
:10EA8000FF8900EF03AA03A9022602F602000497F9
:10EA90000345036701B000BA0045FD96FC4CFC003D
:10EAA000FC01FC06FC00FC85FC1D00CB017A03592F
:10EAB00000BDFED800BA010004FD02280114029E28
:10EAC0000289030004510313013600FDFE1DFEBB45
:10EAD000FF11FD00FCB6FC45FC30FCD1FC42FCA162
:10EAE000FCFFFD6FFF6F021A012B023F023902C3C8
:10EAF000039603C703D501A8006600B4FFEAFC0F24
:10EB0000FE96FF6EFD00FC1BFE62FEDBFFBD0223D6
:10EB1000036202BF01F6008D010002A2FF1101A3F2
:10EB2000FE25FE8BFE8F0030011C01CEFF8FFE35CF
:10EB3000FE23FD21FE360062FF20FD0CFF050026AE
:10EB400002100189FEADFEA7007D000C024201F516
:10EB5000013A03EE03B101EFFDACFC00FCF6FE5DF3
:10EB6000FF28FF2B00C8012F03A501A3FEE2FD1B18
:10EB7000FEBEFDF0FD90FF27FF650085FFC1001E72
:10EB80000187FD28FF89001402B502D401D102F1EA
:10EB90000332014900B0FFEFFDC0FDB7FE68FFF68C
:10EBA000FEF0FD0FFFF2FD57FE8A00C901F601B528
:10EBB000FDC6FF04011F02C80255026A00D8FE5BB1
:10EBC000FFE2FD43FE3EFD76FE8BFD81FD35001F1D
:10EBD000009D02AD03C7020603FC012102DD005EB9
:10EBE000FD86FD6AFE89FF08FF53FC46FCC1FE6CF2
:10EBF000FF19003E01E400C0024902FA008A0159EF
:10EC0000022700E1FEF8FE87FD2CFD73FC25FCFBCE
:10EC1000FC4CFE73FF34FF0901F202AF03EA03B3B9
:10EC200002C402BE0104014701A5008BFF3FFFCED5
:10EC3000FDEFFD8EFD72FD8DFEA0FF1D0041013335
:10EC400001A1004002F900FCFEF8FFF600BDFDCC7A
:10EC5000FEF0FFB7FE70FEB3FD4EFE91FF8E005F2B
:10EC600002D802270279015300030046FFC5FF2A9C
:10EC70000060FF23FECEFE9DFE350053010000BD67
:10EC8000FF59FF8000560203024E00BE00DD001B4C
:10EC9000022901B000E2006E00EAFF07FD3DFC5DC5
:10ECA000FC98FCCAFD10FFFEFFE4FF6AFFFEFE6356
:10ECB000FF0702F201A900D7004401FC019101699C
:10ECC000FF26FE7DFEF1FE1C012E0263014C003684
:10ECD000FF0600F400BD0041FFFBFD23FE2BFFA952
:10ECE000FDDEFC09FE25FEEFFF6E00AE027B038C0D
:10ECF00002F00192FF43005F001B00D0FF7B001F6A
:10ED000001310021014DFFBCFD3CFE94FF07006472
:10ED1000FF87FF8DFEBEFE2D0006019F01B700B9E3
:10ED200000B0007DFFA201CE017D00A500D800A1AA
:10ED3000FF46FFFFFEC4FFCEFFFBFEECFEE6FE75C6
:10ED4000FF23FE34FEB6FE83FFCFFF27011A0184A6
:10ED500000C3FFBDFF1B003500D200BC007900409E
:10ED6000FFEDFEB4FD9CFDBEFD59FE13FFB9002D65
:10ED700000F4FF8F011E011601750257033502359D
:10ED800002AA014D018200A2FE30FE3EFF3FFEEBD3
:10ED9000FDCAFE98FE88FE68FF51004E017301C552
:10EDA000FFE5FF4C00A6008D002B002F00C5FFAF34
:10EDB000FFE5FF24FFE2FEABFFD8FF6200CE000DAF
:10EDC000018E006CFFAAFEEBFDE7FEDFFFBFFF85B3
:10EDD000FFA5FF03017301DEFF5DFF04FF69FFBBB9
:10EDE000000200A3FFE2FF61005D018B00E3FF3A38
:10EDF000008B0025006700C6008DFFE6FEB0FD0E0B
:10EE0000FD53FDECFD20FEB6FEF0FE68FF24008AF7
:10EE100000B101C6010102FD011B012B01D40098C4
:10EE2000009601E7011D01EC0066019200DDFF6321
:10EE3000FE8FFD98FDC8FC64FDAFFEE3FE2BFF30A6
:10EE400000720032000E00CA005601C3FF7C00FEB3
:10EE5000003D0041013C0206028D01F1001FFF1937
:10EE6000FFD7FE76FE82FEFFFE6FFEC3FDACFEBE48
:10EE7000FEC2FF29000800710038007101C401487A
:10EE80000151014101F2006300A40095FFDDFE394C
:10EE9000FE99FDC6FCF8FCADFD91FD25FEC4FEAF5C
:10EEA000FF3E00D5008601CA025A03EA026701DE6E
:10EEB00000E700D6FFFAFFB400C700C4FF66FF18E2
:10EEC000FF73FF69FF39FFE8FF73FFACFE32FF0EEF
:10EED000FF48FFBC00F3FF7C00E100B400000139F3
:10EEE00001F6009DFF96FF1BFF5EFF54FF25FEF11C
:10EEF000FE79FF3F00E1009600E3FF4AFF48FF75FF
:10EF0000FF3B00B0FF3AFF24FF78FFE6FF4900F621
:10EF1000FF3E000E00E1FF6100E1000B0256013FE1
:10EF20000014FF03FF67FF6100A60026002C0055B8
:10EF3000000700EFFFB0FF51FF03FFE7FEA5FFB39F
:10EF4000FFD1FF86FF18FF81FF2600CC0017013498
:10EF500000BCFF2CFFF9FE6EFF80FFA4FFFEFF9AAE
:10EF6000FF9CFF4500DD00510010004B00450031C3
:10EF70000019006901B800A400B70066005B008EAC
:10EF8000FF4DFFB0FFF8FF87FF65FF01FFC8FEBA26
:10EF9000FE75FEC7FE4CFF9EFF5F0018008D0065EA
:10EFA000018F011701F400F5003D004A00CEFF1863
:10EFB000FF5DFE2BFE8DFE20FFDCFE43FFB5FF183C
:10EFC000009C007A00A400A500410014007C00A36E
:10EFD0000031019D005D00D1FF6FFF59FFA7FEE8E2
:10EFE000FE73FEC1FEEFFF53009EFFE2FF5A009644
:10EFF000FF9AFF90000301EEFF3A000201CD005F8F
:10F000000179012101AA002E00B6FF4CFFF2FEDEBD
:10F01000FE91FEEBFDEEFD52FE92FEA9FE6CFFD3CB
:10F02000FF79FFD2FF03003E00E0003F015401667C
:10F030000153014B00BDFF73FFB0FFFDFF230050E4
:10F0400000FEFF390060008A00E0005C0093FF11C1
:10F05000FFEBFE64FF22FFBBFE7AFF3500FFFF4996
:10F060000086008C00C4FF52FFA8FF9BFF290014FC
:10F070000087FFAAFF07007000A6003A0035004E87
:10F080000037009BFF42FF93FFD2FFC6FF3D003DCC
:10F0900000C9FF49002F005900CA006400D7FFE8EB
:10F0A000FFF6FFABFF52FFD4FEE3FE0DFFB9FF41B9
:10F0B00000B9FFD7FFE0FF080081009E00BC009F61
:10F0C000008F004300ACFF3FFFB4FE97FED6FE0A60
:10F0D000FF1FFF5CFFC3FFE3FF61008F008D00B0E7
:10F0E000007700C1007B005D00A800B6009F005FB4
:10F0F000003000AAFFFDFFFFFF7DFFE0FFEBFFB147
:10F10000FFFAFFDFFF81FFF8FE90FEF3FEBFFFCEA8
:10F11000FF2B0063009F006C00D5FFBAFFA5FFD452
:10F12000FFADFFBFFFB2FFE4FFC9FFA5FF4AFF47E6
:10F13000FF31FF19FF5BFF65FF75FF4BFF4AFF596A
:10F14000FFA8FFAEFF8BFFBCFFF2FF0A00290034CF
:10F15000006100BA00E300EB00FE0009012801DCB9
:10F160000010010301E400DF0079001F007AFF16A0
:10F17000FFBCFE84FEFAFE79FF92FF92FF83FFED53
:10F18000FFF5FF1300CCFF24004A00040009002F04
:10F190000060005200B10087004F00DDFFA7FFB6FE
:10F1A000FFE1FF3100DAFF44FF8BFF97FF0C004ABD
:10F1B000005400570045000800AFFFCEFF74FFA5C4
:10F1C000FF99FFA0FF52FF0EFF2DFF8FFFDDFFFC19
:10F1D000FF44002E001E00380003004600C10061FD
:10F1E000008A00780061004600DCFFC3FFA4FFB581
:10F1F000FF1800F6FFD6FFC1FF48FF61FFAFFF29F0
:10F20000002A009EFF3AFF6BFF98FFF9FF3F0017AF
:10F21000003B004200F1FFD2FF1100F8FFCDFFC01C
:10F22000FF1E00E2FF86FFC3FFE7FFFFFF05001A96
:10F23000006D0091005F000200C0FF8BFF11FFB75F
:10F24000FED8FEEEFEE9FE72FFA0FFBDFF0B0055EB
:10F25000005F00B100B000D200BF0076008C000853
:10F260000027003F003B00EEFFB7FFD4FFE8FFE9B7
:10F27000FF93FF40FF55FF36FF58FF9AFF2DFF23F6
:10F28000FF65FF98FFF5FF2100510072006E0066D8
:10F29000003B005600530070001400FDFF240023C3
:10F2A00000390028001700D6FF97FF47FFFDFE003A
:10F2B000FF2EFF2FFF75FFBDFFEEFFE4FFDFFFC94D
:10F2C000FFDCFFF0FFD0FF20006600410054004A41
:10F2D00000FEFF0400D9FFCEFF190065002E00FBE1
:10F2E000FF290015001E003C00EDFFDAFFF3FF05CB
:10F2F00000A5FF56FF39FF53FFA6FF8BFFE0FFF08D
:10F30000FFFBFF1B00F6FFF9FFDEFFFBFF45004F91
:10F31000007C0079005C0048001C002300B8FFA1BD
:10F32000FF97FFBAFFECFFA9FFD9FF01002300EC14
:10F33000FFC3FF180024002C0068005C000D00C60D
:10F34000FF75FF47FF70FF97FFC1FFB1FFF7FF1E7B
:10F35000003200430028003A001E0040000A00DF8F
:10F36000FFE5FFB0FF76FF8DFF9EFFAAFFBAFFC843
:10F37000FFDDFF1E003A001D00F7FFFAFF200052DC
:10F380000058001700EDFFFEFF36002D001A0000A8
:10F3900000F1FFA8FF76FF67FF93FFA8FFD7FFD715
:10F3A000FFB6FFB6FFDFFF1B00FEFF35006E005308
:10F3B000003000EAFFDBFFF0FFCBFFC4FFB6FFCB5E
:10F3C000FFCEFFE1FF81FF76FFAAFFA6FFF1FF005E
:10F3D000000200EBFFD4FFEBFFFDFFBEFFC7FF32D3
:10F3E000004E002E00340076007B0072001500E80D
:10F3F000FF0000B2FFD7FFBAFF82FF4DFF63FF9708
:10F40000FFB4FFB5FFD5FFF5FFC4FFD7FFC5FFAFC2
:10F41000FFCCFFF4FFBEFFB7FFDEFFF8FF200021A7
:10F4200000FFFF0200FCFF1C001300050038004233
:10F4300000240031003B0043000E00C9FFCBFF9ABF
:10F44000FF7BFF32FF26FF21FF42FF73FF8EFFAFDE
:10F45000FFD6FF07001F002E0068005A004400641A
:10F46000003E0068005A004800410023001600ECEE
:10F47000FFC5FFDFFFD7FFECFF0300FEFF10001604
:10F480000024002D003400EAFFD2FF8FFF6BFF6FD6
:10F49000FF4AFF4BFF49FF87FFB5FFDFFF1D003A23
:10F4A000004D0046004C0046004D003B002200236A
:10F4B00000FDFF0400F6FFD8FFA2FF6CFF54FF2BF6
:10F4C000FF35FF5FFF8CFFB3FFF4FF050011001B4A
:10F4D00000290057005D0070005700340020000D27
:10F4E00000DEFFF4FF240027001F003F003A000069
:10F4F00000FCFFC0FF80FF5FFF45FF4DFF46FF564A
:10F50000FFB6FFD0FFD1FFF1FF1E002A001E00381A
:10F51000004A00490049004900490048004B0037B3
:10F5200000F3FFB4FF73FF32FF24FF23FF44FF7596
:10F53000FF9BFFEBFFFEFF17002800210029000CB6
:10F5400000FCFFE0FFBEFF9EFF8FFF96FF8EFFAF28
:10F55000FFB7FFC5FFEAFF070039005E0090009388
:10F560000092009300910095007B0058001600D98E
:10F57000FF94FF6AFF4CFF2AFF24FF17FF0DFF2AAD
:10F58000FF6CFF6BFF81FFB8FFD1FFE2FFD5FFEDFE
:10F59000FF1D0041004A007B009700900091006C25
:10F5A000006F006D005C0030000500F6FFD8FFB36F
:10F5B000FF99FF6FFF77FF80FF8EFFB2FFBFFFDC79
:10F5C000FFDCFFFAFF0500F8FFEFFF020019003F24
:10F5D000004C0047004C0042002500230028000991
:10F5E00000FEFF0100FAFFB1FFA8FFB9FF9FFFC2B5
:10F5F000FFDEFFD9FFE0FFD5FF0000100009001576
:10F60000000D00E6FFBFFFB1FFA0FFC1FFEDFF044B
:10F6100000FFFF000001001B003900500033000B09
:10F62000000400E8FFE3FFE0FFE7FFEDFFFBFFF270
:10F63000FFCBFFB1FFAFFFC9FFCBFFCAFFCCFFCAB3
:10F64000FFCEFFC9FFE3FF0500F4FFFAFF0300FE52
:10F65000FF0100FFFF0000010018002B001E000545
:10F6600000FFFF000000000000FFFFEDFFE7FFD3F9
:10F67000FFC6FFBEFFB0FFB7FFB2FFC2FFDAFFEC6D
:10F68000FFEDFFF8FF010003001500200021002816
:10F69000001E002000270017000D00F6FFF3FFEE0C
:10F6A000FFEEFFF6FFFFFF00000100F8FFF3FF0091
:10F6B00000FFFF0100FAFFF0FFEBFFEDFFECFFE4BE
:10F6C000FFECFFF5FFF9FF00000000000000000064
:10F6D00000FAFFF8FFF1FFEEFFEBFFEAFFF4FFF99E
:10F6E000FFFCFFFFFF0500090008000B000B0007EF
:10F6F0000006000500050002000000FFFFFFFFFFFD
:10F70000FFFEFFFEFFFFFF00004E414E494E4954F1
:10F7100059494E46CDCCCC3D0AD7233C17B7D138FA
:10F7200077CC2B329595E6241FB14F0A000020417B
:10F730000000C84200401C4620BCBE4CCA1B0E5AEA
:10F74000AEC59D7400407A10F35A00A0724E18099D
:10F750000010A5D4E80000E87648170000E40B5438
:10F76000020000CA9A3B000000E1F5050000809607
:10F770009800000040420F000000A0860100000039
:10F78000102700000000E8030000000064000000F3
:10F7900000000A00000000000100000000002C76BC
:10F7A000D888DC674F0823DFC1DFAE59E1B1B796D7
:10F7B000E5E3E453C63AE651997696E8E6C2842634
:10F7C000EB898C9B62ED407C6FFCEFBC9C9F40F210
:10F7D000BAA56FA5F490055A2AF75C936B6CF9678C
:10F7E0006DC11BFCE0E40D47FEF520E6B500D0ED51
:10F7F000902E0300943577050080841E08000020B9
:10F800004E0A000000C80C333333330F986E128356
:10F810001141EF8D2114893BE65516CFFEE6DB182A
:10F82000D1844B381BF77C1D901DA4BBE4242032EF
:10F8300084725E228100C9F124ECA1E53D27BED18E
:10F84000E1D1D1D2D5D211241FBECFEFCDBFDFE39E
:10F85000DEBF00E00CBF18BE19BE1ABE1BBE14E20C
:10F86000A0E0B0E2E2ECFAEC01E00BBF02C00790CE
:10F870000D92A832B107D9F71BBE2AE3A8E2B4E281
:10F8800001C01D92A03DB207E1F718EFC6E4D8EF22
:10F8900000E006C022970109FE010BBF0E9422DD95
:10F8A000CE33D10780E00807A9F70E94B7D10C94A6
:10F8B0005FE50C9400008FE10E943280019729F4EB
:10F8C00088ED84BF23E02093800008951F920F925B
:10F8D0000FB60F92112408B60F9218BE09B60F92F8
:10F8E00019BE0BB60F921BBE8F939F93AF93BF931E
:10F8F000EF93FF9380912C2490912D24A0912E249E
:10F90000B0912F240196A11DB11D80932C249093BA
:10F910002D24A0932E24B0932F249FE0E0E8F1E063
:10F92000908BFF91EF91BF91AF919F918F910F902D
:10F930000BBE0F9009BE0F9008BE0F900FBE0F9028
:10F940001F9018951F920F920FB60F92112408B6B0
:10F950000F9218BE09B60F9219BE8F939F93AF9363
:10F96000BF938091282490912924A0912A24B091BA
:10F970002B240196A11DB11D809328249093292446
:10F98000A0932A24B0932B24BF91AF919F918F9184
:10F990000F9009BE0F9008BE0F900FBE0F901F90E2
:10F9A0001895CF92DF92EF92FF928FB7F894209143
:10F9B00028243091292440912A2450912B24E0E4DA
:10F9C000F9E000A0F1A1E02D8FBFC0902C24D090D1
:10F9D0002D24E0902E24F0902F24A8EEB3E00E9476
:10F9E000E4DC6E0F7F1F811D911D6C0D7D1D8E1D32
:10F9F0009F1DFF90EF90DF90CF9008952F923F9240
:10FA00004F925F926F927F928F929F92AF92BF922E
:10FA1000CF92DF92EF92FF920F931F932FB7F8943C
:10FA2000609128247091292480912A2490912B247C
:10FA3000E0E4F9E080A091A0E0E0F9E0A0A0B1A0AE
:10FA40002FBFB694A794B694A79420E432E44FE075
:10FA500050E00E94F7DC29013A01B62FA72FF82FBA
:10FA6000292E950140E050E060E070E080E090E0F9
:10FA700052016301EB2EFA2E0F2F122D0E9427DD6B
:10FA800079018B01782EB92E9401A8EEB3E00E9483
:10FA9000CEDC1B012C019701B801872D9B2D510154
:10FAA0006201E12CF12C00E010E00E9427DD1F91A3
:10FAB0000F91FF90EF90DF90CF90BF90AF909F900D
:10FAC0008F907F906F905F904F903F902F90089510
:10FAD0008F929F92AF92BF92CF92DF92EF92FF925E
:10FAE000CF93DF938FB7F89480902C2490902D249F
:10FAF000A0902E24B0902F242091282430912924E6
:10FB000040912A2450912B24E0E0F9E000A0F1A1DB
:10FB1000E02DA0E4B9E09096CD91DC9191978FBF54
:10FB2000F695E795F695E79560E472E48FE090E04E
:10FB30000E943BDC6B017C01CE0EDF1EE11CF11C40
:10FB40008C0E9D1EA11CB11CA8EEB3E0A501940172
:10FB50000E94E4DCC60ED71EE81EF91EC701B601DE
:10FB6000DF91CF91FF90EF90DF90CF90BF90AF905B
:10FB70009F908F9008958F929F92AF92BF92CF9255
:10FB8000DF92EF92FF926C010E94687D4B015C0155
:10FB9000E12CF12C0E94687D681979098A099B097A
:10FBA000C616D706E806F906A8F7FF90EF90DF9093
:10FBB000CF90BF90AF909F908F9008958F929F921B
:10FBC000AF92BF92CF92DF92EF92FF926B017C01D6
:10FBD0000E94D17C4B015C010E94D17C681979099B
:10FBE0008A099B09C616D706E806F906A8F7FF900A
:10FBF000EF90DF90CF90BF90AF909F908F9008953F
:10FC0000789480E1809355002091500020612093EA
:10FC100050003091510034FFFCCF48ED44BF50916B
:10FC20004000587F54605093400062E160936D0043
:10FC30007AE770936E00A1E0A093680094E090933F
:10FC40000009E0EAFFE0E0933609F0933709B0914C
:10FC50000109B87FB0930109F2E0F093060988E04A
:10FC60008093400928EE33E020937609309377099A
:10FC700030914109387F3093410940E54093430971
:10FC8000F093460957E8509387016FEF6093B000F7
:10FC900070E17093100610920006109201027093AA
:10FCA00002021092030296E0909304021092060260
:10FCB000A093200210922202A0932302A09300029C
:10FCC0006093B00070933006109220066093B000ED
:10FCD000109250066093B000109270066093B000CE
:10FCE0001092900642E050E06BE57CE78FE10E94C5
:10FCF000AE80A091A200A760A093A200789408957E
:10FD00008093002008958C3028F5E82FF0E0EA5227
:10FD1000F94F85919491909100209295907F9093C6
:10FD2000020220E120930102880F880F880F809340
:10FD3000210280912002806880932002309123026A
:10FD400030FFFCCF41E0409323028091100290915C
:10FD5000110208958FEF9FEF08950E94837E97FF11
:10FD600002C080E090E09595879508950E94837E7B
:10FD7000BC01882777FD8095982F3CE0660F771FA0
:10FD8000881F991F3A95D1F708950E94837E44E019
:10FD9000880F991F4A95E1F708950E94837EBC0160
:10FDA000882777FD8095982F0E94BFD921E038E001
:10FDB00040E859E30E9473DA08957F928F929F92F0
:10FDC000AF92BF92CF92DF92EF92FF920F931F9369
:10FDD000CF93DF93782E5B01E82FF0E0E95CF84FDA
:10FDE0008491282F30E0220F331FF901EB5EF84F8A
:10FDF00005911491F901ED50F94FC591D491E82F77
:10FE0000F0E0EE51F94FC590D4902C54394FF901E0
:10FE1000E590F49061E0872D0E94647F0115110543
:10FE2000A1F04FEF50E0E8014EAB5FAB55E05883D7
:10FE3000698167606983D98020E130E001C0220FC9
:10FE4000CA94EAF7D22AD98214C0209791F02FEFF2
:10FE500030E02EAB3FAB15E0188339813760398332
:10FE6000998020E130E001C0220FCA94EAF7922A7B
:10FE70009982E114F10489F0F701A082B182DF9147
:10FE8000CF911F910F91FF90EF90DF90CF90BF9097
:10FE9000AF909F908F907F900895F0E8AF16B104D7
:10FEA00014F460E001C061E0872DDF91CF911F91D4
:10FEB0000F91FF90EF90DF90CF90BF90AF909F9009
:10FEC0008F907F900C94B47FEF92FF921F93CF930B
:10FED000DF931F92CDB7DEB7E82EF12CF701E75A7A
:10FEE000F84F1491812F69830E948E80F701E558A5
:10FEF000F84FE4916981EE2381F1F0E0EE0FFF1FEE
:10FF0000E356F84FA591B491AD01405F5F4F9FB7A5
:10FF1000F894282F30E0611103C012961C9316C08C
:10FF2000633041F412961C93FA01E20FF31F8081B3
:10FF3000806111C0623041F412961C93FA01E20F05
:10FF4000F31F8081886107C011961C93FA01E20FAC
:10FF5000F31F8081877C80839FBF0F90DF91CF91BB
:10FF60001F91FF90EF900895CF92DF92EF92FF9252
:10FF70001F93CF93DF931F92CDB7DEB7E82EF12CFE
:10FF8000F701E75AF84F1491812F69830E948E8000
:10FF9000F701E95CF84F7491F701E558F84F949137
:10FFA0006981992309F455C0772391F1272F30E017
:10FFB000220F331FF901EB5EF84FC590D4902D50FE
:10FFC000394FF901A591B491E72FF0E0EE51F94FC7
:10FFD000E590F490C114D10461F0F601F18020E1C4
:10FFE00030E001C0220FEA94EAF720952F21218307
:10FFF0000FC0109769F01196DC90119720E130E066
:020000021000EC
:1000000001C0220FEA94EAF720952D2111962C9336
:10001000E92FF0E0EE0FFF1FE356F84FA591B491E2
:100020002FB7F894EC90E12261F4509690E0A80F7D
:10003000B91F8C91611102C0877E01C088618C93C9
:1000400007C0611103C016961C9302C015961C933D
:100050002FBF0F90DF91CF911F91FF90EF90DF9016
:10006000CF9008950F931F93CF93DF9390E0FC01FF
:10007000E95CF84F4491FC01E75AF84F6491FC01A8
:10008000E558F84F8491882309F441C0442381F155
:10009000242F30E0220F331FF901EB5EF84FC5919A
:1000A000D4912D50394FF901A591B491E42FF0E08E
:1000B000EE51F94F45915491209759F0198120E163
:1000C00030E001C0220F4A95EAF7209521232983C9
:1000D0000FC0109769F011969C91119720E130E0C4
:1000E00001C0220F4A95EAF72095292311962C93F7
:1000F000E82FF0E0EE0FFF1FE356F84FC591D491C3
:100100002885262381E090E021F480E002C080E091
:1001100090E0DF91CF911F910F9108958031A1F070
:1001200038F4843069F0883069F0823039F414C0D2
:10013000803471F0803871F0803241F080E00895B1
:1001400082E0089583E0089584E0089585E00895AD
:1001500086E0089587E0089581E00895AF92BF9208
:10016000CF92DF92EF92FF920F931F93CF93DF9383
:100170006B01803308F04BC04530510540F4FA0163
:10018000E659FE4D0081112707FD109502C000E0E1
:1001900010E090E09C012558384F5901F901149165
:1001A000212F30E0220F331F2356384FF901C5911C
:1001B000D491AC01475A584F7A01FA0184910E94B8
:1001C0008E80F501A491B0E0119753E0AA0FBB1FF8
:1001D0005A95E1F7A80FB11DAA0FBB1FAA5CBB4D32
:1001E000CD92DC92998594609987BB84F701C49085
:1001F000CB28CB86FE017096E80FF11D8081802B05
:100200008083D884E12FF0E0E05DFB4DD082DF9168
:10021000CF911F910F91FF90EF90DF90CF90BF9003
:10022000AF900895CF92DF92EF92FF920F931F93BA
:10023000CF93DF93803308F03EC0082F10E0C80151
:100240008558984F7C01FC01249130E0220F331F28
:100250002356384FF901C591D4916E01F0E1CF0ECC
:10026000D11C075A184FF80184910E948E80F70123
:10027000A491B0E01197E3E0AA0FBB1FEA95E1F764
:10028000A80FB11DAA0FBB1FAA5CBB4D1D921C92EB
:100290009B85F8010491009509230B87FB84E82FC7
:1002A000F0E0F11003C01985137F1987EC0DFD1DD7
:1002B0002081287F2083DF91CF911F910F91FF90A4
:1002C000EF90DF90CF9008956F927F929F92AF92C0
:1002D000BF92CF92DF92EF92FF920F931F93CF9333
:1002E000DF93FC01EE0FFF1FE356F84FC591D49149
:1002F000D884FC01E05DFB4DC0800197A82EAA0CBC
:10030000AA0CAA0CD0828E01005F1F4FB12C992439
:1003100093942B2D2A0D3D2D3170632F692570E0AC
:100320008C2D8170A82FA925B0E0882311F03B0106
:1003300002C0612C712C109741F091E0E12C311139
:1003400001C090E0492F5E2D02C040E050E0F8016E
:1003500081918F01877030E0220F331FF901EA5C31
:10036000FB4DE080F180EF28A1F0811104C0A617B9
:10037000B70731F50EC0813019F4452B09F509C0D6
:10038000823019F46728E1F404C0833011F4672B3C
:10039000B9F4D694C694B394F8E0BF12BACF1C85D2
:1003A0001D7F1C87DF91CF911F910F91FF90EF90E0
:1003B000DF90CF90BF90AF909F907F906F90089507
:1003C000F901EA5CFB4D0190F081E02D1995E1CF38
:1003D0001F920F920FB60F92112408B60F9218BEFB
:1003E00009B60F9219BE0BB60F921BBE2F933F9307
:1003F0004F935F936F937F938F939F93AF93BF932D
:10040000EF93FF9381E090E00E946481FF91EF9170
:10041000BF91AF919F918F917F916F915F914F911C
:100420003F912F910F900BBE0F9009BE0F9008BE09
:100430000F900FBE0F901F9018951F920F920FB63E
:100440000F92112408B60F9218BE09B60F9219BE6A
:100450000BB60F921BBE2F933F934F935F936F93F7
:100460007F938F939F93AF93BF93EF93FF9382E01C
:1004700090E00E946481FF91EF91BF91AF919F91B5
:100480008F917F916F915F914F913F912F910F903D
:100490000BBE0F9009BE0F9008BE0F900FBE0F90BD
:1004A0001F9018951F920F920FB60F92112408B645
:1004B0000F9218BE09B60F9219BE0BB60F921BBE53
:1004C0002F933F934F935F936F937F938F939F935C
:1004D000AF93BF93EF93FF9383E090E00E9464811A
:1004E000FF91EF91BF91AF919F918F917F916F910C
:1004F0005F914F913F912F910F900BBE0F9009BECE
:100500000F9008BE0F900FBE0F901F9018951F926E
:100510000F920FB60F92112408B60F9218BE09B6AB
:100520000F9219BE0BB60F921BBE2F933F934F93A2
:100530005F936F937F938F939F93AF93BF93EF934B
:10054000FF9384E090E00E946481FF91EF91BF915E
:10055000AF919F918F917F916F915F914F913F915B
:100560002F910F900BBE0F9009BE0F9008BE0F90F9
:100570000FBE0F901F9018951F920F920FB60F92FB
:10058000112408B60F9218BE09B60F9219BE0BB609
:100590000F921BBE2F933F934F935F936F937F9365
:1005A0008F939F93AF93BF93EF93FF9385E090E07A
:1005B0000E946481FF91EF91BF91AF919F918F91C4
:1005C0007F916F915F914F913F912F910F900BBE53
:1005D0000F9009BE0F9008BE0F900FBE0F901F9096
:1005E00018958091500082608093500020915100B6
:1005F00021FFFCCF309156003460309356004BE120
:100600004093650057EB5093660062E06093CA0127
:10061000EDE1F0E0E491E0936200ECE1F0E0749150
:10062000709363001092CA0191E0909360000C9463
:100630003AD508950895CF93DF9381E090E20E9428
:10064000EDD5811119C0C5E0D0E061E085E10E94DF
:10065000B47F62E370E080E090E00E94DE7D60E0C5
:1006600085E10E94B47F62E370E080E090E00E9448
:10067000DE7D2197209749F7DF91CF910895089566
:100680000E947F8F80E00E94E2910C94F69E7F9200
:100690008F929F92AF92BF92CF92DF92EF92FF9292
:1006A0000F931F93CF93DF93E82EF12C2FE1829FBE
:1006B000F0011124E65AF94D608380912721709052
:1006C000B833833011F47720E9F0C0EFD6E2E3EEDF
:1006D000F6E28CED882E86E2982E80E090E07FEFA7
:1006E000E71AF70A062F10E0A801440F551F445CD3
:1006F0005E4D30E3B32EAA24A394000F111F0B5AB2
:100700001E4D16C08090BA338820F9F241C06E01A8
:10071000ACE0CA1AD108D601DC90D1100DC0019608
:10072000E096F096B0E38B0E911C8530910581F137
:10073000288130E07110EBCF2E153F0581F7DA01EB
:100740002D913C91D40115962D933C931697B89E0C
:100750009001B99E300D11242A52394DD901989635
:100760001D921C9299979A961D921C929B97D40168
:100770001D921D921D921C9213976D3038F0A0822D
:10078000D801CD90DC90C282D382C9CF1082C7CF6E
:10079000DF91CF911F910F91FF90EF90DF90CF905D
:1007A000BF90AF909F908F907F9008950F931F936D
:1007B000CF93DF9380914626C091B424D0E081117D
:1007C00081C08091D12490E00E942E9A0FE10C9F6D
:1007D000F0010D9FF00D1124E65AF94D838B948B97
:1007E000C091B424D0E08091CE2490E00E942E9A53
:1007F0000C9FF0010D9FF00D1124E65AF94D818FE9
:10080000928FC091B424D0E08091C22490E00E94E5
:100810002E9A0C9FF0010D9FF00D1124E65AF94D10
:10082000818B928B8091C02490E00E942E9A9595A6
:100830008795959587958093AC249093AD2445E05A
:100840004093BE244093BD24409312204093B7248C
:1008500050912721523049F48091C82490E00E94A1
:100860002E9A809398249093992460912721633045
:1008700009F087C08091CA2490E00E942E9A80934C
:100880009C2490939D248091C52490E00E942E9AF0
:100890008093962490939724C091B424D0E08091C3
:1008A000C62490E00E942E9A7FE17C9FF0017D9FFC
:1008B000F00D1124E65AF94D838F948F95E09093B3
:1008C000B8245FC08091D02490E00E942E9A0FE15E
:1008D0000C9FF0010D9FF00D1124E65AF94D858B08
:1008E000968BC091B424D0E08091CF2490E00E94F8
:1008F0002E9A0C9FF0010D9FF00D1124E65AF94D30
:10090000878B908F15E01093BC241093BB24C0916B
:10091000B424D0E08091C32490E00E942E9A0C9FD2
:10092000F0010D9FF00D1124E65AF94D858F968F39
:1009300028E22093B5248091C12490E00E942E9A51
:1009400080939E2490939F248091BF2490E00E94E6
:100950002E9A9595879595958795809310209093DD
:1009600011201093B62430912721323061F4809108
:10097000C92490E00E942E9A80939A2490939B24FD
:1009800002C0C0E001C0C1E0A0912721A150A23067
:10099000D8F4D0E08091CD2490E00E942E9ACC0F24
:1009A000DD1FFE01EC55FB4D808391838091CC24AB
:1009B00090E00E942E9AC056DB4D88839983B5E063
:1009C000B093BA24B093B924DF91CF911F910F91C6
:1009D000089583E00E94E0998823E1F081E09091FE
:1009E0004626911180E080934626882389F021E0F5
:1009F000209345260E94D17C68537F4F8F4F9F4F95
:100A000060933E2670933F26809340269093412624
:100A10000C94D683089580930E2090930F2040EC81
:100A2000489F9001499F300D1124C9016CE370E08B
:100A30000E9457DC9B0140E050E060E079E08DE3EC
:100A400090E00E947FDCE0E0FAE026A337A308955F
:100A50002F923F924F925F926F927F928F929F92CE
:100A6000AF92BF92CF92DF92EF92FF920F931F93BC
:100A7000CF93DF9300D0CDB7DEB70E94099502E394
:100A800016E232E4C32E36E2D32EF12CF801808137
:100A90009181A281B381892B8A2B8B2BC9F00E9473
:100AA000D17CF80180809180A280B380681579059F
:100AB0008A059B05E0F031E0F6019081911130E06C
:100AC000D6013C93F80110821182128213820FC06A
:100AD00020912721223019F42090173104C02330AF
:100AE00021F42090B433F21411F0D6011C92F39447
:100AF0000C5F1F4FBFEFCB1ADB0A44E0F412C6CFE6
:100B0000309046263320D9F040903E2650903F2624
:100B10006090402670904126411451046104710494
:100B200071F40E94D17C68537F4F8F4F9F4F609329
:100B30003E2670933F26809340269093412684EB77
:100B400096E30E9432C78111FACF81EE98E30E94AA
:100B500034C88111FACF0E94759F1091272111305E
:100B600009F041C18091CB2490E00E942E9A3C0173
:100B7000BC01882777FD8095982F1F921F921F92A6
:100B800054E05F93A12CB12C6501E12C14E0F12E0F
:100B900000E010E020E030E0A9010E94F6B90091E9
:100BA000B2241091B3240619170917FF03C0119539
:100BB000019511090F900F900F900F9006301105BD
:100BC0000CF47EC02091B42430E02617370709F4D6
:100BD00077C06093B4246092B2247092B3240E94D0
:100BE000D6837091B42455245394570EB1E5CB2E7F
:100BF000B6E2DB2E60E010E3FFE17F9F500111249D
:100C0000C501865A994D1C01EE24E394D6014C91FE
:100C10004F3FB9F150E0149FF001159FF00D1124E2
:100C2000EA52F94D738C76122CC0D1010C91802FB1
:100C300090E09C01220F331F245C3E4DD9018D9022
:100C40009C908386948610A611A612A613A61682DF
:100C50001782108611860D3058F0E586880F991F8F
:100C60008B5A9E4DDC016D907C906786708A01C026
:100C70001586149FF001159FF00D1124EA52F94DCD
:100C8000528E6F5FB4E0CB0ED11C633009F0BECF43
:100C9000072F10E0F801EE5BF94DB1E0B0830E9440
:100CA000D17CF801EE0FFF1FEE0FFF1FEE5CF94D38
:100CB00068537F4F8F4F9F4F6083718382839383ED
:100CC00090904626992009F48CC08091C32490E02E
:100CD0000E942E9A2C01B090B4244B2D50E09FE13D
:100CE000B99EF0011124E65AF94DC58CD68CB2019B
:100CF0006C197D095B0177FF03C0B194A194B10821
:100D00006091B52470E06A157B050CF06AC032E092
:100D10003093B5247FE1749FF001759FF00D11248D
:100D2000E65AF94D458E568EA2014E565140473C2B
:100D3000510508F447C0B201882777FD8095982FA8
:100D4000BEE64B16B1E05B06C4F41F921F921F92E1
:100D50001F92A12CE4E0BE2EC12CD12C1DE6E12E69
:100D6000FF24F39400E010E020E030E0A9010E94AD
:100D7000F6B971956195710914C01F921F9254E0E4
:100D80005F931F92A12CB12C6501EE24EA9413E02D
:100D9000F12E00E010E025E332E040E050E00E9458
:100DA000F6B90F900F900F900F90882777FD8095E0
:100DB000982F0E94BFD920E030E040E85AE30E941B
:100DC00073DA03C060E070E0CB01D090B4241FE17F
:100DD000D19EF0011124E65AF94D65877687878701
:100DE000908B0E949FA4F0912721F23009F0DAC085
:100DF000F0904626F11055C08091C82490E00E94E2
:100E00002E9ABC018090982490909924DC01A81916
:100E1000B909B7FF03C0B195A195B109A630B105D5
:100E20000CF480C0609398247093992420910C3125
:100E3000882777FD8095982F2430D1F01F921F923C
:100E40001F9230E63F9335E1A32EB12CC12CD12C5B
:100E5000EE24EA9413E0F12E00E010E020E030E010
:100E6000A9010E94F6B9609316310E94D0AB56C01A
:100E70001F921F921F92B0E6BF93B5E1AB2EB12C2B
:100E8000C12CD12CEE24EA9413E0F12E00E010E006
:100E900020E030E0A9010E94F6B9862F0E94AEAA98
:100EA0003DC08091C92490E00E942E9A1C0180913F
:100EB0009A2490919B247101E81AF90A8701F7FEA0
:100EC00003C0119501951109063011055CF1B101BE
:100ED000882777FD8095982F20911831309119310E
:100EE0008901222717FD2095322F3F932F931F93BF
:100EF0000F93F2E0AF2EB12CC12CD12CE12C14E0D9
:100F0000F12E00E010E020E030E0A9010E94F6B9E7
:100F10006093153120929A2430929B240F900F9069
:100F20000F900F908091CA2490E00E942E9ABC01ED
:100F300060909C2470909D24AC014619570957FF7E
:100F400003C0519541955109463051054CF13090FF
:100F50000C28311025C060939C2470939D24882711
:100F600077FD8095982F1F921F9221E02F932CE2FE
:100F70002F9354E1A52EB12CC12CD12CEE24EA9450
:100F800013E0F12E00E010E020E030E0A9010E9423
:100F9000F6B9CB010E940B850F900F900F900F9028
:100FA0000E9402AD90912721933009F0E5C1809114
:100FB000C72490E00E942E9A2C012090B2243090F9
:100FC000B324281A390A37FE03C03194219431081A
:100FD0001F921F921F9264E06F93A12CB12C6501A8
:100FE000E12C14E0F12E00E010E020E030E0A90157
:100FF000B201882777FD8095982F0E94F6B96B0182
:101000007C010F900F900F900F9056E02516310441
:101010000CF461C08091B42490E08C159D0509F416
:101020005AC07090B63376E0779EF0011124E45EEA
:10103000FE4C908058E2959E800111248AE0789EB3
:10104000000D111D11240C5C1E4CD8011496BC908F
:1010500020E3B29ED0011124AA52B94D5B968C9127
:101060005B97871115C05596BC91B43089F0F1811A
:10107000F13031F440E0F80160818F5F0E94C49F3D
:10108000A090BA33A11004C0F80184810E94FCA290
:10109000C092B4244092B2245092B324C092B6338A
:1010A0000E94D6830091B42410E0F801EE5BF94D64
:1010B00031E030830E94D17CF801EE0FFF1FEE0F6C
:1010C000FF1FEE5CF94D68537F4F8F4F9F4F60833A
:1010D0007183828393838091CA2490E00E942E9A28
:1010E0004C01C0909C24D0909D247C01EC18FD08FC
:1010F000A701F7FE03C051954195510946305105AE
:1011000054F150900C28511026C0B401882777FD67
:101110008095982F1F921F9211E01F935CE25F93BE
:1011200014E1A12EB12CC12CD12CEE24EA9413E0B1
:10113000F12E00E010E020E030E0A9010E94F6B9B5
:10114000CB010E940B8580929C2490929D240F904D
:101150000F900F900F908091C02490E00E942E9AE3
:1011600095958795959587956090AC247090AD2462
:101170002C0146185708120157FE03C031942194E0
:1011800031084091B72450E042155305A4F4109261
:10119000B7248093AE249093AF248093AC24909393
:1011A000AD24D090AB24D11006C080933E289093FC
:1011B0003F280E9423A98091C62490E00E942E9A85
:1011C000BC01F090B4242F2D30E09FE1F99EF00196
:1011D0001124E65AF94D038D148DCB01801B910B20
:1011E000DC0197FF03C0B195A195B109623071058B
:1011F00014F460E070E04091B82450E04A175B07B7
:10120000C4F08091C52490E00E942E9A1C01609148
:101210009624709197245C01A61AB70AA501B7FE1F
:1012200003C0519541955109443051050CF047C018
:10123000A1C083E08093B8248FE1829FF001839F57
:10124000F00D1124E65AF94D638F748FF090B63388
:10125000882777FD8095982F0E94BFD928E030E23B
:1012600040E85AE30E9473DA26E0F29EF00111246E
:10127000E45EFE4C62837383848395834091BA332A
:10128000E1EFF6E20DEF16E251E030803F1449F055
:101290009F012D503109D9017C90711002C041117C
:1012A00006C06783708781879287D8015C93F09628
:1012B000005D1F4FB7E2E13EFB0739F7A2CF709107
:1012C000BA33772309F456C081E08093B533B10176
:1012D000882777FD8095982F1F921F921F92E0E636
:1012E0009E2E9F92F5E1AF2EB12CC12CD12CEE2475
:1012F000EA9413E0F12E00E010E020E030E0A901D4
:101300000E94F6B92B013C016091962470919724BC
:10131000882777FD8095982F1F921F921F929F928A
:1013200020E030E0A9010E94F6B9461A570A20923F
:1013300096243092972424E331E3CDBFDEBF80E0D2
:1013400090E0F901E80FF91FB081BF3F31F08180D3
:101350009280840C951C8182928288968038F2E07B
:101360009F0779F7265F3F4F41E32C35340739F764
:101370001092B5330E949AB090904626911051C0B9
:101380008091C22490E00E942E9A1C01B090B42457
:101390003FE1B39EF0011124E65AF94D018912890B
:1013A0004C01801A910A97FE03C091948194910890
:1013B0001F921F921F9212E11F93A12CB12C650165
:1013C000E12C14E0F12E00E010E020E030E0A90173
:1013D000B101882777FD8095982F0E94F6B920915A
:1013E000122030E00F900F900F900F9028153905C4
:1013F0000CF060C05090B4245FE1559EF0011124C0
:10140000E65AF94D208130E02617370709F452C01B
:1014100092E090931220218A328A852D0E94478380
:1014200049C08091C12490E00E942E9A2C01C09066
:101430009E24D0909F243C016C187D0877FE03C049
:101440007194619471081F921F921F92F5E0FF93AF
:10145000A12CB12C6501E12C14E0F12E00E010E08C
:1014600020E030E0A901B201882777FD8095982F10
:101470000E94F6B90F900F900F900F90B6E06B1688
:101480007104C4F020911B2830E02617370791F033
:1014900040929E2450929F2460931B28E62FF0E0F8
:1014A000EE0FFF1FEE5CFE4DE080F180E092192808
:1014B000F0921A28D0904626D110A4C08091D12451
:1014C00090E00E942E9A2C019090B424FFE19F9E00
:1014D000F0011124E65AF94DE388F4884C018E1886
:1014E0009F0897FE03C09194819491081F921F92C8
:1014F00011E01F9354EF5F93A12CB12C6501A394CD
:10150000EE24EA9413E0F12E00E010E022E030E057
:1015100040E050E0B201882777FD8095982F0E9427
:10152000F6B90F900F900F900F9032E043165104D0
:1015300014F460E070E08091BE2490E08815990575
:1015400074F41092BE24B090B4249FE1B99EF001CF
:101550001124E65AF94D61837283438A548A80913B
:10156000CE2490E00E942E9A3C015090B4242FE1AA
:10157000529EF0011124E65AF94D618D728D1C01C5
:10158000261A370A37FE03C03194219431081F927E
:101590001F9241E04F9384EF8F93A12CB12C6501F2
:1015A000A394EE24EA9413E0F12E00E010E022E090
:1015B00030E040E050E0B301882777FD8095982F18
:1015C0000E94F6B90F900F900F900F90A2E06A164C
:1015D000710414F460E070E08091BD2490E0821505
:1015E00093050CF0BBC01092BD24D090B424BFE191
:1015F000DB9EF0011124E65AF94D61877287618EF6
:10160000728EACC08091D02490E00E942E9A2C0162
:10161000F090B4242FE1F29EF0011124E65AF94D26
:10162000A589B6893C016A1A7B0A77FE03C07194CA
:10163000619471081F921F9261E06F9344EF4F9382
:10164000A12CB12C6501A394EE24EA9413E0F12EB1
:1016500000E010E022E030E040E050E0B2018827F6
:1016600077FD8095982F0E94F6B90F900F900F90FC
:101670000F9032E04316510414F460E070E0809162
:10168000BC2490E08615970574F41092BC24309029
:10169000B4248FE1389EF0011124E65AF94D63839A
:1016A0007483458A568A8091CF2490E00E942E9AB6
:1016B0001C017090B424E72CF12C7FE1779EF0019F
:1016C0001124E65AF94DA788B08C6C01CA18DB08C2
:1016D0008601D7FE03C01195019511092091BB2405
:1016E00030E020173107D4F51092BB24B1018827D0
:1016F00077FD8095982F0E94BFD92FE632E143E80D
:101700005AE30E9473DABFE1BE9D8001BF9D100DB8
:101710001124065A194D5B016C0120E030E040E8CD
:101720005FE30E9420D9181634F4A12CB12CF0E804
:10173000CF2EAFE3DA2EA501B601D80115964D9351
:101740005D936D937C9318973FE13E9DF0013F9D23
:10175000F00D1124E65AF94D278A308E7091272119
:101760007150723008F05BC1F0904626F1102FC026
:101770008091C02490E00E942E9A9595879595952A
:1017800087954090AC245090AD247C01E418F50876
:101790004701F7FE03C09194819491084091B724CA
:1017A00050E048155905E4F51092B7248093AE2413
:1017B0009093AF248093AC249093AD243090AB24CD
:1017C00031102EC080933E2890933F2827C08091EF
:1017D000BF2490E00E942E9A9595879595958795C0
:1017E000A0901020B09011206C01CA18DB0886016F
:1017F000D7FE03C01195019511094091B62450E020
:10180000401751076CF4A1E0A093B62480931020F8
:101810009093112080933C2890933D280E9423A907
:101820002224239470904626711001C0212C8091AF
:10183000CD2490E00E942E9A8A839B832C016624FB
:1018400057FC6094762C1F921F9233E03F93FFEF7A
:10185000FF93A12CB12C6501EE24EA9413E0F12E44
:1018600000E010E025E030E040E050E0C301B201CC
:101870000E94F6B9312C4101880C991CF401EC55F9
:10188000FB4D208131816A817B81621B730BAB012F
:1018900077FF03C05195419551092091BA2430E05A
:1018A0000F900F900F900F90241735070CF066C023
:1018B0001092BA24F401EC55FB4D8A819B81808300
:1018C0009183F101E655FB4D8101000F111F000FBF
:1018D000111F18161906F4F55081511105C0D401D5
:1018E000AB5EB74D1D921C9291E09083AA80BB80A5
:1018F000A114E2E0BE067CF49801245D374D790125
:10190000C301B2010E94BFD928E230E540E25DE3A5
:101910000E9473DA19C0F801E45DF74D7F016A8116
:101920007B817250882777FD8095982F0E94BFD9C0
:1019300022E334E648E45FE30E9473DA20E030E01B
:1019400040EA51E40E94BCD8F7016083718382832E
:10195000938301C01082F801EC5DF74D20E030E088
:10196000A90160817181828193810E9420D98111B6
:1019700005C0F401E056FB4D108211828091CC2409
:1019800090E00E942E9A3C01BC01882777FD80954B
:10199000982F1F921F9213E01F93BFEFBF9324E174
:1019A000A22EB12CC12CD12CEE24EA9413E0F12EFE
:1019B00000E010E020E030E0A9010E94F6B9F40157
:1019C000E056FB4DC080D1806C187D0877FE03C0C7
:1019D0007194619471082091B92430E00F900F90B8
:1019E0000F900F9026153705D4F41092B924810179
:1019F000000F111F000F111F0C5D174D882777FD79
:101A00008095982F0E94BFD920E030E040E05AE353
:101A10000E9473DAF80160837183828393839090CC
:101A2000AA24992019F080E00E949FA1B090AB24D5
:101A3000BB2019F081E00E949FA15090AB2455205B
:101A400079F1209128283091292840912A28509115
:101A50002B28609120287091212880912228909134
:101A600023280E9473DA20E030E040E053E40E9433
:101A700073DA0E948CD94091AE245091AF24460F66
:101A8000571F4F3F510519F014F04FEF50E057FF2B
:101A900002C040E050E040933E2850933F280CC0E5
:101AA0002090A924222051F00091AE241091AF245F
:101AB00000933E2810933F280E9423A9D090AA2487
:101AC000D092A8247091AB247093A92413EEA12E78
:101AD00016E2B12E00EF802E06E2902E1A821B82B3
:101AE000FA80F98260E3EA80FB806E9DF0016F9DD1
:101AF000F00D1124EA52F94D3081323008F462C100
:101B000080912721813039F4D401EC91EF77F0E016
:101B1000EF5BF94D808350E34A805B80549D8001E8
:101B2000559D100D11240A52194DF8013080F4E032
:101B30003F9EF0011124E258FB4D2081318142810A
:101B40005381F801228333834483558389810E9422
:101B5000AFA6D5017C90711075C0F40180818F779C
:101B600090E00197BFE1B89FF001B99FF00D1124FB
:101B7000E65AF94DC584D684E784F08820E030E049
:101B8000A901C701B6010E9420D9882309F45AC0CF
:101B9000D80112962D903D904D905C90159720E0C5
:101BA00030E0A901C701B6010E9420D987FF16C005
:101BB000F801808190E046971CF04081415001C0BF
:101BC00045E174E0479FF0011124E258FB4D20816C
:101BD000318142815381C201B10116C0F801808177
:101BE00090E08C3691051CF490819F5F01C09CE6CB
:101BF00014E0919FF0011124E258FB4DA2019101E4
:101C000060817181828193810E94BBD8A701960176
:101C10000E9473DA30E36A807B80369D8001379DB5
:101C2000100D11240A52194DD80112962D913D9193
:101C30004D915C9115970E94BCD8F8016283738323
:101C400084839583D5015C90511081C0F40180811B
:101C50008F7790E001976FE1689FF001699FF00D29
:101C60001124E65AF94D238434842114310409F4F3
:101C70006EC080E3EA80FB808E9DF0018F9DF00DA9
:101C80001124EA52F94D628173818481958120810A
:101C900030E037FE18C0273131051CF0208122507A
:101CA00001C025E1B4E02B9FF0011124E258FB4D67
:101CB00020813181428153810E94BBD820E030E0F5
:101CC00040E059E319C02B3631051CF450815E5FAA
:101CD00001C05CE6F4E05F9FF0011124E258FB4D87
:101CE0009B01AC0160817181828193810E94BBD88C
:101CF00020E034E040E059E30E9473DA6B017C019C
:101D000090E34A805B80949D8001959D100D112485
:101D10000A52194DD80112964D905D906D907C90AD
:101D20001597B101882777FD8095982F0E94BFD91C
:101D30009B01AC01C701B6010E9473DAA3019201B5
:101D40000E94BCD8F8016283738384839583D0900A
:101D5000AA24DD20A1F1D501FC90F11030C040E3B0
:101D60006A807B80469D8001479D100D11240A5298
:101D7000194DF801628173818481958122803380BD
:101D80004480558020911C2830911D2840911E28A8
:101D900050911F280E9473DA209124283091252821
:101DA00040912628509127280E9473DAA2019101C0
:101DB0000E94BCD8F80162837383848395838981F0
:101DC0000E9499A56A817B816F5F7F4F6A837B83C5
:101DD00030E3A30EB11C40E3840E911C8A819B81E9
:101DE0008530910509F07CCE07E111E2B2E4AB2E1B
:101DF000B6E2BB2ED5016D915D01F80181918F0195
:101E00000E94B47FF6E4AF16F6E2BF0699F7239678
:101E1000CDBFDEBFDF91CF911F910F91FF90EF906B
:101E2000DF90CF90BF90AF909F908F907F906F90FA
:101E30005F904F903F902F9008951F920F920FB692
:101E40000F92112408B60F9218BE09B60F9219BE50
:101E50000BB60F921BBE2F933F934F935F936F93DD
:101E60007F938F939F93AF93BF93EF93FF9381E003
:101E700090910D20911180E080930D20882341F1F5
:101E800020912721233031F43091B533311120C016
:101E90000E945EB140912721423031F450911B31B4
:101EA0005523B1F00E9493A96091C6277091C7276E
:101EB0008091C8279091C9276F5F7F4F8F4F9F4FA9
:101EC0006093C6277093C7278093C8279093C9272C
:101ED000FF91EF91BF91AF919F918F917F916F9102
:101EE0005F914F913F912F910F900BBE0F9009BEC4
:101EF0000F9008BE0F900FBE0F901F901895CF93B4
:101F0000DF9362E08CE00E94647F62E08DE00E94DB
:101F1000647F62E08FE00E94647F62E08EE00E9456
:101F2000647F61E088E10E94647F61E089E10E9452
:101F3000647F61E084E10E94647F61E085E10E944A
:101F4000647F83E00E94807E85E08093200310926E
:101F5000210310922203C0E0D0E0C0933803D09355
:101F600039038AE090E00E94BB7D2196C11588E08C
:101F7000D80799F721E020930008109201081092E9
:101F80000208109203081092040840E055E04093C4
:101F900026085093270833E0309306082093400822
:101FA000109241081092420810924308109244087F
:101FB00060E07DE7609366087093670820934608A9
:101FC00054E05093000A1092010A1092020A1092F3
:101FD000030A1092040AA0EBB8E2A093260AB09379
:101FE000270A2093060ADF91CF9108951F93CF937C
:101FF000DF9311E0C7E1D1E2612F89910E94B47FA4
:1020000081E2CB31D807C1F7DAE080E00E94E099A5
:102010008823A9F0C7E1D1E260E089910E94B47FF2
